:020000040000FA
:1000000000040020810A000015070000610A0000BA
:100010001F07000029070000330700000000000050
:10002000000000000000000000000000A50A000021
:100030003D070000000000004707000051070000D6
:100040005B070000650700006F07000079070000EC
:10005000830700008D07000097070000A10700003C
:10006000AB070000B5070000BF070000C90700008C
:10007000D3070000DD070000E7070000F1070000DC
:10008000FB070000050800000F0800001908000029
:10009000230800002D080000370800004108000078
:1000A0004B080000550800005F08000069080000C8
:1000B000730800007D080000870800009108000018
:1000C0009B080000A5080000AF080000B908000068
:1000D000C3080000CD080000D7080000E1080000B8
:1000E000EB080000F5080000FF0800000909000007
:1000F000130900001D090000270900003109000054
:100100003B0900001FB500F003F88DE80F001FBD8C
:1001100000F0ACBC40F6FC7108684FF01022401CA7
:1001200008D00868401C09D00868401C04D0086842
:1001300000F037BA9069F5E79069F9E7704770B554
:100140000B46010B184400F6FF70040B4FF0805073
:100150000022090303692403406943431D1B104621
:1001600000F048FA29462046BDE8704000F042BA47
:10017000F0B54FF6FF734FF4B4751A466E1E11E0DA
:10018000A94201D3344600E00C46091B30F8027B3B
:10019000641E3B441A44F9D19CB204EB134394B25D
:1001A00004EB12420029EBD198B200EB134002EBB2
:1001B000124140EA0140F0BDF34992B00446D1E952
:1001C0000001CDE91001FF224021684600F0F4FB58
:1001D00094E80F008DE80F00684610A902E004C8FB
:1001E00041F8042D8842FAD110216846FFF7C0FF7C
:1001F0001090AA208DF8440000F099F9FFF78AFFCB
:1002000040F6FC7420684FF01025401C0FD0206889
:1002100010226946803000F078F92068401C08D030
:100220002068082210A900F070F900F061F9A869AF
:10023000EEE7A869F5E74FF080500369406940F6A2
:10024000FC71434308684FF01022401C06D0086838
:1002500000F58050834203D2092070479069F7E788
:100260000868401C04D00868401C03D00020704778
:100270009069F9E70420704770B504460068C34DE3
:10028000072876D2DFE800F033041929631E250021
:10029000D4E9026564682946304600F062F92A46CE
:1002A0002146304600F031F9AA002146304600F0E0
:1002B00057FB002800D0032070BD00F009FC4FF46C
:1002C000805007E0201D00F040F90028F4D100F034
:1002D000FFFB60682860002070BD241D94E80700C3
:1002E000920000F03DFB0028F6D00E2070BDFFF715
:1002F000A2FF0028FAD1D4E901034FF0805100EBAE
:10030000830208694D69684382420ED840F6F8704E
:1003100005684FF010226D1C09D0056805EB8305B8
:100320000B6949694B439D4203D9092070BD55694A
:10033000F4E70168491C03D00068401C02D003E0C8
:100340005069FAE70F2070BD2046FFF735FFFFF731
:1003500072FF0028F7D1201D00F0F7F80028F2D135
:1003600060680028F0D100F0E2F8FFF7D3FE00F05B
:10037000BFF8072070BD10B50C46182802D0012028
:10038000086010BD2068FFF777FF206010BD41684E
:10039000054609B1012700E0002740F6F8742068FF
:1003A0004FF01026401C2BD02068AA68920000F065
:1003B000D7FA38B3A86881002068401C27D020688D
:1003C000FFF7BDFED7B12068401C22D026684FF051
:1003D0008050AC686D68016942695143A9420DD9EA
:1003E000016940694143A14208D92146304600F0E5
:1003F000B8F822462946304600F087F800F078F831
:100400007069D2E700F093F8FFF784FEF6E77069B1
:10041000D6E77669DBE740F6FC7420684FF01026DB
:10042000401C23D02068401C0CD02068401C1FD0EA
:100430002568206805F18005401C1BD027683879A5
:10044000AA2819D040F6F8700168491C42D001680A
:10045000491C45D00168491C3ED001680968491C07
:100460003ED00168491C39D000683EE0B069DAE747
:10047000B569DEE7B769E2E710212846FFF778FEA5
:100480003968814222D12068401C05D0D4F8001080
:1004900001F18002C03107E0B169F9E730B108CA63
:1004A00051F8040D984201D1012000E000208A4259
:1004B000F4D158B1286810B1042803D0FEE72846CB
:1004C000FFF765FF3149686808600EE0FFF722FE1C
:1004D00000F00EF87169BBE77169BFE7706904E06D
:1004E0004FF480500168491C01D000F0CBFAFEE7C0
:1004F000BFF34F8F26480168264A01F4E06111439B
:100500000160BFF34F8F00BFFDE72DE9F0411746B3
:100510000D460646002406E03046296800F054F8EF
:10052000641C2D1D361DBC42F6D3BDE8F08140F69B
:10053000FC700168491C04D0D0F800004FF48051D1
:10054000FDE54FF010208069F8E74FF080510A690F
:10055000496900684A43824201D810207047002050
:10056000704770B50C4605464FF4806608E0284693
:1005700000F017F8B44205D3A4F5806405F5805562
:10058000002CF4D170BD0000F40A0000000000202F
:100590000CED00E00400FA05144801680029FCD0C5
:1005A0007047134A0221116010490B68002BFCD0E0
:1005B0000F4B1B1D186008680028FCD0002010603D
:1005C00008680028FCD07047094B10B501221A605A
:1005D000064A1468002CFCD0016010680028FCD08A
:1005E0000020186010680028FCD010BD00E4014015
:1005F00004E5014070B50C46054600F073F810B9EB
:1006000000F07EF828B121462846BDE8704000F091
:1006100007B821462846BDE8704000F037B8000012
:100620007FB5002200920192029203920A0B000B06
:100630006946012302440AE0440900F01F0651F80C
:10064000245003FA06F6354341F82450401C8242F8
:10065000F2D80D490868009A10430860081D016827
:10066000019A1143016000F03DF800280AD00649C4
:1006700010310868029A10430860091D0868039A3F
:10068000104308607FBD00000006004030B50F4CED
:10069000002200BF04EB0213D3F800582DB9D3F8A1
:1006A000045815B9D3F808581DB1521C082AF1D3C3
:1006B00030BD082AFCD204EB0212C2F80008C3F8CD
:1006C00004180220C3F8080830BD000000E0014013
:1006D0004FF08050D0F83001082801D0002070473A
:1006E000012070474FF08050D0F83011062905D016
:1006F000D0F83001401C01D0002070470120704725
:100700004FF08050D0F830010A2801D00020704707
:100710000120704708208F490968095808471020B0
:100720008C4909680958084714208A4909680958FA
:100730000847182087490968095808473020854923
:100740000968095808473820824909680958084744
:100750003C20804909680958084740207D490968BC
:100760000958084744207B49096809580847482028
:1007700078490968095808474C207649096809589A
:10078000084750207349096809580847542071499F
:1007900009680958084758206E49096809580847E8
:1007A0005C206C4909680958084760206949096854
:1007B00009580847642067490968095808476820AC
:1007C00064490968095808476C2062490968095852
:1007D000084770205F4909680958084774205D4937
:1007E00009680958084778205A490968095808478C
:1007F0007C205849096809580847802055490968EC
:10080000095808478420534909680958084788202F
:1008100050490968095808478C204E490968095809
:10082000084790204B4909680958084794204949CE
:10083000096809580847982046490968095808472F
:100840009C204449096809580847A0204149096883
:1008500009580847A4203F49096809580847A820B3
:100860003C49096809580847AC203A4909680958C1
:100870000847B0203749096809580847B420354966
:10088000096809580847B8203249096809580847D3
:10089000BC203049096809580847C0202D4909681B
:1008A00009580847C4202B49096809580847C82037
:1008B0002849096809580847CC2026490968095879
:1008C0000847D0202349096809580847D4202149FE
:1008D000096809580847D8201E4909680958084777
:1008E000DC201C49096809580847E02019490968B3
:1008F00009580847E4201749096809580847E820BB
:100900001449096809580847EC2012490968095830
:100910000847F0200F49096809580847F4200D4995
:10092000096809580847F8200A490968095808471A
:10093000FC2008490968095808475FF48070054998
:10094000096809580847000003480449024A034B54
:100950007047000000000020000B0000000B0000AA
:1009600040EA010310B59B070FD1042A0DD310C82C
:1009700008C9121F9C42F8D020BA19BA884201D97E
:10098000012010BD4FF0FF3010BD1AB1D30703D0C6
:10099000521C07E0002010BD10F8013B11F8014B7C
:1009A0001B1B07D110F8013B11F8014B1B1B01D198
:1009B000921EF1D1184610BD02F0FF0343EA032254
:1009C00042EA024200F005B87047704770474FF0A6
:1009D00000020429C0F0128010F0030C00F01B800C
:1009E000CCF1040CBCF1020F18BF00F8012BA8BF1A
:1009F00020F8022BA1EB0C0100F00DB85FEAC17CDE
:100A000024BF00F8012B00F8012B48BF00F8012B90
:100A100070474FF0000200B51346944696462039C1
:100A200022BFA0E80C50A0E80C50B1F12001BFF4A7
:100A3000F7AF090728BFA0E80C5048BF0CC05DF80D
:100A400004EB890028BF40F8042B08BF704748BF5B
:100A500020F8022B11F0804F18BF00F8012B7047CF
:100A6000014B1B68DB6818470000002009480A4951
:100A70007047FFF7FBFFFFF745FB00BD20BFFDE719
:100A8000064B1847064A1060016881F308884068E1
:100A900000470000000B0000000B000017040000DE
:100AA000000000201EF0040F0CBFEFF30881EFF3ED
:100AB0000981886902380078182803D100E0000015
:100AC000074A1047074A12682C3212681047000084
:100AD00000B5054B1B68054A9B58984700BD0000B0
:100AE0007703000000000020F00A0000040000006E
:100AF000001000000000000000FFFFFF0090D00386
:10100000C01300202151020005C1000087500200DA
:1010100005C1000005C1000005C10000000000007E
:10102000000000000000000000000000AD510200C0
:1010300005C100000000000005C1000005C100005E
:10104000155202001B52020005C1000005C100003C
:1010500005C1000005C1000005C1000005C1000078
:101060002152020005C1000005C100002752020004
:1010700005C100002D520200335202003952020015
:1010800005C1000005C1000005C1000005C1000048
:1010900005C1000005C1000005C1000005C1000038
:1010A00005C100003F52020005C1000005C100005B
:1010B00005C1000005C1000005C1000005C1000018
:1010C0004552020005C1000005C1000005C1000035
:1010D00005C1000005C1000005C1000005C10000F8
:1010E00005C1000005C1000005C1000005C10000E8
:1010F00005C1000005C1000005C1000005C10000D8
:1011000005C1000005C1000000F002F823F0F7FF60
:101110000AA090E8000C82448344AAF10107DA4552
:1011200001D123F0ECFFAFF2090EBAE80F0013F083
:10113000010F18BFFB1A43F00103184700460200D5
:10114000204602000A444FF0000C10F8013B13F057
:10115000070408BF10F8014B1D1108BF10F8015B10
:10116000641E05D010F8016B641E01F8016BF9D103
:1011700013F0080F1EBF10F8014BAD1C0C1B09D15A
:101180006D1E58BF01F801CBFAD505E014F8016BCC
:1011900001F8016B6D1EF9D59142D6D3704700005E
:1011A0000023002400250026103A28BF78C1FBD870
:1011B000520728BF30C148BF0B6070471FB500F011
:1011C00003F88DE80F001FBD23F096BF70B51A4CD1
:1011D00005460A202070A01C00F0D5F85920A080F8
:1011E00029462046BDE8704008F078B908F081B97A
:1011F00070B50C461149097829B1A0F160015E294A
:1012000008D3012013E0602804D0692802D043F2FB
:1012100001000CE020CC0A4E94E80E0006EB8000A2
:10122000A0F58050241FD0F8806E2846B04720607B
:1012300070BD012070470000080000201C00002045
:10124000885202003249884201D2012070470020B2
:10125000704770B50446A0F500002E4EB0F1786FCF
:1012600002D23444A4F500042948844201D2012565
:1012700000E0002500F043F848B125B9B44204D39A
:101280002548006808E0012070BD002070BD002DD9
:10129000F9D1B442F9D321488442F6D2F3E710B52C
:1012A0000446A0F50000B0F1786F03D21948044459
:1012B000A4F5000400F023F84FF0804130B1164847
:1012C000006804E08C4204D2012003E01348844209
:1012D000F8D2002080F0010010BD10B520B1FFF75A
:1012E000DEFF08B1012010BD002010BD10B520B1F7
:1012F000FFF7AFFF08B1012010BD002010BD084866
:1013000008490068884201D10120704700207047D9
:1013100000600200000000202000002008000020E3
:101320005C000020BEBAFECA10B5044600210120B0
:1013300000F042F800210B2000F03EF800210820C8
:1013400000F03AF80421192000F036F804210D20AD
:1013500000F032F804210E2000F02EF804210F20B6
:1013600000F02AF80421C84300F026F806211620D0
:1013700000F022F80621152000F01EF82046FFF7A5
:1013800025FF002010BD4FF4927101807047FFF7D8
:101390002DBF1148704710487047104A10B51468A7
:1013A0000E4B0F4A08331A60FFF722FF0B48001D4F
:1013B000046010BD704770474907090E002804DB20
:1013C00000F1E02080F80014704700F00F0000F1F9
:1013D000E02080F8141D704703F900421005024018
:1013E00001000001FD48002101604160018170475A
:1013F0002DE9FF4F93B09B46209F160004460DD069
:101400001046FFF726FF18B1102017B0BDE8F08F87
:101410003146012001F0D3FE0028F6D101258DF8D8
:1014200042504FF4C050ADF84000002210A92846A9
:1014300006F0BBFC0028E8D18DF84250A8464FF4D6
:1014400028500025ADF840001C2229466846079523
:101450000CF0DDFF9DF81C000DF11C0A20F00F00C0
:10146000401C20F0F00010308DF81C0020788DF822
:101470001D0061789DF81E000DF1400961F34200E6
:1014800040F001008DF81E009DF8000008AA40F011
:1014900002008DF800002089ADF83000ADF8325020
:1014A0006089ADF83400CDF82CA060680E900AA9D0
:1014B000CDF82890684606F086FA0028A5D1606825
:1014C000FFF70BFF40B16068FFF710FF20B96078AD
:1014D00000F00300022801D0012000E00020BF4CF2
:1014E00008AA0AA92072BDF8200020808DF8428049
:1014F00042F60120ADF840009DF81E0020F00600E5
:10150000801C20F001008DF81E000220ADF8300094
:10151000ADF8340014A80E90684606F054FA00287E
:1015200089D1BDF82000608036B1211D304600F021
:101530005FF90028C2D109E0BBF1000F05D00CF023
:10154000E1FCE8BB0CF0DEFCD0BBA58017B1012F9D
:1015500043D04AE08DF8428042F6A620ADF8400024
:1015600046461C220021684607950CF050FF9DF866
:101570001C00ADF8346020F00F00401C20F0F0009B
:1015800010308DF81C009DF81D0020F0FF008DF834
:101590001D009DF81E0020F0060040F00100801C98
:1015A0008DF81E009DF800008DF8446040F00200A8
:1015B0008DF80000CDE90A9AADF8306011A800E07E
:1015C00011E00E9008AA0AA9684606F0FCF9002866
:1015D000A6D1BDF82000E08008E00CF093FC10B923
:1015E0000CF090FC08B103200FE7E58000200CE729
:1015F0003EB50446794D0820ADF80000A88828B112
:101600002046FFF726FE18B110203EBD06203EBD45
:101610002146012001F0D3FD0028F8D12088ADF843
:1016200004006088ADF80600A088ADF80800E088E6
:10163000ADF80A00A88801AB6A46002106F0A0FDBB
:10164000BDF800100829E2D003203EBD7FB5634DF0
:101650000446A88868B1002002900820ADF8080070
:10166000CDF80CD02046FFF7F4FD20B1102004B0D7
:1016700070BD0620FBE7A98802AA4FF6FF7006F0AE
:10168000C2FF0028F3D1BDF80810082901D00320BB
:10169000EDE7BDF800102180BDF802106180BDF8B3
:1016A0000410A180BDF80610E180E0E701B582B02A
:1016B0000220ADF80000494802AB6A46408800218C
:1016C00006F05EFDBDF80010022900D003200EBD1B
:1016D0001CB5002100910221ADF800100190FFF728
:1016E000DEFD08B110201CBD3C486A4641884FF61B
:1016F000FF7006F088FFBDF800100229F3D0032028
:101700001CBDFEB5354C06461546207A0F46C0076F
:1017100005D00846FFF79DFD18B11020FEBD0F2033
:10172000FEBDF82D01D90C20FEBD3046FFF791FD1E
:1017300018BB208801A905F030FE0028F4D13078CC
:101740008DF80500208801A906F0F9FC0028EBD1EE
:1017500000909DF800009DF8051040F002008DF803
:101760000000090703D040F008008DF80000208831
:10177000694606F081FC0028D6D1ADF808502088D3
:101780003B4602AA002106F0FBFCBDF80810A94266
:10179000CAD00320FEBD7CB5054600200090019014
:1017A0000888ADF800000C4628460195FFF795FD26
:1017B00018B92046FFF773FD08B110207CBD15B1A4
:1017C000BDF8000060B105486A4601884FF6FF7019
:1017D00006F019FFBDF8001021807CBD2402002016
:1017E0000C20FAE72F48C088002800D0012070475D
:1017F00030B5044693B000200D46014600901422F7
:1018000001A80CF004FE1C22002108A80CF0FFFD2A
:101810009DF80000CDF808D020F00F00401C20F00B
:10182000F00010308DF800009DF8010006AA20F0AD
:10183000FF008DF801009DF8200001A940F0020092
:101840008DF8200001208DF8460042F60420ADF806
:10185000440011A801902088ADF83C006088ADF8E4
:101860003E00A088ADF84000E088ADF842009DF849
:10187000020020F00600801C20F001008DF802001C
:101880000820ADF80C00ADF810000FA8059008A8CE
:1018900006F099F8002803D1BDF818002880002030
:1018A00013B030BD24020020F0B5007B059F1E461A
:1018B00014460D46012800D0FFDF0C2030803A206E
:1018C0003880002C08D0287A032806D0287B0128ED
:1018D00000D0FFDF17206081F0BDA889FBE72DE96C
:1018E000F0470D4686B095F80C900E991446B9F164
:1018F000010F0BD01022007B2E8A9046052807D0BE
:10190000062839D0FFDF06B0BDE8F0870222F2E7F3
:10191000E8890C2200EB400002EB400018803320E5
:101920000880002CEFD0E8896081002720E0009635
:10193000688808F1020301AA696900F097FF06EBC5
:101940000800801C07EB470186B204EB4102BDF89A
:1019500004009081F848007808B1012300E00023DA
:101960000DF1060140460E3213F0C5FD7F1CBFB2DB
:101970006089B842DBD8C6E734200880E889B9F12D
:10198000010F11D0122148430E301880002CBAD01C
:10199000E88960814846B9F1010F00D00220207328
:1019A00000270DF1040A1FE00621ECE70096688885
:1019B00008F1020301AA696900F058FF06EB08006C
:1019C000801C86B2B9F1010F12D007EBC70004EBFF
:1019D0004000BDF80410C18110220AF1020110304C
:1019E0000CF0EBFC7F1CBFB26089B842DED88AE7FE
:1019F00007EB470104EB4102BDF80400D0810AF176
:101A000002014046103213F098FDEBE72DE9F04754
:101A10000E4688B090F80CC096F80C80378AF5898D
:101A20000C20DFF81493109902F10C04BCF1030FA1
:101A300008D0BCF1040F3DD0BCF1070F75D0FFDF1B
:101A400008B061E705EB850C00EB4C0018803120F5
:101A50000880002AF4D0A8F1060000F0FF0A5581A2
:101A600024E01622002101A80CF0D1FC0097708818
:101A7000434601AA716900F0F9FEBDF80400208018
:101A8000BDF80600E080BDF80800208199F800004C
:101A900008B1012300E00023A21C0DF10A01504609
:101AA00013F029FD07EB080087B20A346D1EADB2B2
:101AB000D7D2C5E705EB850C00EB4C00188032202F
:101AC0000880002ABCD0A8F1050000F0FF0A55816B
:101AD00037E000977088434601AA716900F0C6FE9E
:101AE0009DF80600BDF80410E1802179420860F3FA
:101AF000000162F34101820862F38201C20862F3CD
:101B0000C301020962F30411420962F3451182091B
:101B100062F386112171C0096071BDF80700208150
:101B200099F8000010B1012301E00EE000232246E5
:101B30000DF10901504613F0DEFC07EB080087B2F7
:101B40000A346D1EADB2C4D27AE7A8F1020084B2A5
:101B500005FB08FC0CF10E00188035200880002AD7
:101B6000A7D05581948100971FFA8CF370880E32AC
:101B7000716900F07BFE63E72DE9F84F1E460A9D70
:101B80000C4681462AB1607A00F58070D080E089E9
:101B9000108199F80C000C274FF000084FF00E0A46
:101BA0000D2872D2DFE800F09D070E1B272F374566
:101BB000546972727200214648460095FFF774FE20
:101BC000BDE8F88F207B9146082802D0032800D07A
:101BD000FFDF3780302009E0A9F80A80F0E7207B9A
:101BE0009146042800D0FFDF378031202880B9F1EA
:101BF000000FF1D1E4E7207B9146042800D0FFDFFD
:101C000037803220F2E7207B9146022800D0FFDFA8
:101C100037803320EAE7207B1746022800D0FFDF19
:101C20003420A6F800A02880002FC9D0A7F80A8089
:101C3000C6E7207B1746042800D0FFDF3520A6F832
:101C400000A02880002FBBD04046A7F80A8012E0F1
:101C5000207B1746052802D0062800D0FFDF102081
:101C6000308036202880002FAAD0E0897881A7F81C
:101C70000E80B9F80E00B881A2E7207B91460728B4
:101C800000D0FFDF37803720B0E72AE04FF01200A6
:101C900018804FF038001700288091D0E0897881B3
:101CA000A7F80E80A7F8108099F80C000A2805D034
:101CB0000B2809D00C280DD0FFDF81E7207B0A28F4
:101CC00000D0FFDF01200AE0207B0B2800D0FFDFDF
:101CD000042004E0207B0C2800D0FFDF05203873AF
:101CE0006EE7FFDF6CE770B50C46054601F0AAFB16
:101CF00020B10078222804D2082070BD43F20200EF
:101D000070BD0521284611F06DFE206008B100204D
:101D100070BD032070BD30B44880087820F00F00FB
:101D2000C01C20F0F000903001F8080B1DCA81E8BB
:101D30001D0030BC07F053BC100000202DE9FF4708
:101D400084B0002782460297079890468946123051
:101D50000AF029FA401D20F00306079828B907A9C0
:101D60005046FFF7C0FF002854D1B9F1000F05D04D
:101D70000798017B19BB052504681BE098F8000053
:101D8000092803D00D2812D0FFDF46E0079903256C
:101D90004868B0B3497B42887143914239D98AB2CD
:101DA000B3B2011D11F091FC0446078002E0079CCC
:101DB000042508340CB1208810B1032D29D02CE063
:101DC0000798012112300AF020FAADF80C00024603
:101DD00002AB2946504608F0A8FA070001D1A01C22
:101DE000029007983A461230C8F80400A8F802A0FA
:101DF00003A94046029B0AF015FAD8B10A2817D267
:101E000000E006E0DFE800F007091414100B0D14E1
:101E10001412132014E6002012E6112010E6082008
:101E20000EE643F203000BE6072009E60D2007E665
:101E3000032005E6BDF80C002346CDE900702A46D4
:101E40005046079900F022FD57B9032D08D1079895
:101E5000B3B2417B406871438AB2011D11F049FC65
:101E6000B9F1000FD7D0079981F80C90D3E72DE98D
:101E7000FE4F91461A881C468A468046FAB102AB4C
:101E8000494608F052FA050019D04046A61C27889A
:101E900011F0EBFE3246072629463B46009611F02C
:101EA000FAFA20882346CDE900504A46514640467A
:101EB00000F0ECFC002020800120BDE8FE8F002017
:101EC000FBE710B586B01C46AAB104238DF800309C
:101ED0001388ADF808305288ADF80A208A788DF85A
:101EE0000E200988ADF80C1000236A462146FFF742
:101EF00025FF06B010BD1020FBE770B50D4605218B
:101F000011F070FD040000D1FFDF294604F112003A
:101F1000BDE870400AF062B92DE9F8430D468046ED
:101F2000002607F059FB04462878102878D2DFE80D
:101F300000F0773B345331311231313108313131D6
:101F400031312879001FC0B2022801D0102810D1E9
:101F500014BBFFDF35E004B9FFDF0521404611F077
:101F600041FD007B032806D004280BD0072828D089
:101F7000FFDF072655E02879801FC0B2022820D055
:101F800050B1F6E72879401FC0B2022819D01028B6
:101F900017D0EEE704B9FFDF13E004B9FFDF2879BB
:101FA00001280ED1172137E00521404611F01AFD16
:101FB000070000D1FFDF07F1120140460AF0EBF8FD
:101FC0002CB12A4621464046FFF7A5FE29E0132101
:101FD000404602F019FD24E004B9FFDF0521404628
:101FE00011F000FD060000D1FFDF694606F1120086
:101FF0000AF0DBF8060000D0FFDFA988172901D21C
:10200000172200E00A46BDF80000824202D90146CC
:1020100002E005E01729C5D3404600F047FCD0E7B1
:10202000FFDF3046BDE8F883401D20F0030219B100
:1020300002FB01F0001D00E000201044704713B5C2
:10204000009858B10024684611F0E9FA002C04D138
:10205000F749009A4A6000220A701CBD0124002042
:10206000F2E72DE9F0470C461546242200212046D0
:102070000CF0CDF905B9FFDFA87860732888DFF888
:10208000B0A3401D20F00301AF788946DAF80400C0
:1020900011F0E3FA060000D1FFDF4FF000082660E0
:1020A000A6F8008077B109FB07F1091D0AD0DAF81C
:1020B000040011F0D2FA060000D1FFDF6660C6F816
:1020C000008001E0C4F80480298804F11200BDE812
:1020D000F0470AF051B82DE9F047804601F11200AF
:1020E0000D4681460AF05FF8401DD14F20F00302F3
:1020F0006E7B14462968786811F0DAFA3EB104FB69
:1021000006F2121D03D06968786811F0D1FA052033
:1021100011F010FC0446052011F014FC201A0128CF
:1021200002D1786811F08EFA49464046BDE8F04782
:102130000AF038B870B50546052111F053FC0400CB
:1021400000D1FFDF04F112012846BDE870400AF01B
:1021500022B82DE9F04F91B04FF0000BADF828B048
:10216000ADF804B047880C4605469246052138462E
:1021700011F038FC060000D1FFDF24B1A780A4F8DD
:1021800006B0A4F808B0297809220B20B2EB111F81
:1021900073D12A7A04F1100138274FF00C084FF060
:1021A00012090291102A69D2DFE802F068F2F1F018
:1021B0008008D3898EA03DDCF3EEB7B7307B0228D0
:1021C00000D0FFDFA88908EBC001ADF80410302172
:1021D000ADF82810002C25D06081B5F80E800027BE
:1021E0001DE004EBC709317C89F80E10F189A9F8CC
:1021F0000C10CDF800806888042305AA296900F036
:1022000035FBBDF81410A9F8101008F10400BDF852
:1022100016107F1C1FFA80F8A9F81210BFB260894F
:10222000B842DED80CE1307B022800D0FFDFE9891C
:1022300008EBC100ADF804003020ADF8280095F897
:102240000C90002CA9F10400C0B20F90EAD061817B
:10225000B5F81080002725E0CDF8008068884B464F
:1022600003AA696900F002FB08EB09001FFA80F875
:102270006F48007818B1012302E0DDE0DAE00023C6
:1022800004EBC702009204A90C320F9813F033F943
:10229000009ABDF80C007F1C1082009ABDF80E0059
:1022A000BFB250826089B842D6D8C9E00AA800906F
:1022B00001AB224629463046FFF711FBC0E0307BD8
:1022C000082805D0FFDF03E0307B082800D0FFDFBF
:1022D000E8891030ADF804003620ADF82800002C55
:1022E0003FD0A9896181F189A18127E0307B09284C
:1022F00000D0FFDFA88901460C30ADF8040037207C
:10230000ADF82800002C2CD06181E8890090AB89C1
:10231000688804F10C02296955E0E88939211030F8
:1023200080B2ADF80400ADF82810002C72D0A98955
:102330006181287A0E280AD002212173E989E1817E
:10234000288A0090EB8968886969029A3BE001213C
:10235000F3E70AA8009001AB224629463046FFF772
:1023600055FB6DE0307B0A2800D0FFDFADF804900C
:10237000ADF828704CB3A9896181A4F810B0A4F815
:102380000EB0012020735BE020E002E030E038E096
:1023900041E0307B0B2800D0FFDF288AADF82870A1
:1023A0001230ADF8040084B104212173A989618140
:1023B000E989E181298A2182688A00902B8A6888CC
:1023C00004F11202696900F051FA39E0307B0C28FF
:1023D00000D0FFDFADF80490ADF828703CB30521C4
:1023E0002173A4F80AB0A4F80EB0A4F810B027E046
:1023F0000AA8009001AB224629463046FFF754FA5E
:102400001EE00AA8009001AB224629463046FFF79D
:10241000B3FB15E034E03B21ADF80400ADF8281023
:1024200074B30120E080A4F808B084F80AB007E093
:1024300010000020FFDF03E0297A012917D0FFDF19
:10244000BDF80400AAF800006CB1BDF82800208097
:10245000BDF804006080BDF82800392803D03C286E
:1024600001D086F80CB011B00020BDE8F08F3C21FF
:10247000ADF80400ADF8281014B1697AA172DFE755
:10248000AAF80000EFE72DE9F84356880F4680468A
:1024900015460521304611F0A5FA040000D1FFDFF2
:1024A000123400943B46414630466A6809F0EEFF1C
:1024B000B8E570B50D46052111F094FA040000D17D
:1024C000FFDF294604F11200BDE8704009F078BE34
:1024D00070B50D46052111F085FA040000D1FFDF2B
:1024E000294604F11200BDE8704009F096BE70B5AF
:1024F0000546052111F076FA040000D1FFDF04F152
:10250000080321462846BDE870400422AFE470B5B8
:102510000546052111F066FA040000D1FFDF2146CF
:1025200028462368BDE870400522A0E470B5064641
:10253000052111F057FA040000D1FFDF04F1120069
:1025400009F031FE401D20F0030511E0011D008857
:102550000322431821463046FFF789FC00280BD0A0
:10256000607BABB2684382B26068011D11F0F7F87E
:10257000606841880029E9D170BD70B50E460546F6
:1025800007F02AF8040000D1FFDF012020726672F4
:102590006580207820F00F00C01C20F0F000303063
:1025A0002070BDE8704007F01AB8602801D00720FD
:1025B00070470878C54900F0010008700020704796
:1025C0002DE9F0438BB00D461446814606A9FFF76E
:1025D0008AFB002814D14FF6FF7601274FF42058CC
:1025E0008CB103208DF800001020ADF8100007A872
:1025F000059007AA204604A912F0A1FF78B1072090
:102600000BB0BDE8F0830820ADF808508DF80E70CF
:102610008DF80000ADF80A60ADF80C800CE006986B
:10262000A17801742188C1818DF80E70ADF8085031
:10263000ADF80C80ADF80A606A4602214846069B58
:10264000FFF77CFBDCE708B501228DF8022042F69B
:102650000202ADF800200A4603236946FFF731FC69
:1026600008BD08B501228DF8022042F60302ADF83C
:1026700000200A4604236946FFF723FC08BD00B585
:1026800087B079B102228DF800200A88ADF80820C1
:102690004988ADF80A1000236A460521FFF74EFB72
:1026A00007B000BD1020FBE709B1072309E40720AC
:1026B000704770B588B00D461446064606A9FFF768
:1026C00012FB00280ED17CB10620ADF808508DF821
:1026D0000000ADF80A40069B6A460821DC813046BE
:1026E000FFF72CFB08B070BD05208DF80000ADF899
:1026F0000850F0E700B587B059B107238DF80030D6
:10270000ADF80820039100236A460921FFF716FB64
:10271000C6E71020C4E770B588B00C460646002511
:1027200006A9FFF7E0FA0028DCD106980121123053
:1027300009F06BFD9CB12178062921D2DFE801F078
:10274000200505160318801E80B2C01EE28880B2E4
:102750000AB1A3681BB1824203D90C20C2E7102042
:10276000C0E7042904D0A08850B901E00620B9E7E9
:10277000012913D0022905D004291CD005292AD00B
:102780000720AFE709208DF800006088ADF8080049
:10279000E088ADF80A00A068039023E00A208DF8D5
:1027A00000006088ADF80800E088ADF80A00A06875
:1027B0000A25039016E00B208DF800006088ADF824
:1027C0000800A088ADF80A00E088ADF80C00A06809
:1027D0000B25049006E00C208DF8000060788DF841
:1027E00008000C256A4629463046069BFFF7A6FAE4
:1027F00078E700B587B00D228DF80020ADF80810FD
:1028000000236A461946FFF799FA49E700B587B0F1
:1028100071B102228DF800200A88ADF8082049889D
:10282000ADF80A1000236A460621FFF787FA37E75A
:10283000102035E770B586B0064601200D46ADF88C
:1028400008108DF80000014600236A463046FFF765
:1028500075FA040008D12946304605F0ABFC00218A
:10286000304605F0C5FC204606B070BDF8B51C46E4
:1028700015460E46069F11F0E6F92346FF1DBCB231
:1028800031462A46009410F0D2FDF8BD30B411460E
:10289000DDE902423CB1032903D0002330BC08F03B
:1028A00022BE0123FAE71A8030BC704770B50C468F
:1028B0000546FFF722FB2146284605F08AFC2846FC
:1028C000BDE87040012105F093BC0000100000201D
:1028D0004FF0E0224FF400400021C2F88001BFF326
:1028E0004F8FBFF36F8F1748016001601649900248
:1028F00008607047134900B500220A600A60124B55
:102900004FF060721A60002808BF00BD0F4A104BDC
:10291000DFF840C001280CD002281CBFFFDF00BD3B
:10292000032008601A604FF4000000BFCCF80000DC
:1029300000BD022008601A604FF04070F6E700B555
:10294000FFDF00BD00F5004008F50140A4020020B3
:1029500014F5004004F5014070B50B2000F0BDF9FE
:10296000082000F0BAF900210B2000F0D4F9002172
:10297000082000F0D0F9F44C01256560A560002026
:10298000C4F84001C4F84401C4F848010B2000F029
:10299000B5F9082000F0B2F90B2000F091F925609C
:1029A00070BD10B50B2000F098F9082000F095F9E3
:1029B000E548012141608160E4490A68002AFCD1B0
:1029C0000021C0F84011C0F84411C0F848110B2094
:1029D00000F094F9BDE81040082000F08FB910B560
:1029E0000B2000F08BF9BDE81040082000F086B9FC
:1029F00000B530B1012806D0022806D0FFDF002044
:102A000000BDD34800BDD34800BDD248001D00BD65
:102A100070B5D1494FF000400860D04DC00BC5F8EB
:102A20000803CF4800240460C5F840410820C4359D
:102A300000F053F9C5F83C41CA48047070BD08B5B0
:102A4000C14A002128B1012811D002281CD0FFDF83
:102A500008BD4FF48030C2F80803C2F84803BB48F1
:102A60003C300160C2F84011BDE80840D0E74FF4A7
:102A70000030C2F80803C2F84803B448403001608F
:102A8000C2F84411B3480CE04FF48020C2F80803A8
:102A9000C2F84803AD4844300160C2F84811AD485F
:102AA000001D0068009008BD70B516460D4604462E
:102AB000022800D9FFDF0022A348012304F11001FE
:102AC0008B4000EB8401C1F8405526B1C1F840218C
:102AD000C0F8043303E0C0F80833C1F84021C0F85F
:102AE000443370BD2DE9F0411D46144630B1012834
:102AF00033D0022838D0FFDFBDE8F081891E0022E4
:102B000021F07F411046FFF7CFFF012D23D0002099
:102B1000944D924F012668703E61914900203C39E6
:102B200008600220091D08608D49042030390860C2
:102B30008B483D34046008206C6000F0DFF83004FE
:102B4000C7F80403082000F0BBF88349F007091F09
:102B500008602E70D0E70120DAE7012B02D00022B6
:102B6000012005E00122FBE7012B04D00022022016
:102B7000BDE8F04198E70122F9E774480068704722
:102B800070B500F0D8F8704C0546D4F84001002626
:102B9000012809D1D4F80803C00305D54FF48030CB
:102BA000C4F80803C4F84061D4F8440101280CD1EA
:102BB000D4F80803800308D54FF40030C4F80803A4
:102BC000C4F84461012013F08AFCD4F848010128BC
:102BD0000CD1D4F80803400308D54FF48020C4F882
:102BE0000803C4F84861022013F079FC5E480560D0
:102BF00070BD70B500F09FF85A4D0446287850B16A
:102C0000FFF706FF687818B10020687013F067FCC2
:102C10005548046070BD0320F8E74FF0E0214FF401
:102C20000010C1F800027047152000F067B84B494A
:102C300001200861082000F061B848494FF47C1079
:102C4000C1F808030020024601EB8003C3F84025C9
:102C5000C3F84021401CC0B20628F5D37047410A92
:102C600043F609525143C0F3080010FB02F000F58F
:102C7000807001EB5020704710B5430B48F2376469
:102C800063431B0C5C020C60384C03FB0400384BA4
:102C90004CF2F72443435B0D13FB04F404EB402098
:102CA00000F580704012107008681844086010BD6C
:102CB0002C484068704729490120C1F8000270473C
:102CC000002809DB00F01F0201219140400980002B
:102CD00000F1E020C0F80011704700280DDB00F083
:102CE0001F02012191404009800000F1E020C0F85E
:102CF0008011BFF34F8FBFF36F8F7047002809DB40
:102D000000F01F02012191404009800000F1E02005
:102D1000C0F8801270474907090E002804DB00F153
:102D2000E02080F80014704700F00F0000F1E02070
:102D300080F8141D70470C48001F00680A4A0D49AE
:102D4000121D11607047000000B0004004B5004043
:102D50004081004044B1004008F50140008000403F
:102D6000408500403C00002014050240F7C2FFFFF0
:102D70006F0C0100010000010A4810B50468094900
:102D800009480831086013F03EFC0648001D046045
:102D900010BD0649002008604FF0E0210220C1F874
:102DA000800270471005024001000001FC1F004036
:102DB000374901200860704770B50D2000F049F8D0
:102DC000344C0020C4F800010125C4F804530D2040
:102DD00000F050F825604FF0E0216014C1F80001C8
:102DE00070BD10B50D2000F034F82A480121416073
:102DF0000021C0F80011BDE810400D2000F03AB8E5
:102E0000254810B504682449244808310860214940
:102E1000D1F80001012804D0FFDF1F48001D046025
:102E200010BD1B48001D00680022C0B2C1F800217F
:102E300014F0A3F8F1E710B5164800BFD0F8001160
:102E40000029FBD0FFF7DCFFBDE810400D2000F0AB
:102E500011B800280DDB00F01F020121914040094C
:102E6000800000F1E020C0F88011BFF34F8FBFF366
:102E70006F8F7047002809DB00F01F02012191408D
:102E80004009800000F1E020C0F880127047000087
:102E900004D5004000D000401005024001000001B0
:102EA0004FF0E0214FF00070C1F8800101F5C071D2
:102EB000BFF34F8FBFF36F8FC1F80001394B8022F2
:102EC00083F8002441F8800C704700B502460420C6
:102ED000354903E001EBC0031B792BB1401EC0B2A2
:102EE000F8D2FFDFFF2000BD41F8302001EBC00128
:102EF00000224A718A7101220A7100BD2A4A00210A
:102F000002EBC0000171704710B50446042800D3DD
:102F1000FFDF254800EBC4042079012800D0FFDF43
:102F20006079A179401CC0B2814200D060714FF03D
:102F3000E0214FF00070C1F8000210BD70B504250B
:102F4000194E1A4C16E0217806EBC1000279012ACD
:102F500008D1427983799A4204D04279827156F835
:102F6000310080472078401CC0B22070042801D373
:102F7000002020706D1EEDB2E5D270BD0C4810B57A
:102F800004680B490B4808310860064890F80004B3
:102F90004009042800D0FFDFFFF7D0FF0448001DE0
:102FA000046010BD19E000E0E0050020580000209A
:102FB00010050240010000010548064A01689142DF
:102FC00001D1002101600449012008607047000020
:102FD0005C000020BEBAFECA40E5014070B50C4658
:102FE000054609F0EFFB21462846BDE870400AF08F
:102FF000D0BC7047704770470021016081807047E6
:103000002CFFFFFFDBE5B151006002002401FFFF50
:103010008400000078DB6A007A2E9AC67DB66CFACE
:10302000F35721CCC310D5E51471FB3C30B5FC4DF2
:103030000446062CA9780ED2DFE804F0030E0E0E2B
:103040000509FFDF08E0022906D0FFDF04E00329BD
:1030500002D0FFDF00E0FFDFAC7030BD30B50446CA
:103060001038EF4D07280CD2DFE800F0040C060CF6
:103070000C0C0C00FFDF05E0287E112802D0FFDFDA
:1030800000E0FFDF2C7630BD2DE9F04112F0C2FBED
:10309000044613F0FFFD201AC5B2062010F04AFCCA
:1030A0000446062010F04EFC211ADD4C207E12282A
:1030B00018D000200F18072010F03CFC064607200F
:1030C00010F040FC301A3918207E13280CD0002054
:1030D0000144A078042809D000200844281AC0B26E
:1030E000BDE8F0810120E5E70120F1E70120F4E7E8
:1030F000CB4810B590F825004108C94800F12600DA
:1031000005D00EF01BFDBDE8104006F082B80EF0B1
:10311000F6FCF8E730B50446A1F120000D460A2878
:103120004AD2DFE800F005070C1C2328353A3F445B
:10313000FFDF42E0207820283FD1FFDF3DE0B848A4
:103140008178052939D0007E122836D020782428AD
:1031500033D0252831D023282FD0FFDF2DE0207851
:1031600022282AD0232828D8FFDF26E0207822280A
:1031700023D0FFDF21E0207822281ED024281CD075
:1031800026281AD0272818D0292816D0FFDF14E0C7
:103190002078252811D0FFDF0FE0207825280CD0DB
:1031A000FFDF0AE02078252807D0FFDF05E0207840
:1031B000282802D0FFDF00E0FFDF257030BD1FB5FB
:1031C00004466A46002001F09FFEB4B1BDF802201B
:1031D0004FF6FF700621824201D1ADF80210BDF812
:1031E0000420824201D1ADF80410BDF808108142DC
:1031F00003D14FF44860ADF8080068460FF082F83C
:1032000006F007F804B010BD70B516460C4605462A
:10321000FEF71FF848B90CB1B44208D90C2070BDB4
:1032200055F82400FEF715F808B1102070BD2046AF
:10323000641EE4B2F4D270BD2DE9F04105461F468C
:1032400090460E4600240068FEF750F830B9A98871
:1032500028680844401EFEF749F808B110203FE7EF
:1032600028680028A88802D0B84202D850E0002878
:10327000F5D0092034E72968085DB8B1671CCA5D3C
:10328000152A2ED03CDC152A3AD2DFE802F039129A
:10329000222228282A2A313139393939393939391C
:1032A00039392200085D30BB641CA4B2A242F9D8AF
:1032B00033E00228DDD1A01C085C88F80000072854
:1032C00001D2400701D40A200AE7307840F001001B
:1032D00015E0C143C90707E0012807D010E0062028
:1032E000FEE60107A1F180510029F5D01846F7E666
:1032F0003078810701D50B20F2E640F002003070F3
:103300002868005D384484B2A888A04202D2B0E7A1
:103310004FF4485382B2A242ADD80020E0E610B587
:10332000027843F2022354080122022C12D003DC5B
:103330003CB1012C16D106E0032C10D07F2C11D10A
:1033400012E0002011E080790324B4EB901F09D132
:103350000A700BE08079B2EB901F03D1F8E7807917
:103360008009F5D0184610BDFF200870002010BD60
:1033700008B500208DF80000294890F82E1051B1B2
:1033800090F82F0002280FD003280FD0FFDF00BFD6
:103390009DF8000008BD22486946253001F003FE73
:1033A0000028F5D0FFDFF3E7032000E001208DF8CF
:1033B0000000EDE738B50C460546694601F0F3FD1F
:1033C00000280DD19DF80010207861F3470020708F
:1033D00055F8010FC4F80100A888A4F805000020E2
:1033E00038BD38B5137888B102280FD0FF281BD01C
:1033F0000CA46D46246800944C7905EB9414247851
:1034000064F347031370032805D010E023F0FE0394
:1034100013700228F7D1D8B240F001000AE0000092
:10342000F00100200302FF0143F0FE00107010784D
:1034300020F0010010700868C2F801008888A2F826
:10344000050038BD022110F0CDBA38B50C46097818
:10345000222901D2082038BDADF800008DF80220E5
:1034600068460EF0ADFB05F0D4FE050003D1212126
:103470002046FFF74FFE284638BD1CB500208DF8CA
:103480000000CDF80100ADF80500FE4890F82E00D0
:10349000022801D0012000E000208DF807006846D6
:1034A0000EF014FC002800D0FFDF1CBD00220A80B3
:1034B000437892B263F3451222F040020A8000780A
:1034C0000C282BD2DFE800F02A06090E1116191C71
:1034D0001F220C2742F0110009E042F01D00088075
:1034E0000020704742F0110012E042F0100040F05E
:1034F0000200F4E742F01000F1E742F00100EEE7CD
:1035000042F0010004E042F00200E8E742F002006D
:1035100040F00400E3E742F00400E0E707207047D2
:103520002DE9FF478AB00025BDF82C6082461C4675
:1035300090468DF81C50700703D56068FDF789FE32
:1035400068B9D04F4FF0010997F82E0058B197F89D
:103550002F00022807D16068FDF7C8FE18B11020BF
:103560000EB0BDE8F087300702D5A089802816D8B4
:10357000700705D4B8F1000F02D097F8240070B19D
:10358000E07DC0F300108DF81B00617D072041B184
:10359000012906D00229E3D00429E1D12CE007203B
:1035A000DEE749468DF81790F00609D4A27D072082
:1035B00032B1012A04D0022A05D0042AD0D11BE05E
:1035C0008DF8191002E002208DF819008DF8158091
:1035D0006068B0B107A9FFF7A2FE0028C0D19DF82E
:1035E0001C00FF280AD0606850F8011FCDF80F10AA
:1035F0008088ADF8130008E00620B1E743F202200E
:10360000AEE7CDF80F50ADF81350E07B0028F3D1B2
:10361000207C0028F0D1607C0028EDD1A07C00281F
:10362000EAD1E07CC006E7D18DF800A0BDF82C00FF
:10363000ADF80200A0680190A068029004F10F00AC
:1036400001F0A5FC8DF80C00FFF792FE8DF80D003F
:103650009DF81C008DF80E008DF816508DF818504E
:10366000E07D08A900F00F008DF81A0068460EF002
:1036700091FF05F0CEFD73E7F0B58FB000258DF812
:1036800030508DF814508DF8345006468DF828507F
:10369000019502950395049519B10FC901AC84E811
:1036A0000F00784CA078052801D004280CD101988F
:1036B0006168884200D120B90398E168884203D14B
:1036C00010B108200FB0F0BD207DC00601D51F2726
:1036D00000E0FF273B460DAA05A903A8FFF7ACFDB4
:1036E0000028EFD1A08AC10702D0C00600D4EE277F
:1036F0003B460AAA0CA901A8FFF79EFD0028E1D1CC
:103700009DF81400C00701D00A20DBE7A08A41071A
:1037100008D4A17D31B19DF82810890702D043F269
:103720000120CFE79DF82810C90709D0400707D42A
:10373000208818B144F25061884201D90720C1E7BE
:103740008DF818508DF81960BDF80800ADF81A0012
:103750000198079006A80EF029FF05F05AFD0028F1
:10376000B0D18DF820508DF82160BDF81000ADF873
:1037700022000398099008A80EF03AFF05F049FDD1
:1037800000289FD101AD241D95E80F0084E80F00AB
:10379000002097E770B586B00D46040005D0FDF710
:1037A000A5FD20B1102006B070BD0820FBE72078F1
:1037B000C107A98802D0FF2902D303E01F2901D243
:1037C0000920F0E780073BD4FFF75EFC38B1217891
:1037D000C1F3C100012804D0032802D005E0132062
:1037E000E1E7284890F82400C8B1C8074FF0010667
:1037F0004FF0000502D08DF80F6001E08DF80F50FA
:10380000FFF7B6FD8DF8000020786946C0F3C100CF
:103810008DF8010060788DF80250C20801D00720B1
:10382000C1E778B1C20701D08DF80260820705D5E3
:103830009DF8022042F002028DF80220400703D5D5
:103840000620B0E78DF80260002022780B18C2F342
:103850008002DA7001EB40026388D380401CA388A9
:10386000C0B253810228F0D3207A0028E8D1607AD0
:103870000028E5D1A07A0028E2D1E07A0028DFD143
:10388000207B01E0F0010020C006D9D104F108003E
:1038900001F07DFB8DF80E0068460EF0E4FA05F0AD
:1038A000B8FC00288DD18DF810608DF81150E0889B
:1038B000ADF81200ADF8145004A80EF027FB05F087
:1038C000A8FC00288CD12078C00701D0152000E08A
:1038D0001320FFF7C3FB002065E72DE9FF47022017
:1038E000FD4E8DF804000027708EADF80600B84636
:1038F00043F202094CE001A80FF0DBFF050006D0FF
:10390000708EA8B3A6F83280ADF806803EE0039C26
:10391000A07F01072DD504F124000090A28EBDF8F0
:103920000800214604F1360301F0B8FC050005D07B
:103930004D452AD0112D3CD0FFDF3AE0A07F20F08A
:103940000801E07F420862F3C711A177810861F3A3
:103950000000E07794F8210000F01F0084F82000B8
:103960002078282826D129212046FFF7D3FB21E003
:1039700014E040070AD5BDF8080004F10E0101F07B
:103980001CFB05000DD04D4510D100257F1CFFB25A
:1039900002200FF0CFFF401CB842ACD8052D11D04B
:1039A00008E0A07F20F00400A07703E0112D00D0F4
:1039B000FFDF0025BDF806007086052D04D02846DF
:1039C00004B0CEE5A6F832800020F9E770B50646CF
:1039D000FFF738FD054605F0FFFD040000D1FFDFCD
:1039E0006680207820F00F00801C20F0F00020304E
:1039F00020700320207295F83E006072BDE8704090
:103A000005F0EDBD2DE9F04786B0040000D1FFDFE1
:103A10002078B14D20F00F00801C20F0F0007030B5
:103A2000207060680178491F1B2933D2DFE801F05C
:103A3000FE32323255FD320EFDFD42FC323232781A
:103A4000FCFCFBFA32FCFCF9F8FCFC00C6883046B2
:103A5000FFF7F8FC0546304607F03BFCE0B1606834
:103A6000007A85F83E0021212846FFF753FB3046B7
:103A7000FEF760FB304603F0D3FE3146012013F021
:103A800041FDA87F20F01000A877FFF726FF00284F
:103A900000D0FFDF06B064E5207820F0F000203091
:103AA00020700320207266806068007A607205F0E2
:103AB00096FDD8E7C5882846FFF7C4FC00B9FFDFAC
:103AC00060680079012800D0FFDF6068017A06B0E5
:103AD0002846BDE8F04707F0E1BDC6883046FFF74D
:103AE000B1FC050000D1FFDF05F079FD60683146CB
:103AF0000089288160684089688160688089A88120
:103B0000012013F0FFFC0020A875A87F00F003003F
:103B10000228BFD1FFF7E1FE0028BBD0FFDFB9E7E5
:103B2000007928B10228B5D03C28B3D0FFDFB1E737
:103B300005F055FD6668B6F806A0307A361D0128F6
:103B400006D0687E814605F0D0FA070003D101E077
:103B5000E878F7E7FFDF0022022150460FF039FF37
:103B6000040000D1FFDF22212046FFF7D3FA30798D
:103B7000012800D00220A17F804668F30101A177CF
:103B8000308B2081708B6081B08BA08184F8229073
:103B90008DF80880B8680090F86801906A460321A3
:103BA00050460FF016FF00B9FFDFB888ADF81000DF
:103BB000B8788DF8120004AA052150460FF009FFCD
:103BC00000B9FFDFB888ADF80C00F8788DF80E006A
:103BD00003AA042150460FF0FCFE00B9FFDF0621C6
:103BE00006F112000DF07FF840B37079800700D520
:103BF000FFDF7179E07D61F34700E075D6F80600DC
:103C0000A0617089A083062106F10C000DF06BF80D
:103C1000F0B195F825004108607861F3470006E0AF
:103C200041E039E071E059E04EE02FE043E06070A0
:103C3000D5F82600C4F80200688D12E0E07D20F07F
:103C4000FE00801CE075D6F81200A061F08AD9E76A
:103C5000607820F0FE00801C6070F068C4F80200FC
:103C6000308AE080B8F1010F04D0B8F1020F05D01E
:103C7000FFDF0FE70320FFF7D9F90BE7287E1228B3
:103C800000D0FFDF1120FFF7E9F903E706B0204677
:103C9000BDE8F04701F08EBD05F0A1FC15F8300F2E
:103CA00040F0020005E005F09AFC15F8300F40F0F6
:103CB00004002870EEE6287E13280AD01528D8D1F3
:103CC0005FF01600FFF7CAF906B0BDE8F04705F04F
:103CD00086BC1420F6E70000F0010020A978052931
:103CE00009D00429C5D105F07AFC022006B0BDE850
:103CF000F047FFF79BB900790028BAD0E87801F0C7
:103D00002DF905F06CFC0320F0E7287E122802D183
:103D1000687E01F023F91120D4E72DE9F05F054614
:103D200000784FF000080009DFF8B8A891460C466B
:103D3000464601286ED002286DD007280BD00A28ED
:103D40006AD0FFDFA9F8006014B1A4F80080668093
:103D50000020BDE8F09F6968012704F108000B7896
:103D60004FF0020B5B1F4FF6FF721B2B7ED2DFE87A
:103D700003F0647D7D7D0E7D7D7D7D7D7D217D7D5E
:103D80007D2BFDFCFBFA7D14D2F9E7F8F700C8881B
:103D90004FF01208102621469AE14FF01C080A261F
:103DA000BCB38888A0806868807920726868C07910
:103DB0006072C7E74FF01B08142654B3032020722B
:103DC00068688088A080BDE70A793C2ABAD00D1DBA
:103DD0004FF010082C26E4B16988A180298B6182FC
:103DE000298B2182698BA182A98BE1826B790246A2
:103DF000A91D1846FFF7F5FA2979002001290CD0F2
:103E000084F80FB0FF212176E06120626062A06239
:103E100098E70FE03BE15EE199E1E77320760AF174
:103E2000040090E80E00DAF81000C4E90930C4E993
:103E3000071287E7A9F800608AE72C264FF01D08D3
:103E4000002CF7D0A28005460F1D897B008861F306
:103E500000002880B97A490861F341002880B97AC6
:103E6000890861F382002880B97A00E00CE1C90872
:103E700061F3C3002880B97AAA1C0911491C61F3B7
:103E8000041000F07F0028807878B91CFFF7A9FAA9
:103E9000387D05F1090207F11501FFF7A2FA387B19
:103EA00001F0A9F82874787B01F0A5F86874F87E11
:103EB000A874787AE874387F2875B87B6875388A72
:103EC000E882DAF81C10A961B97A504697F808A080
:103ED000C1F34111012904D0008C504503D2824620
:103EE00009E0FFDF10E0022903D0288820F06000FD
:103EF00009E0504504D1288820F06000403002E0FD
:103F0000288840F060002880A4F824A0524607F1D9
:103F10001D01A8699BE011264FF02008002C89D0D4
:103F2000A280686804F10A02007920726868007B48
:103F3000607269688B1D48791946FFF752FA01E7EC
:103F40000A264FF02108002CE9D08888A0806868F4
:103F5000807920726868C07960729AF8301006E043
:103F600078E06BE052E07FE019E003E03AE021F016
:103F70000401A6E00B264FF02208002CCFD0C88801
:103F8000A0806868007920726868007A01F033F8D0
:103F900060726868407A01F02EF8A072D2E61C26A2
:103FA0004FF02608002CBAD0A28068684079607271
:103FB0006868007AA0720AF1040090E80E00DAF84E
:103FC0001000C4E90530C4E90312686800793C2890
:103FD00003D0432803D0FFDFB4E62772B2E684F8AB
:103FE00008B0AFE610264FF02408002C97D0888840
:103FF000A0806868807920816868807A60816868BC
:104000000089A08168688089E0819BE610264FF0D6
:104010002308002C98D08888A0806868C0882081F8
:1040200068680089608168684089A08168688089C3
:10403000E0819AF8301021F0020142E030264FF082
:104040002508002C9AD0A2806968282249680AF0C5
:10405000B4F977E62A264FF02F08002C8ED0A280E4
:1040600069682222091DF2E714264FF01B08002C74
:1040700084D0A280686800790128B0D02772DAE97C
:104080000710C4E903105DE64A46214660E0287A3D
:10409000012803D0022817D0FFDF53E610264FF087
:1040A0001F08002CA2D06888A080A8892081E889F8
:1040B0006081288AA081688AE0819AF8301021F016
:1040C00001018AF830103DE64FF01208102668888A
:1040D00000F07EFF36E6287AC8B3012838D00228DF
:1040E00036D0032801D0FFDF2CE609264FF0110857
:1040F000002C8FD06F883846FFF7A4F990F822A0E3
:10410000A780687A2072042138460FF07DFC0521D3
:1041100038460FF079FC002138460FF075FC01217C
:1041200038460FF071FC032138460FF06DFC022178
:1041300038460FF069FC062138460FF065FC072170
:1041400038460FF061FC504600F008FFFAE5FFE743
:104150002846BDE8F05F01F0B7BC70B5012803D078
:10416000052800D0FFDF70BD8DB22846FFF76AF941
:10417000040000D1FFDF20782128F4D005F02CFACC
:1041800080B1017821F00F01891C21F0F00110317C
:1041900001700221017245800020A075BDE87040C9
:1041A00005F01DBA21462846BDE870401322FFF7EE
:1041B0004CB92DE9F04116460C00804600D1FFDFD6
:1041C000307820F00F00801C20F0F00010303070AC
:1041D0002078012804D0022818D0FFDFBDE8F08144
:1041E0004046FFF72FF9050000D1FFDF0320A87537
:1041F00005F0F5F994E80F00083686E80F00F94855
:1042000010F8301F41F001010170E7E74046FFF769
:1042100019F9050000D1FFDFA1884FF6FF700027D4
:10422000814202D1E288824203D0814201D1E088FA
:1042300040B105F0D4F994E80F00083686E80F0085
:10424000AF75CBE7A87D0128C8D17823002241466D
:1042500013F0AEF80220A875C0E738B50C46242844
:104260005CD008DC20280FD0212825D022284BD074
:10427000232806D14CE0252841D0262832D03F28DB
:1042800051D00725284638BD0021052013F010F92C
:1042900008B1112038BDA01C0EF087F804F0B9FF5A
:1042A0000500EFD1002208231146052013F080F805
:1042B0000528E7D0FFDFE5E76068FDF70EF808B1F5
:1042C000102038BD618820886A460EF022FB04F079
:1042D000A0FF0500D6D160680028D3D0BDF800103B
:1042E0000180CFE7206820B1FDF700F808B1102564
:1042F000C8E720460EF0E6FB1DE00546C2E7A178C0
:1043000020880EF037FB16E0086801F089FEF4E71C
:10431000087800F001000DF0E5FB0CE061882088D2
:104320000EF073FA07E0087800F001008DF8000045
:1043300068460DF0A2FE04F06CFFDEE770B505469E
:104340000C460846FCF7ABFF08B1102070BD202DCD
:1043500007D0212D0DD0222D0BD0252D09D00720DF
:1043600070BD2088A11C0DF08FFCBDE8704004F0EA
:1043700050BF062070BD9B482530704708B53422D9
:10438000002198480AF043F80120FEF74FFE112063
:10439000FEF764FE93496846263105F0B3F891486C
:1043A0009DF8002010F8251F62F3470121F001015C
:1043B0000170002141724FF46171A0F807100221D1
:1043C0008172FEF795FE00B1FFDFFDF70BF801F0FB
:1043D000BAF908BD10B50C464022002120460AF06B
:1043E00016F8A07F20F00300A07720202070002086
:1043F000A07584F8230010BD70472DE9FC410746E5
:10440000FCF727FF10B11020BDE8FC81754E06F1C6
:104410002501D6F825000090B6F82950ADF80450D3
:1044200096F82B408DF806403846FEF7C3FF00286B
:10443000EAD1FEF75DFE0028E6D0009946F8251F78
:10444000B580B471E0E710B50446FCF728FF08B169
:10445000102010BD63486349224690F8250026319C
:104460004008FEF7BEFF002010BD3EB504460D46D5
:104470000846FCF714FF08B110203EBD14B143F20A
:1044800004003EBD57488078052803D0042801D099
:1044900008203EBD694602A80AF0B8FB2A466946D4
:1044A0009DF80800FEF79DFF00203EBDFEB50D46BD
:1044B00004004FF0000712D00822FEF7A5FE0028E6
:1044C00012D1002609E000BF54F826006946FEF725
:1044D00026FF002808D1761CF6B2AE42F4D30DF0C8
:1044E0004BFA10B143F20320FEBD3E4E86F8247015
:1044F0000CB300271BE000BF54F8270002A9FEF709
:104500000EFF00B1FFDF9DF808008DF8000054F8A1
:10451000270050F8011FCDF801108088ADF8050084
:1045200068460DF04EFA00B1FFDF7F1CFFB2AF42CC
:10453000E2D386F824500020FEBD2DE9F0418AB078
:104540001546884604001ED00F4608222946FEF76D
:104550005BFE002811D1002613E000BF54F82600AE
:104560006946103000F01FFD002806D13FB157F812
:104570002600FCF76EFE10B110200AB02EE6761C65
:10458000F6B2AE42EAD3681EC6B217E0701CC7B2DC
:1045900012E000BF54F82600017C4A0854F82710A6
:1045A0000B7CB2EB530F05D106221130113109F00B
:1045B000D7FE50B17F1CFFB2AF42EBD3761EF6B2EE
:1045C000E4D2464624B1012003E043F20520D4E7BB
:1045D00000200DF01BFA10B90DF024FA20B143F2BF
:1045E0000420CAE7F001002064B300270DF117088A
:1045F00026E000BF54F827006946103000F0D3FCD5
:1046000000B1FFDF54F82700102250F8111FCDF839
:1046100001108088ADF8050054F827100DF107004F
:1046200009F0CBFE96B156F827101022404609F04B
:10463000C4FE68460DF0AAF900B1FFDF7F1CFFB28F
:10464000AF42D7D3FEF719FF002096E7404601F0AE
:10465000DBFCEEE730B585B00446FDF7C3F830B9B2
:1046600006200FF067F910B1062005B030BD2046D6
:10467000FCF7EFFD18B96068FCF738FE08B11020B0
:10468000F3E760884AF2B811884206D82078F94DDD
:1046900028B1012806D0022804D00720E5E7FEF75C
:1046A00027FD18E06078022804D0032802D043F2E6
:1046B0000220DAE785F82F00C1B200200090ADF8A3
:1046C000040002292CD0032927D0FFDF68460DF013
:1046D00035FA04F09EFD0028C7D1606801F087FC20
:1046E000207858B101208DF800000DF1010001F093
:1046F0008BFC68460EF0ADF900B1FFDF207885F83D
:104700002E00FEF7BAFE608860B1A88580B20DF079
:1047100075F900B1FFDF0020A7E78DF80500D5E7A8
:104720004020FAE74FF46170EFE710B50446FCF75C
:10473000B6FD20B9606838B1FCF7CFFD08B1102094
:1047400010BD606801F060FCCA4830F82C1F618021
:10475000C178617080782070002010BD2DE9F84389
:10476000144689460646FCF79AFDA0B94846FCF770
:10477000BDFD80B92046FCF7B9FD60B9BD4DA878F4
:10478000012800D13CB13178FF2906D049B143F26C
:104790000400BDE8F8831020FBE7012801D00420C5
:1047A000F7E7CCB3052811D004280FD0694620467E
:1047B000FEF77CFE0028ECD1217D49B1012909D00A
:1047C000022909D0032909D00720E2E70820E0E701
:1047D000024604E0012202E0022200E003228046B9
:1047E0002346174600200099FEF79AFE0028D0D1F4
:1047F000A0892880A07BE875BDF80000A882AF756D
:10480000BDF80010090701D5A18931B1A18929801E
:10481000C00704D0032003E006E08021F7E7022070
:10482000FEF704FC86F800804946BDE8F843002006
:10483000FEF722BF7CB58F4C05460E46A0780228B5
:1048400003D0032801D008207CBD15B143F2040039
:104850007CBD07200FF076F810B9A078032806D0A9
:10486000FEF712FC28B1A078032804D009E012203A
:104870007CBD13207CBD304600F053FB0028F9D1ED
:10488000E670FEF775FD0AF0FEF801208DF80000D5
:104890008DF801008DF802502088ADF80400E07D0D
:1048A0008DF8060068460DF073FF04F0B2FC002896
:1048B000E0D1A078032805D05FF00400FEF7B6FB36
:1048C00000207CBDE07800F03CFB0520F6E71CB53D
:1048D00010B143F204001CBD664CA078042803D03C
:1048E000052801D008201CBD00208DF80000012102
:1048F0008DF801108DF8020068460DF049FF04F0B4
:1049000088FC0028EFD1A078052805D05FF00200D0
:10491000FEF78CFB00201CBDE07800F01FFB03209D
:10492000F6E72DE9FC4180460E4603250846FCF7D4
:10493000DDFC002866D14046FEF784FD040004D06B
:104940002078222804D208205EE543F202005BE5CD
:10495000A07F00F003073EB1012F0CD000203146AC
:10496000FEF72DFC0500EFD1012F06D0022F1AD043
:10497000FFDF284648E50120F1E7A07D3146022807
:1049800001D011B107E011203EE56846FCF75EFE5C
:104990000028D9D16946404606F043FE0500E8D11B
:1049A0000120A075E5E7A07D032804D1314890F8E7
:1049B0003000C00701D02EB30EE026B1A07F400723
:1049C0001ED4002100E00121404606F04AFE050009
:1049D000CFD1A075002ECCD03146404600F0EDFA84
:1049E00005461128C5D1A07F4107C2D4316844F8DB
:1049F0000E1F7168616040F0040020740025B8E764
:104A00001125B6E71020FFE470B50C460546FEF709
:104A100019FD010005D022462846BDE87040FEF78A
:104A200014BD43F2020070BD10B5012807D1114B2F
:104A30009B78012B00D011B143F2040010BD0DF0A2
:104A40000FF8BDE8104004F0E4BB012300F090BA79
:104A500000231A46194600F08BBA70B506460C467C
:104A60000846FCF7F6FB18B92068FCF718FC18B1EB
:104A7000102070BDF0010020F84D2A7E112A04D0CC
:104A8000132A00D33EB10820F3E721463046FEF753
:104A900081FE60B1EDE70920132A0DD0142A0BD056
:104AA000A188FF29E5D31520FEF7D8FA0020D4E924
:104AB0000012C5E90712DCE7A1881F29D9D313200A
:104AC000F2E71CB5E548007E132801D208201CBD82
:104AD00000208DF8000068460DF018FA04F099FBEC
:104AE0000028F4D11120FEF7B9FA00201CBD2DE9F1
:104AF000F04FDFF868A3814691B09AF818009B4602
:104B000015460C46132803D3FFF7DBFF00281FD1FF
:104B10002046FCF79EFB78BB2846FCF79AFB58BB67
:104B200020784FF00107C0074FF0000102D08DF848
:104B30003A7001E08DF83A1020788846C0F3C10041
:104B40008DF8000060788DF80910C10803D00720A7
:104B500011B0BDE8F08F80B1C10701D08DF80970A8
:104B6000810705D59DF8091041F002018DF8091063
:104B7000400704D50620EBE720E08DF809709DF88A
:104B80000900810703D540F001008DF809000020DD
:104B90006E4606EB400162884A81401CA288C0B282
:104BA0000A820328F5D32078C0F3C100012821D060
:104BB00003281FD04846FCF74CFB08B11020C7E77C
:104BC00099F80000400808D0012809D0022807D031
:104BD000032805D043F20220BAE78DF8028001E0F5
:104BE0008DF80270484650F8011FCDF803108088F8
:104BF000ADF80700FEF7BCFB8DF80100002042462F
:104C000006EB40012B88CB826B888B83AB884B846F
:104C1000EB880B85401CCA85C0B28A860328EFD377
:104C2000E088ADF83C0068460DF01DFA00288ED1F2
:104C30009AF818005546112801D0082088E7062068
:104C40000EF080FE38B12078C0F3C100012804D0F6
:104C5000032802D006E012207AE795F82400002805
:104C60003FF475AFFEF710FA022801D213206FE768
:104C7000584600F056F90028A1D185F819B06846C9
:104C80000DF01AFB04F0C5FA040098D1687E00F01C
:104C900058F91220FEF7E2F9204659E770B56F4D3A
:104CA000287E122801D00820E3E60DF008FB04F06E
:104CB000B0FA040005D1687E00F050F91120FEF72B
:104CC000CDF92046D5E670B5064615460C46084691
:104CD000FCF7E5FA18B92846FCF7E1FA08B110200C
:104CE000C7E62A46214630460DF0F3FD04F091FA5E
:104CF0000028F5D121787F29F2D10520B9E67CB5CD
:104D000005460C460846FCF7A4FA08B110207CBD05
:104D10002846FEF797FB20B10078222804D208200D
:104D20007CBD43F202007CBD4C4890F83000400747
:104D300001D511207CBD2178C80802D16078C20855
:104D400001D007207CBD890801D1800801D0062050
:104D50007CBDADF8005020788DF8020060788DF8A9
:104D600003000220ADF8040068460CF06EFC04F06D
:104D700050FA7CBD70B586B014460D460646FEF767
:104D800061FB28B10078222805D2082006B070E621
:104D900043F20200FAE72846FCF7A8FA20B944B12A
:104DA0002046FCF79AFA08B11020EFE700202060B7
:104DB000A0802A4890F83000800701D51120E5E74F
:104DC00003A930460CF07EFC18B100BF04F021FAB4
:104DD000DCE7ADF80060BDF81400ADF80200BDF8E6
:104DE0001600ADF80400BDF81000BDF81210ADF8C3
:104DF0000600ADF808107DB1298809B1ADF806109C
:104E0000698809B1ADF80210A98809B1ADF8081098
:104E1000E98809B1ADF80410DCB1BDF80610814293
:104E200001D9081A2080BDF80210BDF81400814293
:104E300001D9081A6080BDF80800BDF80410BDF85B
:104E400016200144BDF812001044814201D9081A0D
:104E5000A08068460CF004FDB8E70000F0010020D7
:104E60001CB56A490968CDE9001068460DF0FDF8E7
:104E700004F0CFF91CBD1CB50020009001906846DD
:104E80000DF0F3F804F0C5F91CBD70B505460C46ED
:104E90000846FCF704FA08B11020EAE52146284646
:104EA0000CF03CFFBDE8704004F0B3B93EB50546D8
:104EB0000C460846FCF7F3F908B110203EBD00206F
:104EC000009001900290ADF800502089ADF80800E4
:104ED00020788DF80200606801902089ADF8080004
:104EE0006089ADF80A0068460CF02AFF04F091F9D9
:104EF0003EBD0EB5ADF800000020019068460CF0F4
:104F00001FFF04F086F90EBD108008885080488885
:104F10009080C88810818888D0800020508190813E
:104F2000704710B5044604F0E0F830B1407830B175
:104F3000204604F0F8FB002010BD052010BD122013
:104F400010BD10B504F0D1F8040000D1FFDF607887
:104F500000B9FFDF6078401E607010BD10B504F02E
:104F6000C4F8040000D1FFDF6078401C607010BD01
:104F70001CB5ADF800008DF802308DF803108DF8E7
:104F8000042068460DF068FC04F043F91CBD0CB524
:104F90001FA2D2E90012CDE900120079694601EBA7
:104FA000501000780CBD0278520804D0012A02D0BB
:104FB00043F202207047FEF7B2B91FB56A46FFF709
:104FC000A3FF68460DF0AEF904F023F904B010BD5C
:104FD00070B50C0006460DD0FEF734FA050000D17E
:104FE000FFDFA68028892081288960816889A081C7
:104FF000A889E0813DE500B530B1012803D0022841
:1050000001D0FFDF002000BDFF2000BDFC530200E7
:10501000070605040302010010B50446FCF719F960
:1050200008B1102010BD2078C0F30210042807D862
:105030006078072804D3A178102901D8814201D2D1
:10504000072010BDE078410706D421794A0703D430
:10505000000701D4080701D5062010BD002010BDAF
:1050600010B513785C08837F64F3C71383771378D4
:105070009C08C37F64F30003C3771078C3094878A2
:1050800063F34100487013781C090B7864F34713ED
:105090000B701378DB0863F3000048705078487198
:1050A00010BD10B5C4780B7864F300030B70C4789E
:1050B000640864F341030B70C478A40864F38203AA
:1050C0000B70C478E40864F3C3030B7003791178A0
:1050D00063F30001117003795B0863F34101117000
:1050E00003799B0863F3820111700079C00860F3B3
:1050F000C301117010BD70B514460D46064604F08C
:105100006BFA80B10178182221F00F01891C21F07F
:10511000F001A03100F8081B214609F04EF9BDE866
:10512000704004F05CBA29463046BDE87040132256
:10513000FEF78BB92DE9F047064608A8904690E89F
:10514000300489461F4614220021284609F05FF9E1
:105150000021CAF80010B8F1000F03D0B9F1000F18
:1051600003D114E03878C00711D02068FCF797F815
:10517000C0BBB8F1000F07D120681230286020684A
:10518000143068602068A8602168CAF80010387878
:10519000800724D56068FCF7A0F818BBB9F1000FB0
:1051A00021D0FFF7E8F80168C6F868118188A6F8F1
:1051B0006C11807986F86E0101F013FDF94FEF60F4
:1051C000626862B196F8680106F26911400810320F
:1051D000FEF707F910223946606809F0EEF8002062
:1051E000BDE8F08706E0606820B1E8606068C6F856
:1051F0006401F4E71020F3E730B5054608780C4663
:1052000020F00F00401C20F0F00110312170002030
:10521000607095F8230030B104280FD0052811D014
:10522000062814D0FFDF20780121B1EB101F04D233
:1052300095F8200000F01F00607030BD21F0F000F4
:10524000203002E021F0F00030302070EBE721F058
:10525000F0004030F9E7F0B591B0022715460C4652
:1052600006463A46ADF80870092103AB05F05DF833
:105270000490002810D004208DF804008DF80170EF
:10528000E034099605948DF818500AA9684610F084
:10529000A2F800B1FFDF012011B0F0BD10B588B059
:1052A0000C460A99ADF80000CBB11868CDF80200A1
:1052B000D3F80400CDF80600ADF80A20102203A8A8
:1052C00009F07BF868460DF09DF803F0A2FF002876
:1052D00003D1A17F41F01001A17708B010BD0020DB
:1052E000CDF80200E6E72DE9F84F0646808A0D4624
:1052F00080B28246FEF7A6F804463078DFF8A48232
:1053000000274FF00209A8F120080F2870D2DFE82B
:1053100000F06FF23708387D8CC8F1F0EFF35FF3DF
:10532000F300A07F00F00300022809D05FF0000026
:1053300080F0010150460EF055FB050003D101E05D
:105340000120F5E7FFDF98F85C10C90702D0D8F814
:1053500060000BE0032105F11D0011F0ECFDD5F814
:105360001D009149B0FBF1F201FB1200C5F81D00D0
:1053700070686867B068A8672078252800D0FFDFCC
:10538000CAE0A07F00F00300022809D05FF000000F
:1053900080F0010150460EF025FB060003D101E02C
:1053A0000120F5E7FFDF3078810702D52178252934
:1053B00004D040F001003070BDE8F88F85F800900F
:1053C000307F287106F11D002D36C5E90206F3E78E
:1053D000A07F00F00300022808D0002080F0010127
:1053E00050460EF0FFFA040004D102E00120F5E778
:1053F000A7E1FFDF2078C10604D5072028703D34DF
:105400006C60D9E740F008002070D5E7E07F000726
:1054100000D5FFDF307CB28800F0010301B05046B8
:10542000BDE8F04F092106F05EB804B9FFDF7168EE
:1054300021B1102204F1240008F0BFFF28212046EA
:10544000FDF768FEA07F00F0030002280ED104F1F2
:105450002400002300901A4621465046FFF71EFF05
:10546000112807D029212046FDF754FE307A84F810
:105470002000A1E7A07F000700D5FFDF14F81E0F72
:1054800040F008002070E782A761E761C1096078F9
:1054900061F34100014660F382016170307AE0708F
:1054A0008AE7A07F00F00300022809D05FF0000027
:1054B00080F0010150460EF095FA040003D101E09E
:1054C0000120F5E7FFDF022104F1850011F033FD33
:1054D0000420287004F5B4706860B4F88500288250
:1054E000304810387C346C61C5E9028064E703E021
:1054F00024E15BE02DE015E0A07F00F0030002282E
:1055000007D0002080F0010150460EF06BFA18B968
:1055100001E00120F6E7FFDF324621465046BDE8B4
:10552000F84FE8E504B9FFDF20782128A1D93079C8
:10553000012803D1E07F40F00800E07732462146A1
:105540005046FFF7D8FD2046BDE8F84F2321FDF770
:10555000E1BD3279AA8005F108030921504604F023
:10556000E4FEE86010B10520287025E7A07F00F078
:105570000300022808D0002080F0010150460EF000
:1055800031FA040003D101E00120F5E7FFDF04F167
:10559000620102231022081F0EF0ABF80770317968
:1055A000417009E75002002040420F00A07F00F048
:1055B0000300022808D0002080F0010150460EF0C0
:1055C00011FA050003D101E00120F5E7FFDF95F8AE
:1055D000840000F0030001287AD1A07F00F00307C7
:1055E000E07F10F0010602D0022F04D133E095F8DD
:1055F000A000C0072BD0D5F8601121B395F8832007
:10560000087C62F387000874A17FCA09D5F860118D
:1056100062F341000874D5F8601166F30000087465
:10562000AEB1D5F86001102204F12401883508F0EC
:10563000C4FE287E40F001002876287820F0010082
:1056400005F8880900E016B1022F04D02DE095F886
:105650008800C00727D0D5F85C1121B395F88320C6
:10566000087C62F387000874A17FCA09D5F85C1131
:1056700062F341000874D5F85C1166F30000087409
:105680008EB1D5F85C01102204F12401883508F0B0
:1056900094FE287840F0010005F8180B287820F0D7
:1056A000010005F8A009022F44D0002000EB4000C3
:1056B00005EBC00090F88800800709D595F87C00BC
:1056C000D5F86421400805F17D011032FDF789FE0F
:1056D0008DF8009095F884006A4600F003008DF87C
:1056E000010095F888108DF8021095F8A0008DF84B
:1056F00003002146504601F05DFA2078252805D0A8
:10570000212807D0FFDF2078222803D92221204634
:10571000FDF700FDA07F00F0030002280CD0002060
:1057200080F0010150460EF06FF900283FF44FAEB3
:10573000FFDF41E60120B9E70120F1E7706847701B
:105740003AE6FFDF38E670B5FE4C002584F85C5081
:1057500025660FF00CFE04F11001204603F0F8FE60
:1057600084F8305070BD70B50D46FDF76BFE040037
:1057700000D1FFDF4FF4B8720021284608F047FE41
:1057800004F124002861A07F00F00300022809D062
:105790005FF0010105F1E0000FF0EAFD002800D004
:1057A000FFDF70BD0221F5E70A46014602F1E00085
:1057B0000FF0FFBD70B50546406886B001780A2934
:1057C00006D00D2933D00E292FD0FFDF06B070BDD3
:1057D00086883046FDF736FE040000D1FFDF2078D2
:1057E0002128F3D028281BD1686802210E3001F04F
:1057F000D6F9A8B168680821801D01F0D0F978B108
:1058000004F1240130460CF0C5FF03F002FD00B1A5
:10581000FFDF06B02046BDE870402921FDF77ABCC5
:1058200006B0BDE8704003F0DABE0121017268687D
:10583000C6883046FDF706FE040000D1FFDFA07FDA
:1058400000F00301022902D120F01000A077207897
:1058500021280AD06868017A09B1007980B1A07F57
:1058600000F00300022862D0FFDFA07F00F00300F9
:105870000228ABD1FEF731F80028A7D0FFDFA5E75B
:1058800003F0ADFEA17F08062BD5E07FC00705D051
:1058900094F8200000F01F00102820D05FF00500D1
:1058A00084F82300207829281DD02428DDD1314612
:1058B000042011F027FE22212046FDF72BFCA07FBB
:1058C00000F00300022830D05FF0000080F00101FA
:1058D00030460EF099F80028C7D0FFDFC5E7062054
:1058E000DEE70420DCE701F00300022808D00020F6
:1058F00080F0010130460EF075F8050003D101E09B
:105900000120F5E7FFDF25212046FDF703FC0320FA
:105910008DF80000694605F1E0000FF041FD022816
:10592000A3D00028A1D0FFDF9FE70120CEE703F03E
:1059300056FE9AE72DE9F04387B099461646884609
:105940000746FDF77FFD04004BD02078222848D37E
:10595000232846D0E07F000743D4A07F00F0030057
:10596000022809D05FF0000080F0010138460EF0F7
:1059700039F8050002D00CE00120F5E7A07F00F027
:105980000300022805D00121002238460EF021F83C
:1059900005466946284601F034F9009800B9FFDF52
:1059A00045B10098E03505612078222806D02428EA
:1059B00004D007E000990020086103E0252120467B
:1059C000FDF7A8FB0098012141704762868001A97C
:1059D000C0E902890FF0FFFC022802D0002800D0A5
:1059E000FFDF07B0BDE8F08370B586B00546FDF770
:1059F00029FD017822291ED9807F00F003000228AA
:105A000008D0002080F0010128460DF0EBFF0400D3
:105A10002FD101E00120F5E7FFDF2AE0B4F85E00B6
:105A200004F1620630440178427829B121462846C3
:105A3000FFF711FCB0B9C9E6ADF8042009212846EA
:105A400002AB04F072FC03900028F4D005208DF81E
:105A50000000694604F1E0000FF0A2FC022801D02A
:105A600000B1FFDF02231022314604F15E000DF089
:105A700076FEB4F860000028D0D1A7E610B586B055
:105A80000446FDF7DFFC017822291BD9807F00F056
:105A90000300022808D0002080F0010120460DF00C
:105AA000A1FF040003D101E00120F5E7FFDF06209C
:105AB0008DF80000694604F1E0000FF071FC002849
:105AC00000D0FFDF06B010BD2DE9F05F05460C46A3
:105AD00000270078904601093E4604F1080BBA46BB
:105AE00002297DD0072902D00A2909D146E0686839
:105AF00001780A2905D00D2930D00E292ED0FFDFDC
:105B0000BBE114271C26002C6BD08088A080FDF7F9
:105B100099FC5FEA000900D1FFDF99F817005A46A7
:105B2000400809F11801FDF75CFC6868C089208213
:105B3000696851F8060FC4F812004868C4F81600E6
:105B4000A07E01E03002002020F0060040F00100BD
:105B5000A07699F81E0040F020014DE01A270A2691
:105B6000002CD1D0C088A080FDF76CFC050000D1CE
:105B7000FFDF59462846FFF73FFB7EE10CB1A88BBB
:105B8000A080287A0B287DD006DC01287BD0022853
:105B900008D0032804D135E00D2875D00E2874D024
:105BA000FFDF6AE11E270926002CADD0A088FDF793
:105BB00049FC5FEA000900D1FFDF287B00F0030009
:105BC0000128207A1BD020F001002072297B89084F
:105BD00061F341002072297BC90861F3820001E072
:105BE00041E1F2E02072297B090961F3C3002072D0
:105BF00099F81E0040F0400189F81E103DE140F088
:105C00000100E2E713270D26002CAAD0A088FDF79B
:105C100019FC8146807F00F00300022808D0002094
:105C200080F00101A0880DF0DDFE050003D101E048
:105C30000120F5E7FFDF99F81E0000F00302022AB9
:105C400050D0686F817801F003010129217A4BD08F
:105C500021F00101217283789B0863F341012172D5
:105C60008378DB0863F38201217283781B0963F375
:105C7000C3012172037863F306112172437863F341
:105C8000C71103E061E0A9E090E0A1E0217284F88F
:105C900009A0C178A172022A29D00279E17A62F3BF
:105CA0000001E1720279520862F34101E172027966
:105CB000920862F38201E1720279D20862F3C301B1
:105CC000E1724279217B62F300012173427952082B
:105CD00062F3410121734279920862F382012173D8
:105CE000407928E0A86FADE741F00101B2E74279C1
:105CF000E17A62F30001E1724279520862F34101F4
:105D0000E1724279920862F38201E1724279D2082B
:105D100062F3C301E1720279217B62F30001217316
:105D20000279520862F3410121730279920862F309
:105D3000820121730079C00860F3C301217399F8CF
:105D40000000232831D9262140E018271026E4B38B
:105D5000A088FDF777FB8346807F00F003000228D0
:105D600009D0002080F00101A0880DF03BFE5FEA21
:105D7000000903D101E00120F4E7FFDFE868A0603B
:105D800099F8000040F0040189F8001099F801002A
:105D9000800708D5012020739BF8000023286CD9C8
:105DA0002721584651E084F80CA066E015270F26FD
:105DB0005CB1A088FDF746FB814606225946E8689B
:105DC00008F084FB0120A073A0E041E048463CE0DD
:105DD00016270926E4B3287B20724EE0287B19277A
:105DE0000E26ACB3C4F808A0A4F80CA0012807D074
:105DF000022805D0032805D0042803D0FFDF0DE0DA
:105E0000207207E0697B042801F00F0141F0800156
:105E100021721ED0607A20F003006072A088FDF726
:105E200011FB05460078212827D0232800D0FFDF6A
:105E3000A87F00F00300022813D0002080F00101A9
:105E4000A0880DF0E1FD22212846FDF763F914E05A
:105E500004E0607A20F00300401CDEE7A8F8006050
:105E600010E00120EAE70CB16888A080287A68B3C6
:105E700001280AD002284FD0FFDFA8F800600CB13B
:105E8000278066800020BDE8F09F15270F26002C94
:105E9000E4D0A088FDF7D6FA807F00F00300022846
:105EA00008D0002080F00101A0880DF09BFD0500C6
:105EB00003D101E00120F5E7FFDFD5F81D00062240
:105EC000594608F003FB84F80EA0D6E717270926E9
:105ED000002CC3D0A088FDF7B5FA8146807F00F082
:105EE0000300022808D0002080F00101A0880DF0F6
:105EF00079FD050003D101E00120F5E7FFDF6878B7
:105F0000800701D5022000E00120207299F80000EE
:105F10002328B2D9272159E719270E26002C9DD016
:105F2000A088FDF78FFA5FEA000900D1FFDFC4F80F
:105F300008A0A4F80CA084F808A0A07A40F0030000
:105F4000A07299F81E10C90961F38200A07299F835
:105F50001F2099F81E1012EAD11F05D099F82010C1
:105F600001F01F0110292BD020F00800A07299F831
:105F70001F10607A61F3C3006072697A01F0030157
:105F80000129A2D140F00400607299F81E0000F0CF
:105F900003000228E87A16D0217B60F30001217308
:105FA000AA7A607B62F300006073EA7A520862F3B7
:105FB00041012173A97A490861F3410060735CE7EC
:105FC00040F00800D2E7617B60F300016173AA7AB8
:105FD000207B62F300002073EA7A520862F34101E9
:105FE0006173A97A490861F34100207345E710B550
:105FF000FE4C30B10146102204F1200008F0DDF91A
:10600000012084F8300010BD10B5044600F0E9FD11
:10601000F64920461022BDE81040203108F0CDB9E5
:1060200070B5F24D06004FF0000413D0FBF711F9E4
:1060300008B110240CE00621304608F02EFA411C6D
:1060400005D028665FF0010085F85C0000E00724B9
:10605000204670BD0020F7E7007810F00F0204D052
:10606000012A05D0022A0CD110E0000909D10AE06A
:106070000009012807D0022805D0032803D00428EE
:1060800001D0072070470870002070470620704735
:1060900005282AD2DFE800F003070F171F00087851
:1060A00020F0FF001EE0087820F00F00401C20F0D8
:1060B000F000103016E0087820F00F00401C20F0AF
:1060C000F00020300EE0087820F00F00401C20F097
:1060D000F000303006E0087820F00F00401C20F07F
:1060E000F0004030087000207047072070472DE90D
:1060F000F041804688B00D4600270846FBF7F6F8C9
:10610000A8B94046FDF79EF9040003D02078222864
:1061100015D104E043F2020008B0BDE8F08145B9B2
:10612000A07F410603D500F00300022801D0102013
:10613000F2E7A07FC10601D4010702D50DB1082006
:10614000EAE7E17F090701D50D20E5E700F003004C
:1061500002280DD165B12846FEF75EFF0700DBD1AE
:10616000FBF740FB20B9E878800701D50620D3E78C
:10617000A07F00F00300022808D0002080F0010179
:1061800040460DF02FFC060002D00FE00120F5E79D
:10619000A07F00F0030002280ED0002080F0010153
:1061A000002240460DF015FC060007D0A07F00F04D
:1061B0000300022804D009E00120EFE70420ABE748
:1061C00025B12A4631462046FEF74AFF6946304649
:1061D00000F017FD009800B9FFDF0099022006F1DA
:1061E000E0024870C1F824804A6100220A81A27F3F
:1061F00002F00302022A1CD001200871287800F066
:106200000102087E62F3010008762A78520862F3E0
:10621000820008762A78920862F3C30008762A780A
:10622000D20862F30410087624212046FCF772FF9E
:1062300033E035B30871301D886130784009087744
:106240007078C0F340004877287800F00102887F1A
:1062500062F301008877A27FD20962F38200887717
:10626000E27F62F3C3008877727862F30410887764
:10627000A878C87701F1210228462031FEF711FFE6
:1062800003E0032008710520087625212046FCF74D
:1062900041FFA07F20F04000A07701A900980FF0F7
:1062A0009AF8022801D000B1FFDF384634E72DE923
:1062B000FF4F8DB09A4693460D4600270D98FDF787
:1062C000C1F8060006D03078262806D0082011B084
:1062D000BDE8F08F43F20200F9E7B07F00F0030958
:1062E000B9F1020F11D04DB95846FEF795FE0028BE
:1062F000EDD1B07F00F00300022806D0BBF1000F03
:1063000011D0FBF76FFA20B10DE0BBF1000F50D1B7
:1063100009E006200DF00EFB28B19BF80300800772
:1063200001D50620D3E7B07F00F00300022809D092
:106330005FF0000080F001010D980DF053FB0400A8
:1063400003D101E00120F5E7FFDF852D27D007DC31
:10635000EDB1812D1DD0822D1DD0832D08D11CE0E3
:10636000862D1ED0882D1ED0892D1ED08A2D1ED0A0
:106370000F2020710F281CD003F02EF9D8B1012076
:106380008DF81400201D06902079B0B156E1002050
:10639000EFE70120EDE70220EBE70320E9E7052026
:1063A000E7E70620E5E70820E3E70920E1E70A2020
:1063B000DFE707208BE7112089E7B9F1020F03D04F
:1063C000A56F03D1A06F02E0656FFAE7606F8046AA
:1063D00031D04FF0010001904FF0020000905A467A
:1063E00021463046FEF73CFE02E00000300200206D
:1063F0009BF8000000F00101A87861F30100A8708B
:10640000B17FC90961F38200A870F17F61F3C30015
:10641000A870617861F30410A87020784009287092
:106420006078C0F3400068709BF80200E8700020BC
:106430006871287103E00220019001200090A87883
:1064400098F80210C0F3C000C1F3C00108400390E7
:106450002CD05046FAF7FDFEC0BBDAF80C00FAF774
:10646000F8FE98BBDAF81C00FAF7F3FE70BBDAF816
:106470000C00A060DAF81C00E060607898F8012059
:1064800042EA500161F34100607098F80210C0B216
:1064900000EA111161F3000060700020207700997C
:1064A00006F11700022907D0012106E0607898F86C
:1064B000012002EA5001E5E7002104EB8101486177
:1064C0000199701C022902D0012101E028E000217D
:1064D00004EB81014861A87800F00300012857D13E
:1064E00098F8020000F00300012851D1B9F1020F21
:1064F00004D02A1D691D5846FEF7D3FD287998F867
:10650000041008408DF82C00697998F80520114096
:106510008DF8301008433BD05046FAF79AFE08B188
:106520001020D4E60AF110018B46B9F1020F17D002
:106530000846002104F18C03CDE9000304F5AE7296
:1065400002920BAB2046039AFEF7F4FD0028E8D137
:10655000B9F1020F08D0504608D14FF0010107E011
:1065600050464FF00101E5E75846F5E74FF00001CE
:1065700004F1A403CDE9000304F5B072029281F0A6
:1065800001010CAB2046039AFEF7D4FD0028C8D1C8
:106590006078800733D4A87898F80210C0F38000A0
:1065A000C1F3800108432AD0297898F80000F94AFD
:1065B000B9F1020F06D032F811204300DA4002F0A0
:1065C00003070AE032F810204B00DA4012F003070C
:1065D00005D0012F0AD0022F0AD0032F06D0039A2C
:1065E0006AB1012906D0042904D008E00227F6E7A1
:1065F0000127F4E7012801D0042800D10427B07F47
:1066000040F08000B077F17F039860F30001F177EC
:106610006078800705D50320A071039870B9002029
:1066200029E00220022F18D0012F18D0042F2AD0E1
:106630000020A071B07F20F08000B0772521304687
:10664000FCF768FD05A904F1E0000EF0A9FE10B109
:10665000022800D0FFDF002039E6A071DFE7A0713B
:106660000D22002104F1200007F0D1FE207840F037
:106670000200207001208DF8100004AA31460D9808
:1066800000F098FADAE70120A071D7E72DE9F0438E
:1066900087B09046894604460025FCF7D3FE0600E5
:1066A00006D03078272806D0082007B0BDE8F08350
:1066B00043F20200F9E7B07F00F00300022809D09E
:1066C0005FF0000080F0010120460DF08BF904001E
:1066D00003D101E00120F5E7FFDFA7795FEA0900B8
:1066E00005D0012821D0B9F1020F26D110E0B8F170
:1066F000000F22D1012F05D0022F05D0032F05D086
:10670000FFDF2EE00C252CE001252AE0022528E001
:106710004046FAF79EFDB0B9032F0ED11022414634
:1067200004F11D0007F049FE1BE0012F02D0022FEB
:1067300003D104E0B8F1000F13D00720B5E74046BD
:10674000FAF787FD08B11020AFE71022002104F10D
:106750001D0007F05CFE0621404607F09EFEC4F8CF
:106760001D002078252140F0020020703046FCF703
:10677000D1FC2078C10713D020F001002070022046
:106780008DF8000004F11D0002908DF80450694658
:10679000C3300EF005FE022803D010B1FFDF00E089
:1067A0002577002081E730B587B00D460446FCF719
:1067B00049FE98B1807F00F00300022811D000202C
:1067C00080F0010120460DF00DF904000ED028469E
:1067D000FAF73FFD38B1102007B030BD43F2020098
:1067E000FAE70120ECE72078400701D40820F3E71E
:1067F000294604F13D002022054607F0DEFD207801
:1068000040F01000207001070FD520F00800207024
:1068100007208DF80000694604F1E00001950EF0B4
:10682000BFFD022801D000B1FFDF0020D4E770B522
:106830000D460646FCF706FE18B10178272921D13E
:1068400002E043F2020070BD807F00F003000228E6
:1068500008D0002080F0010130460DF0C3F804009C
:1068600003D101E00120F5E7FFDFA079022809D17B
:106870006078C00706D02A4621463046FEF7EBFC7A
:1068800010B10FE0082070BDB4F860000E280BD2E4
:1068900004F1620102231022081F0CF02AFF0121DB
:1068A00001704570002070BD112070BD70B50646A6
:1068B00014460D460846FAF7CCFC18B92046FAF7FC
:1068C000EEFC08B1102070BDA6F57F40FF380ED059
:1068D0003046FCF7B7FD38B1417822464B08811CA1
:1068E0001846FCF77EFD07E043F2020070BD20462B
:1068F000FDF7A9FD0028F9D11021E01D10F01BFBC8
:10690000E21D294604F1170000F08BF9002070BD4C
:106910002DE9F04104468AB015468846002708460E
:10692000FAF7E4FC18B92846FAF7E0FC18B1102091
:106930000AB0BDE8F0812046FCF784FD060003D0D4
:10694000307827281BD102E043F20200F0E7B07F45
:1069500000F00300022809D05FF0000080F0010180
:1069600020460DF03FF8040003D101E00120F5E7D7
:10697000FFDF2078400702D56078800701D4082027
:10698000D6E7B07F00F00300022805D0A06F05D144
:10699000A16F04E004540200606FF8E7616F407873
:1069A00000B19DB1487810B1B8F1000F0ED0ADB173
:1069B000EA1D06A8E16800F034F9102206A905F1E5
:1069C000170007F0CDFC18B1042707E00720AFE758
:1069D0001022E91D04F12D0007F0EFFCB8F1000FC3
:1069E00006D0102208F1070104F11D0007F0E5FCB4
:1069F0002078252140F0020020703046FCF78AFB09
:106A00002078C10715D020F00100207002208DF8F9
:106A1000000004F11D000290103003908DF8047006
:106A20006946B3300EF0BCFC022803D010B1FFDF82
:106A300000E0277700207BE7F8B515460E460746AD
:106A4000FCF700FD040004D02078222804D00820A0
:106A5000F8BD43F20200F8BDA07F00F00300022859
:106A600002D043F20500F8BD3046FAF7F2FB18B940
:106A70002846FAF7EEFB08B11020F8BD00953288E1
:106A8000B31C21463846FEF709FC112815D0002812
:106A9000F3D1297C4A08A17F62F3C711A177297C31
:106AA000E27F61F30002E277297C890884F82010F4
:106AB000A17F21F04001A177F8BDA17F0907FBD498
:106AC000D6F80200C4F83600D6F80600C4F83A003A
:106AD0003088A0861022294604F1240007F06DFCBE
:106AE000287C4108E07F61F34100E077297C61F375
:106AF0008200E077287C800884F82100A07F40F0A5
:106B00000800A0770020D3E770B50D4606460BB10C
:106B1000072070BDFCF796FC040007D020782228DF
:106B200002D3A07F800604D4082070BD43F2020087
:106B300070BDADB1294630460BF02CFE02F069FB6A
:106B4000297C4A08A17F62F3C711A177297CE27FE3
:106B500061F30002E277297C890884F8201004E0C0
:106B600030460BF03AFE02F054FBA17F21F02001E9
:106B7000A17770BD70B50D46FCF764FC040005D02C
:106B80002846FAF78CFB20B1102070BD43F20200BA
:106B900070BD29462046FEF72FFB002070BD04E0A3
:106BA00010F8012B0AB100207047491E89B2F7D2B4
:106BB0000120704770B51546064602F00DFD040031
:106BC00000D1FFDF207820F00F00801C20F0F000C3
:106BD0002030207066802868A060BDE8704002F018
:106BE000FEBC10B5134C94F83000002808D104F115
:106BF0002001A1F110000EF015FC012084F83000F6
:106C000010BD10B190F8B9202AB10A4890F83500AB
:106C100018B1002003E0B83001E0064834300860C5
:106C2000704708B50023009313460A460DF0D7F8C5
:106C300008BD00003002002018B18178012938D148
:106C400001E010207047018842F60112881A914233
:106C500031D018DC42F60102A1EB020091422AD0A9
:106C60000CDC41B3B1F5C05F25D06FF4C0500818FB
:106C700021D0A0F57060FF381BD11CE001281AD08C
:106C800002280AD117E0B0F5807F14D008DC012873
:106C900011D002280FD003280DD0FF2809D10AE017
:106CA000B0F5817F07D0A0F58070033803D00128AC
:106CB00001D0002070470F2070470A281FD008DC41
:106CC0000A2818D2DFE800F0191B1F1F171F231D09
:106CD0001F21102815D008DC0B2812D00C2810D04A
:106CE0000D2816D00F2806D10DE011280BD08428CE
:106CF0000BD087280FD00320704700207047052055
:106D00007047072070470F20704704207047062007
:106D100070470C20704743F20200704738B50C46AC
:106D2000050041D06946FFF797F9002819D19DF871
:106D30000010607861F3020060706946681CFFF71C
:106D40008BF900280DD19DF80010607861F3C50023
:106D50006070A978C1F34101012903D0022905D04F
:106D6000072038BD217821F0200102E0217841F090
:106D700020012170410704D0A978C90861F3861069
:106D80006070607810F0380F07D0A978090961F3B6
:106D9000C710607010F0380F02D16078400603D53C
:106DA000207840F040002070002038BD70B50446C7
:106DB0000020088015466068FFF7B0FF002816D154
:106DC0002089A189884211D860688078C0070AD0DC
:106DD000B1F5007F0AD840F20120B1FBF0F200FBD0
:106DE0001210288007E0B1F5FF7F01D90C2070BD9B
:106DF00001F201212980002070BD10B504781378BC
:106E000064F3000313700478640864F3410313709F
:106E10000478A40864F3820313700478E40864F32C
:106E2000C30313700478240964F304131370047803
:106E3000640964F3451313700078800960F38613C6
:106E4000137031B10878C10701D1800701D5012045
:106E500000E0002060F3C713137010BD42785307A1
:106E600002D002F0070306E012F0380F02D0C2F39E
:106E7000C20300E001234A7863F302024A704078BB
:106E800010F0380F02D0C0F3C20005E0430702D073
:106E900000F0070000E0012060F3C5024A7070476F
:106EA0002DE9F04F95B00D00824613D0122200213B
:106EB000284607F0ACFA4FF6FF7B05AA0121584699
:106EC00007F06DF80024264637464FF420586FF43B
:106ED000205972E0102015B0BDE8F08F9DF81E001B
:106EE00001280AD1BDF81C1041450BD011EB090057
:106EF0000AD001280CD002280CD0042C0ED0052C6E
:106F00000FD10DE0012400E00224BDF81A6008E072
:106F1000032406E00424BDF81A7002E0052400E012
:106F20000624BDF81A10514547D12C74BEB34FF05A
:106F3000000810AA4FF0070ACDE90282CDE900A8A7
:106F40000DF13C091023CDF81090424631465846C9
:106F500007F0F5F808BBBDF83C002A46C0B210A9FE
:106F60000EF0EBFAC8B9AE81CFB1CDE900A80DF1B2
:106F7000080C0AAE40468CE8410213230022394631
:106F8000584607F0DCF840B9BDF83C00F11CC01EC3
:106F9000C0B22A1D0EF0D1FA10B103209BE70AE01F
:106FA000BDF82900E881062C05D19DF81E00A872C5
:106FB000BDF81C00288100208DE705A806F0FBFF26
:106FC00000288BD0FFF779FE85E72DE9F0471C46B6
:106FD000DDE90978DDF8209015460E00824600D1E3
:106FE000FFDF0CB1208818B1D5B11120BDE8F087C2
:106FF000022D01D0012100E0002106F1140005F06E
:1070000097FEA8F8000002463B462946504603F08A
:107010008CF9C9F8000008B9A41C3C600020E5E721
:107020001320E3E7F0B41446DDE904528DB10023E8
:1070300014B1022C09D101E0012306E00D7CEE071A
:1070400003D025F0010501230D742146F0BC04F0A6
:107050004ABA1A80F0BC70472DE9FE4F91461A8853
:107060001C468A468046FAB102AB494603F05DF9F8
:10707000050019D04046A61C27880CF0F6FD3246C4
:10708000072629463B4600960CF005FA2088234641
:10709000CDE900504A4651464046FFF7C3FF002065
:1070A00020800120BDE8FE8F0020FBE72DE9F0479E
:1070B00086B082460EA8904690E8B000894604AAA1
:1070C00005A903A88DE807001E462A46214650461A
:1070D000FFF77BFF039901B101213970002818D116
:1070E000FA4904F1140204AB0860039805998DE88D
:1070F000070042464946504606F0CDF9A8B1092896
:1071000011D2DFE800F005080510100A0C0C0E0083
:10711000002006B06AE71120FBE70720F9E7082006
:10712000F7E70D20F5E70320F3E7BDF8101003980B
:10713000CDE9000133462A4621465046FFF772FF4B
:10714000E6E72DE9F04389B01646DDE910870D46E4
:1071500081461C461422002103A807F058F901209B
:1071600002218DF810108DF80C008DF81170ADF81B
:10717000146064B1A278D20709D08DF81600E088B7
:10718000ADF81A00A088ADF81800A068079008A80C
:107190000095CDE90110424603A948466B68FFF708
:1071A00085FF09B0BDE8F083F0B58BB0002406463A
:1071B000069407940727089405A80994019400975A
:1071C0000294CDE903400D4610232246304606F0D6
:1071D000B6FF78B90AA806A9019400970294CDE9F0
:1071E0000310BDF8143000222946304606F045FD54
:1071F000002801D0FFF761FD0BB0F0BD06F0D6BB53
:107200002DE9FC410C468046002602F0E5F90546D2
:1072100020780D287ED2DFE800F0BC0713B325BD2F
:1072200049496383AF959B00A848006820B1417825
:1072300041F010014170ADE0404602F0FDF9A9E0D7
:10724000042140460CF0CEFB070000D1FFDF07F120
:107250001401404605F001FDA5BB13214046FDF792
:10726000D3FB97E0042140460CF0BCFB070000D1A3
:10727000FFDFE088ADF800000020B8819DF8000035
:10728000010704D5C00602D5A088B88105E09DF8A5
:10729000010040067ED5A088F88105B9FFDF2246AF
:1072A0002946404601F0ACFC022673E0E188ADF8C7
:1072B00000109DF8011009060FD5072803D00628F5
:1072C0000AD00AE024E0042140460CF08BFB0600C3
:1072D00000D1FFDFA088F0810226CDB9FFDF17E0E3
:1072E000042140460CF07EFB070000D1FFDF07F1D0
:1072F000140006F092FB90F0010F02D1E079000635
:1073000048D5387C022640F00200387405B9FFDF0A
:10731000224600E03DE02946404601F071FC39E09C
:10732000042140460CF05EFB017C002D01F00206BA
:10733000C1F340016171017C21F002010174E7D1C8
:10734000FFDFE5E702260121404602F0A7F921E030
:10735000042140460CF046FB0546606800902089F9
:10736000ADF8040001226946404602F0B8F9287CD5
:1073700020F0020028740DE0002DC9D1FFDFC7E71F
:10738000022600214046FBF7A3F8002DC0D1FFDF05
:10739000BEE7FFDF3046BDE8FC813EB50C0009D0FA
:1073A00001466B4601AA002006F04EFF20B1FFF710
:1073B00084FC3EBD10203EBD00202080A0709DF8C2
:1073C000050002A900F00700FEF762FE50B99DF823
:1073D000080020709DF8050002A9C0F3C200FEF766
:1073E00057FE08B103203EBD9DF8080060709DF86F
:1073F0000500C109A07861F30410A0709DF8051084
:10740000890961F3C300A0709DF80410890601D5B5
:10741000022100E0012161F342009DF8001061F3B8
:107420000000A07000203EBD70B5144606460D4613
:1074300051EA040005D075B10846F9F74EFF78B956
:1074400001E0072070BD2946304606F064FF10B108
:10745000BDE8704031E454B12046F9F73EFF08B171
:10746000102070BD21463046BDE8704095E70020F1
:1074700070BD2DE9FC5F0C4690460546002701785B
:107480000822007A3E46B2EB111F7DD104F10A01B9
:1074900000910A31821E4FF0020A04F1080B01919B
:1074A000092A72D2DFE802F0EDE005F528287BAA70
:1074B000CE00688804210CF095FA060000D1FFDFA9
:1074C000B08928B152270726C3E0000094020020AB
:1074D00051271026002C7DD06888A0800120A07143
:1074E000A88900220099FFF79FFF002873D1A8897F
:1074F0002081288AE081D1E0B5F81290072824D1B4
:10750000E87B000621D5512709F1140086B2002C32
:10751000E1D0A88900220099FFF786FF00285AD100
:107520006888A08084F806A0A88920810120A07323
:10753000288A2082A4F81290A88A009068884B4676
:10754000A969019A01F038FBA8E0502709F112005F
:1075500086B2002C3ED0A88900225946FFF764FF6E
:10756000002838D16888A080A889E080287A072878
:1075700013D002202073288AE081E87BC009607361
:10758000A4F81090A88A01E085E082E00090688865
:107590004B4604F11202A969D4E70120EAE7B5F8E5
:1075A0001290512709F1140086B2002C66D0688829
:1075B00004210CF017FA83466888A080A88900226D
:1075C0000099FFF731FF00286ED184F806A0A88942
:1075D000208101E052E067E00420A073288A208225
:1075E000A4F81290A88A009068884B46A969019A6D
:1075F00001F0E2FAA989ABF80E104FE06888FBF7BA
:1076000021FF0746688804210CF0ECF9064607B90B
:10761000FFDF06B9FFDF687BC00702D051271426C1
:1076200001E0502712264CB36888A080502F06D066
:1076300084F806A0287B594601F0CEFA2EE0287B7C
:10764000A11DF9E7FE49A8894989814205D154273E
:1076500006269CB16888A08020E053270BE068884C
:10766000A080A889E08019E0688804210CF0BAF9AC
:1076700000B9FFDF55270826002CF0D1A8F80060DC
:1076800011E056270726002CF8D06888A08000203B
:1076900013E0FFDF02E0012808D0FFDFA8F8006058
:1076A0000CB1278066800020BDE8FC9F5727072685
:1076B000002CE3D06888A080687AA071EEE7401DB6
:1076C00020F0030009B14143091D01EB4000704760
:1076D00013B5DB4A00201071009848B100246846B9
:1076E0000BF09DFF002C02D1D64A009911601CBD01
:1076F00001240020F4E770B50D461446064686B016
:107700005C220021284606F082FE04B9FFDFA07843
:107710006874A2782188284601F089FA0020A8819F
:10772000E881228805F11401304605F07AFA6A46AC
:107730000121304606F033FC1AE000BF9DF803003B
:10774000000715D5BDF806103046FFF72DFD9DF852
:107750000300BDF8061040F010008DF80300BDF8DE
:107760000300ADF81400FF233046059A06F09BFD98
:10777000684606F020FC0028E0D006B070BD10B5C9
:107780000C4601F1140005F084FA0146627C2046A3
:10779000BDE8104001F080BA30B50446A84891B069
:1077A0004FF6FF75C18905AA284606F0F8FB30E0C0
:1077B0009DF81E00A0422AD001282AD1BDF81C0045
:1077C000B0F5205F03D042F60101884221D10020AC
:1077D00002AB0AAA0CA9019083E8070007200090D9
:1077E000BDF81A1010230022284606F0A8FC38B96C
:1077F000BDF828000BAAC0B20CA90DF09EFE10B176
:10780000032011B030BD9DF82E00A04201D1002010
:10781000F7E705A806F0CFFB0028C9D00520F0E760
:1078200070B5054604210CF0DDF8040000D1FFDF3F
:1078300004F114010C46284605F00FFA21462846AB
:10784000BDE8704005F010BA70B58AB00C46064627
:10785000FBF7F8FD050014D02878222827D30CB1B7
:10786000A08890B101208DF80C0003208DF8100045
:1078700000208DF8110054B1A088ADF818002068E0
:1078800007E043F202000AB070BD0920FBE7ADF843
:1078900018000590042130460CF0A4F8040000D133
:1078A000FFDF04F1140005F00AFA000701D40820F4
:1078B000E9E701F091FE60B108A802210094CDE94A
:1078C000011095F8232003A930466368FFF7EEFB0B
:1078D000D9E71120D7E72DE9F04FB2F802A083468F
:1078E00089B0154689465046FBF7ACFD0746042192
:1078F00050460CF077F80026044605964FF0020833
:107900000696ADF81C6007B9FFDF04B9FFDF4146FA
:10791000504603F04FFF50B907AA06A905A88DE805
:1079200007004246214650466368FFF74EFB444835
:1079300007AB0660DDE9051204F11400CDF80090F4
:10794000CDE90320CDE9013197F82320594650466F
:107950006B6805F0FDF906000AD0022E04D0032E54
:1079600014D0042E00D0FFDF09B03046BDE8F08F00
:10797000BDF81C000028F7D00599CDE9001042465B
:10798000214650466368FFF74DFBEDE7687840F00D
:1079900008006870E8E710B50C46FFF7BFF900284B
:1079A0000BD1607800F00701012905D110F0380FE4
:1079B00002D02078810601D5072010BD40F0C80014
:1079C0002070002010BD2DE9F04F99B004464FF013
:1079D00000081B48ADF81C80ADF82080ADF824806D
:1079E000A0F80880ADF81480ADF81880ADF82880B4
:1079F000ADF82C80007916460D464746012808D080
:107A0000022806D0032804D0042802D0082019B088
:107A1000ACE72046F9F71DFCF0BB2846F9F719FC46
:107A2000D0BB6068F9F762FCB0BB606868B1608980
:107A30002189884202D8B1F5007F05D90C20E6E7FC
:107A4000940200201800002080460EAA06A92846AD
:107A5000FFF7ACF90028DAD168688078C0F34100FC
:107A6000022808D19DF8190010F0380F03D02869BA
:107A7000F9F733FC80B905A92069FFF74FF9002811
:107A8000C5D1206950B1607880079DF8150000F0DD
:107A9000380002D5F0B301E011E0D8BB9DF8140026
:107AA00080060ED59DF8150010F0380F03D06068E1
:107AB000F9F713FC18B96068F9F718FC08B1102041
:107AC000A5E70BA906A8FFF7C9F99DF82D000BA99A
:107AD00020F00700401C8DF82D006069FFF75BFF68
:107AE000002894D10AA9A069FFF718F900288ED1BF
:107AF0009DF8280080062BD4A06940B19DF829008C
:107B000000F00701012923D110F0380F20D0E068E0
:107B100028B100E01CE00078D0B11C2818D20FAAD0
:107B2000611C2046FFF769F90121384661F30F20F7
:107B300082468DF85210B94642F603000F46ADF862
:107B400050000DF13F0218A928680DF0F8FC08B1AB
:107B500007205CE79DF8600015A9CDF80090C01CD7
:107B6000CDE9019100F0FF0B00230BF201225146F9
:107B700014A806F03FF9E8BBBDF854000C90FB4890
:107B80002A8929690092CDE901106B89BDF8382056
:107B90002868069906F02EF9010077D120784FF079
:107BA000020AC10601D4800616D58DF8527042F63D
:107BB0000210ADF85000CDF80C9008A903AACDF83A
:107BC00000A0CDE90121002340F2032214A80B9963
:107BD00006F010F9010059D1E4484D4608380089F3
:107BE000ADF83D000FA8CDE90290CDF80490CDF896
:107BF000109000E00CE04FF007095B460022CDF842
:107C00000090BDF854104FF6FF7006F036F810B132
:107C1000FFF753F8FBE69DF83C00000624D5294603
:107C2000012060F30F218DF852704FF4245003951A
:107C3000ADF8500062789DF80C00002362F300005C
:107C40008DF80C006278CDF800A0520862F3410074
:107C50008DF80C0003AACDE9012540F2032214A8F7
:107C600006F0C8F8010011D1606880B32069A0B99E
:107C700005A906A8FFF7F2F86078800707D49DF8F9
:107C8000150020F038008DF8150006E077E09DF82B
:107C9000140040F040008DF814008DF8527042F648
:107CA0000110ADF85000208940F20121B0FBF1F243
:107CB00001FB1202606809ABCDF80080CDE9010339
:107CC000002314A8059906F095F8010057D12078F3
:107CD000C00728D00395A06950B90AA906A8FFF7E4
:107CE000BDF89DF8290020F00700401C8DF8290000
:107CF0009DF8280007A940F040008DF828008DF875
:107D0000527042F60310ADF8500003AACDF800A05F
:107D1000CDE90121002340F2032214A80A9906F0BC
:107D200069F801002BD1E06868B32946012060F3AF
:107D30000F218DF8527042F60410ADF85000E06843
:107D4000002302788DF8582040788DF85900E068BB
:107D500016AA4088ADF85A00E06800798DF85C00FA
:107D6000E068C088ADF85D00CDF80090CDE9012550
:107D70004FF4027214A806F03DF8010003D00C98ED
:107D800000F0B6FF43E6794803210838017156B187
:107D900000893080BDF824007080BDF82000B080DC
:107DA000BDF81C00F080002031E670B501258AB0D6
:107DB00016460B46012802D0022816D104E08DF8A1
:107DC0000E504FF4205003E08DF80E5042F60100A3
:107DD000ADF80C005BB10024601C60F30F2404AA12
:107DE00008A918460DF0ABFB18B107204BE5102091
:107DF00049E504A99DF820205C48CDE90021801EBA
:107E000002900023214603A802F2012205F0F2FFAE
:107E100010B1FEF752FF36E5544808380EB1C1885C
:107E20003180057100202EE5F0B593B0044601269F
:107E30008DF83E6041F601000F46ADF83C0011AAF6
:107E40000FA93046FFF7B1FF002837D12000474C7B
:107E50004FF00005A4F1080432D01C22002102A832
:107E600006F0D5FA9DF808008DF83E6040F020003D
:107E70008DF8080042F60520ADF83C000420079775
:107E8000ADF82C00ADF8300039480A900EA80D90DE
:107E90000E950FA80990ADF82E506A4609A902A8C0
:107EA000FFF791FD002809D1BDF800006081BDF801
:107EB0000400A081401CE0812571002013B0F0BDBA
:107EC0006581A581BDF84400F4E72DE9F74F274906
:107ED000A0B00024083917940A79A146012A04D0D9
:107EE000022A02D0082023B040E5CA88824201D08D
:107EF0000620F8E721988A46824201D10720F2E75E
:107F00000120214660F30F21ADF848004FF6FF78BD
:107F10008DF86E000691ADF84A8042F6020B8DF89E
:107F200072401CA9ADF86CB0ADF870401391ADF87B
:107F3000508012A806F06EF800252E462F460DAB95
:107F4000072212A9404606F068F898B10A2861D1C4
:107F5000B5B3AEB3ADF86450ADF866609DF85E00A1
:107F60008DF8144019AC012868D06FE09C02002005
:107F70000E5402009DF83A001FB3012859D1BDF8F4
:107F8000381059451FD118A809A901940294CDE9C8
:107F9000031007200090BDF8361010230022404641
:107FA00006F0CDF8B0BBBDF86000042801D006286B
:107FB0004AD1BDF82410219881423AD10F2092E78E
:107FC0003AE0012835D1BDF83800B0F5205F03D084
:107FD00042F6010188422CD1BAF80600BDF83610ED
:107FE000884201D1012700E0002705B19EB1219808
:107FF00081421ED118A809AA01940294CDE9032058
:10800000072000900D4610230022404606F097F806
:1080100000B902E02DE04E460BE0BDF860000228FA
:1080200001D0102810D1C0B217AA09A90DF085FA05
:1080300050B9BDF8369082E7052054E705A917A886
:10804000221D0DF07CFA08B103204CE79DF81400C6
:108050000023001DC2B28DF8142022980092CDE9B1
:1080600001401BA8069905F0C5FE10B902228AF846
:108070000420FEF722FE36E710B50B46401E88B0FE
:1080800084B205AA00211846FEF7B7FE00200DF1C4
:10809000080C06AA05A901908CE8070007200090AB
:1080A0000123002221464FF6FF7005F0E6FD04464D
:1080B000BDF81800012800D0FFDF2046FEF7FDFDC7
:1080C00008B010BDF0B5FF4F044687B038790E46B2
:1080D000032804D0042802D0082007B0F0BD04AA69
:1080E00003A92046FEF762FE0500F6D1606880789D
:1080F000C0F3410002280AD19DF80D0010F0380F9E
:1081000005D02069F9F7E9F808B11020E5E72089E2
:1081100005AA21698DE807006389BDF81020206851
:10812000039905F067FE10B1FEF7C7FDD5E716B15C
:10813000BDF814003080042038712846CDE7F8B52A
:108140000C0006460BD001464FF6FF7500236A4629
:10815000284606F079F820B1FEF7AFFDF8BD1020F3
:10816000F8BD69462046FEF7D9FD0028F8D1A07871
:10817000314600F001032846009A06F094F8EBE738
:1081800030B587B0144600220DF1080C05AD019200
:108190008CE82C00072200920A46014623884FF6FD
:1081A000FF7005F06AFDBDF814102180FEF785FD13
:1081B00007B030BD70B50D4604210BF013FC040070
:1081C00000D1FFDF294604F11400BDE8704004F03F
:1081D0006FBD70B50D4604210BF004FC040000D106
:1081E000FFDF294604F11400BDE8704004F083BDB0
:1081F00070B50D4604210BF0F5FB040000D1FFDF44
:10820000294604F11400BDE8704004F09BBD70B530
:10821000054604210BF0E6FB040000D1FFDF2146F8
:1082200028462368BDE870400122FEF715BF70B5EF
:10823000064604210BF0D6FB040000D1FFDF04F159
:10824000140004F026FD401D20F0030511E0011D7F
:1082500000880022431821463046FEF7FDFE002824
:108260000BD0607CABB2684382B2A068011D0BF0FA
:1082700076FAA06841880029E9D170BD70B505463D
:1082800004210BF0AFFB040000D1FFDF214628469C
:108290006368BDE870400222FEF7DEBE70B50E4690
:1082A000054601F099F9040000D1FFDF012020729A
:1082B00066726580207820F00F00001D20F0F0002D
:1082C00040302070BDE8704001F089B910B5044617
:1082D000012900D0FFDF2046BDE810400121FAF758
:1082E000F7B82DE9F04F97B04FF0000A0C00834625
:1082F000ADF814A0D04619D0E06830B1A068A8B19C
:108300000188ADF81410A0F800A05846FBF79AF8C1
:10831000070043F2020961D0387822285CD3042197
:1083200058460BF05FFB050005D103E0102017B0A5
:10833000BDE8F08FFFDF05F1140004F0AAFC401D3A
:1083400020F00306A078012803D0022801D00720DE
:10835000EDE7218807AA584605F021FE30BB07A8A3
:1083600005F029FE10BB07A805F025FE48B99DF8C9
:108370002600012805D1BDF82400A0F524510239BA
:1083800002D04FF45050D2E7E068B0B1CDE902A07E
:108390000720009005AACDF804A00492A2882188A5
:1083A000BDF81430584605F068FC10B1FEF785FCA6
:1083B000BDE7A168BDF8140008809DF81F00C00645
:1083C00002D543F20140B2E70B9838B1A1780078AA
:1083D000012905D080071AD40820A8E74846A6E757
:1083E000C007F9D002208DF83C00A8684FF00009C2
:1083F000A0B1697C4288714391420FD98AB2B3B26D
:10840000011D0BF062F98046A0F800A006E00320F1
:108410008DF83C00D5F800804FF001099DF8200050
:1084200010F0380F00D1FFDF9DF820002649C0F37F
:10843000C200084497F8231010F8010C884201D9B3
:108440000F2074E72088ADF8400014A90095CDE90D
:108450000191434607220FA95846FEF727FE002840
:1084600091D19DF8500050B9A078012807D1687CBF
:10847000B3B2704382B2A868011D0BF03AF9002034
:1084800055E770B5064615460C460846FEF7D4FB80
:10849000002805D12A4621463046BDE8704084E4D4
:1084A00070BD12E570B51E4614460D000ED06CB1BD
:1084B000616859B160B10349C988814208D0072079
:1084C00070BD000094020020115402001020F7E754
:1084D0002068FEF7B1FB0028F2D13246214628463B
:1084E000BDE87040FFF76FBA70B515460C0006D0B6
:1084F00038B1FE490989814203D00720E0E7102006
:10850000DEE72068FEF798FB0028D9D129462046EF
:10851000BDE87040D6E570B5064686B00D461446F7
:108520001046F8F7BCFED0BB6068F8F7DFFEB0BBC2
:10853000A6F57F40FF3803D03046FAF783FF80B1BD
:1085400028466946FEF7ACFC00280CD19DF81010B7
:108550000F2008293DD2DFE801F008060606060ACA
:108560000A0843F2020006B0AAE70320FBE79DF8E1
:108570000210012908D1BDF80010B1F5C05FF2D09A
:108580006FF4C052D142EED09DF8061001290DD1F2
:10859000BDF80410A1F52851062907D200E029E012
:1085A000DFE801F0030304030303DCE79DF80A108E
:1085B00001290FD1BDF80810B1F5245FD3D0A1F681
:1085C0000211B1F50051CED00129CCD0022901D140
:1085D000C9E7FFDF606878B9002305AA294630465D
:1085E00005F032FE10B1FEF768FBBCE79DF8140001
:1085F000800601D41020B6E76188224628466368C9
:10860000FFF7BEFDAFE72DE9F043814687B088460E
:1086100014461046F8F743FE18B1102007B0BDE825
:10862000F083002306AA4146484605F00DFE10B12E
:10863000FEF743FBF2E79DF81800C00602D543F2AF
:108640000140EBE70025072705A801950097029553
:10865000CDE9035062884FF6FF734146484605F066
:108660006EFD060013D16068F8F719FE60B9606806
:108670000195CDE902500097049523886288414610
:10868000484605F05CFD0646BDF8140020803046E3
:10869000CEE739B1954B0A889B899A4202D843F2BA
:1086A000030070471DE610B586B0904C0423ADF86A
:1086B0001430638943B1A4898C4201D2914205D917
:1086C00043F2030006B010BD0620FBE7ADF8101022
:1086D000002100910191ADF8003002218DF80210C7
:1086E00005A9029104A90391ADF812206946FFF78C
:1086F000F8FDE7E72DE9FC4781460D460846F8F707
:10870000A8FD88BB4846FAF79DFE5FEA00080AD03C
:1087100098F80000222829D3042148460BF062F97A
:10872000070005D103E043F20200BDE8FC87FFDF4C
:1087300007F1140004F0C3FA06462878012803D094
:10874000022804D00720F0E7B0070FD502E016F0AA
:108750001C0F0BD0A8792C1DC00709D0E08838B1B8
:10876000A068F8F776FD18B11020DEE70820DCE7F6
:1087700021882A780720B1F5847F35D01EDC40F2AD
:108780000315A1F20313A94226D00EDCB1F5807FB8
:10879000CBD003DCF9B1012926D1C6E7A1F580735E
:1087A000013BC2D0012B1FD113E0012BBDD0022B06
:1087B0001AD0032BB9D0042B16D112E0A1F2091262
:1087C000082A11D2DFE802F00B0404101010100484
:1087D000ABE7022AA9D007E0012AA6D004E03207BD
:1087E00000E0F206002AA0DACDB200F0F5FE50B1AA
:1087F00098F82300CDE90005FA8923463946484612
:10880000FEF79FFC91E711208FE72DE9F04F8BB029
:108810001F4615460C4683460026FAF713FE28B17C
:108820000078222805D208200BB081E543F202002F
:10883000FAE7B80801D00720F6E7032F00D1002798
:108840004FF6FF79CCB1022D71D32046F8F74EFDDB
:1088500030B904EB0508A8F10100F8F747FD08B1AD
:108860001020E1E7AD1E38F8028CAAB22146484636
:1088700005F03EFE40455AD1ADB21C49B80702D5BD
:108880008889401C00E001201FFA80F8F80701D019
:108890008F8900E04F4605AA4146584605F07FFB08
:1088A0004FF0070A4FF00009FCB1204608E040886D
:1088B00010283CD8361D304486B2AE4237D2A019BB
:1088C00002884245F3D352E09DF8170002074ED5C7
:1088D0007CB304EB0608361DB8F80230B6B2102B94
:1088E00025D89A19AA4222D802E040E0940200203A
:1088F000B8F8002091421AD1C0061BD5CDE900A9D5
:108900000DF1080C0AAAA11948468CE80700B8F82E
:1089100000100022584605F0B0F910B1FEF7CDF96D
:1089200082E7B8F80200BDF82810884202D00B2078
:108930007AE704E0B8F80200304486B206E0C006E8
:1089400004D55846FEF730FC00288AD19DF8170060
:10895000BDF81A1020F010008DF81700BDF81700B0
:10896000ADF80000FF235846009A05F09CFC05A8CE
:1089700005F021FB18B9BDF81A10B942A4D9042199
:1089800058460BF02FF8040000D1FFDFA2895AB13E
:10899000CDE900A94D46002321465846FEF7D1FBFC
:1089A0000028BDD1A5813FE700203DE72DE9FF4F1D
:1089B0008BB01E4617000D464FF0000412D0B008D1
:1089C00002D007200FB0B3E4032E00D100265DB122
:1089D0000846F8F782FC28B93888691E0844F8F779
:1089E0007CFC08B11020EDE7C74AB00701D5D1895A
:1089F00000E00121F0074FF6FF7802D0D089401E39
:108A000000E0404686B206AA0B9805F0C8FA4FF07F
:108A100000094FF0070B0DF1140A38E09DF81B0018
:108A2000000734D5CDF80490CDF800B0CDF808900B
:108A3000CDE9039A434600220B9805F080FB60BB0A
:108A400005B3BDF814103A8821442819091D8A423B
:108A500030D3BDF81E2020F8022BBDF8142020F8DA
:108A6000022BCDE900B9CDE90290CDF810A0BDF8F8
:108A70001E10BDF8143000220B9805F060FB08B101
:108A800003209FE7BDF814002044001D84B206A80F
:108A900005F091FA20B10A2806D0FEF70EF991E709
:108AA000BDF81E10B142B9D934B17DB13888A11CCE
:108AB000884203D20C2085E7052083E72246294619
:108AC000404605F015FD014628190180A41C3C8094
:108AD000002077E710B50446F8F7E1FB08B1102055
:108AE00010BD8948C0892080002010BDF0B58BB032
:108AF0000D4606461422002103A805F088FC01203B
:108B00008DF80C008DF8100000208DF81100ADF8E4
:108B100014503046FAF796FC48B10078222812D358
:108B2000042130460AF05EFF040005D103E043F261
:108B300002000BB0F0BDFFDF04F11400074604F0A3
:108B4000BEF8800601D40820F3E7207C022140F023
:108B50000100207409A80094CDE90110072203A99F
:108B600030466368FEF7A2FA20B1217C21F00101B2
:108B70002174DEE729463046F9F79BFC08A9384600
:108B800004F08CF800B1FFDFBDF82040172C01D2B3
:108B9000172000E02046A84201D92C4602E0172CFD
:108BA00000D2172421463046FFF713FB21463046FA
:108BB000F9F7A3F90020BCE7F8B51C4615460E46A8
:108BC000069F0BF040F82346FF1DBCB231462A46F3
:108BD00000940AF02CFCF8BD70B50C4605460E2238
:108BE0000021204605F013FC002020802DB1012D2E
:108BF00001D0FFDF64E4062000E00520A0715FE4FF
:108C000010B548800878134620F00F00001D20F0B2
:108C1000F00080300C4608701422194604F1080058
:108C200005F0CBFB00F0DBFC3748046010BD2DE9FC
:108C3000F047DFF8D890491D064621F0030117469A
:108C40000C46D9F800000AF008FD050000D1FFDF4E
:108C50004FF000083560A5F800802146D9F80000E3
:108C60000AF0FBFC050000D1FFDF7560A5F800806D
:108C70007FB104FB07F1091D0BD0D9F800000AF001
:108C8000ECFC040000D1FFDFB460C4F80080BDE854
:108C9000F087C6F80880FAE72DE9F0411746491D2C
:108CA00021F00302194D06460168144628680AF0AF
:108CB000FFFC2246716828680AF0FAFC3FB104FB09
:108CC00007F2121D03D0B16828680AF0F1FC0420F5
:108CD0000AF030FE044604200AF034FE201A01286F
:108CE00004D12868BDE8F0410AF0ACBCBDE8F081D1
:108CF00010B50C4605F022F900B1FFDF2046BDE8B3
:108D00001040FDF7DABF0000940200201800002098
:108D100038B50C468288817B19B14189914200D9CE
:108D20000A462280C188121D90B26A4609F066FE8A
:108D3000BDF80000032800D30320C1B2208801F051
:108D40001AF838BD38B50C468288817B19B1018983
:108D5000914200D90A462280C188121D90B26A460B
:108D600009F04CFEBDF80000022800D30220C1B279
:108D7000208801F000F8401CC0B238BD2DE9FF5F2B
:108D800082468B46F74814460BF10302D0E90110E6
:108D9000CDE9021022F0030201A84FF49071019274
:108DA0000AF03DFCF04E002C02D1F049019A8A6095
:108DB000019901440191B57F05F1010504D1E8B2A3
:108DC0000CF03EFB00B1FFDF019800EB0510C01C6A
:108DD00020F0030101915CB9707AB27A1044C2B2FA
:108DE00000200870B08C80B204F007FF00B1FFDFF4
:108DF0000198716A08440190214601A800F07EFFA5
:108E000080460198C01C20F003000190B37AF27AEA
:108E1000717A04B100200AF0F8FC0199084401902D
:108E2000214601A800F0B2FFCF4800273D4690F848
:108E300001900CE0284600F044FF064681788088C7
:108E4000F9F7F2F871786D1C00FB0177EDB24D4532
:108E5000F0D10198C01C20F00300019004B1002063
:108E60003946F9F7ECF80199002708440190BE480B
:108E70003D4690F801900CE0284600F022FF06469F
:108E8000C1788088FEF71BFC71786D1C00FB0177B0
:108E9000EDB24D45F0D10198C01C20F003000190C7
:108EA00004B100203946FEF713FC01994FF0000988
:108EB00008440190AC484D4647780EE0284600F043
:108EC00000FF0646807B30B106F1080002F096F9FB
:108ED000727800FB02996D1CEDB2BD42EED1019893
:108EE000C01C20F00300019004B100209F494A7883
:108EF000494602F087F9019908440190214601A8EA
:108F000000F0B2FE0198C01D20F007000190DAF8D1
:108F10000010814204D3A0EB0B01B1F5803F04DBCC
:108F20004FF00408CAF8000004E0CAF80000B8F1E5
:108F3000000F03D0404604B0BDE8F09F84BB8C49CD
:108F40000020019A0EF072FBFBF718FA864C207F86
:108F50000090607F012825D0002328B3002282489A
:108F600000211030F8F744FA00B1FFDF7E49E07FBE
:108F70002031FEF759FF00B1FFDF7B484FF4F67256
:108F80000021443005F043FA77480421443080F84A
:108F9000E91180F8EA11062180F8EB110321017133
:108FA0000020C8E70123D8E702AAD8E770B56E4CC5
:108FB00006464434207804EB4015E078083598B92B
:108FC000A01990F8E80100280FD0A0780F2800D34E
:108FD000FFDF20220021284605F019FA687866F3A1
:108FE000020068700120E070284670BD2DE9F04154
:108FF00005460C4600270078052190463E46B1EB19
:10900000101F00D0FFDF287A50B101280ED0FFDFFB
:10901000A8F800600CB1278066800020BDE8F081D0
:109020000127092674B16888A08008E00227142669
:1090300044B16888A0802869E060A88A2082287BE3
:109040002072E5E7A8F80060E7E730B5464C01205C
:10905000002120706170207260720322A272E0729F
:109060006177217721732174052121831F21618379
:10907000607440A161610A21A177E07739483B4DD6
:10908000B0F801102184C07884F822004FF4B06059
:1090900060626868C11C21F00301814200D0FFDFDB
:1090A0006868606030BD30B5304C15686368103357
:1090B0009D4202D20420136030BD2B4B5D785A686C
:1090C00002EB0512107051700320D08017209080A1
:1090D0000120D0709070002090735878401C587018
:1090E000606810306060002030BD70B506461E48D4
:1090F0000024457807E0204600F0E3FD0178B14206
:1091000004D0641CE4B2AC42F5D1002070BDF7B5C8
:10911000074608780C4610B3FFF7E7FF0546A7F1AE
:109120002006202F06D0052E19D2DFE806F00F38D2
:109130003815270000F0D0FD0DB1697800E000215E
:10914000401AA17880B20844FF2808D8A07830B12E
:10915000A088022831D202E0608817282DD207208B
:10916000FEBD000018540200B00300201C000020C7
:10917000000000206E52463578000000207AE0B1F1
:1091800061881729EBD3A1881729E8D3A179002991
:10919000E5D0E1790029E2D0402804D9DFE7242F87
:1091A0000BD1207A48B161884FF6FB70814202D81A
:1091B000A188814201D90420D2E765B9207802AAAA
:1091C0000121FFF770FF0028CAD12078FFF78DFF3B
:1091D000050000D1FFDF052E18D2DFE806F0030BF3
:1091E0000E081100A0786870A088E8800FE0608801
:1091F000A8800CE0A078A87009E0A078E87006E0EC
:1092000054F8020FA8606068E86000E0FFDF00200B
:10921000A6E71A2835D00DDC132832D2DFE800F09B
:109220001B31203131272723252D3131293131318F
:10923000312F0F00302802D003DC1E2821D1072057
:1092400070473A3809281CD2DFE800F0151B0F1BC5
:109250001B1B1B1B07000020704743F204007047D4
:1092600043F202007047042070470D2070470F2022
:109270007047082070471120704713207047062060
:1092800070470320704710B5007800F0010009F026
:10929000A7FBBDE81040BCE710B5007800F0010066
:1092A00009F0A7FBBDE81040B3E70EB5017801F067
:1092B00001018DF80010417801F001018DF80110D5
:1092C0000178C1F340018DF802104178C1F34001EB
:1092D0008DF80310017889088DF804104178890809
:1092E0008DF8051081788DF80610C1788DF807107B
:1092F00000798DF80800684608F02DFCFFF789FF1B
:109300000EBD2DE9FC5FDFF8F883FE4C00264FF41C
:1093100090771FE0012000F07CFD0120FFF746FE62
:1093200005463946D8F808000AF097F9686000B990
:10933000FFDF686808F0DDFAB0B12846FAF762FB93
:10934000284600F06CFD28B93A466968D8F808004C
:109350000AF0AEF994F9E9010428DBDA02200AF0F8
:10936000E9FA07460025AAE03A466968D8F80800F5
:109370000AF09EF9F2E7B8F802104046491C89B29B
:10938000A8F80210B94201D3002141800221B8F8A7
:1093900002000AF027FB002866D0B8F802006946F0
:1093A00009F084FAFFF735FF00B1FFDF9DF80000F8
:1093B000019078B1B8F802000AF057FC5FEA0009A2
:1093C00000D1FFDF484609F0C6FE18B1B8F8020028
:1093D00002F0DEF9B8F802000AF035FC5FEA000995
:1093E00000D1FFDF484609F0AEFEE8BB0321B8F824
:1093F00002000AF0F7FA5FEA000B4BD1FFDF49E009
:10940000DBF8100010B10078FF284DD0022000F0EA
:1094100000FD0220FFF7CAFD8246484609F09FFF83
:10942000CAF8040000B9FFDFDAF804000AF067F8B0
:10943000002100900170B8F802105046AAF80210FE
:1094400002F0ACF848460AF05CF800B9FFDF01987A
:1094500000B10126504600F0E2FC18B99AF801006C
:10946000000705D5009800E027E0CBF8100011E0D8
:10947000DBF8101039B10878401C10F0FF000870BC
:1094800008D1FFDF06E000221146484600F0EAFB63
:1094900000B9FFDF94F9EA01022805DBB8F8020001
:1094A00002F043F80028ABD194F9E901042804DB69
:1094B00048460AF08AF800B101266D1CEDB2BD42A3
:1094C00004D294F9EA010228BFF655AF002E7FF4CA
:1094D0001DAFBDE8FC5F032000F09BBC10B5884CBD
:1094E000E06008682061AFF2E510F9F7EEFC60700B
:1094F00010BD8448002144380170814801708249C0
:109500004160704770B505464FF080500C46D0F86A
:10951000A410491C05D1D0F8A810C9430904090CAE
:109520000BD050F8A01F01F00101297041682160A3
:109530008068A080287830B970BD062120460DF0E3
:10954000FAFC01202870607940F0C000607170BDA5
:1095500070B54FF080540D46D4F88010491C0BD1E3
:10956000D4F88410491C07D1D4F88810491C03D1C1
:10957000D4F88C10491C0CD0D4F880100160D4F8B9
:1095800084104160D4F888108160D4F88C10C160D8
:1095900002E010210DF0CFFCD4F89000401C0BD15C
:1095A000D4F89400401C07D1D4F89800401C03D193
:1095B000D4F89C00401C09D054F8900F28606068D3
:1095C0006860A068A860E068E86070BD2846BDE8F3
:1095D000704010210DF0AFBC4A480079E6E470B548
:1095E000484CE07830B3207804EB4010407A00F02B
:1095F0000700204490F9E801002800DCFFDF207814
:10960000002504EB4010407A00F00700011991F8A2
:10961000E801401E81F8E8012078401CC0B22070AB
:109620000F2800D12570A078401CA0700DF07AFBA7
:10963000E57070BDFFDF70BD3EB5054603210AF041
:10964000D1F9044628460AF0FEFA054604B9FFDFC0
:10965000206918B10078FF2800D1FFDF01AA694610
:10966000284600F0FFFA60B9FFDF0AE0002202A9F5
:10967000284600F0F7FA00B9FFDF9DF8080000B1B6
:10968000FFDF9DF80000411E8DF80010EED220692A
:109690000199884201D1002020613EBD70B5054688
:1096A000A0F57F400C46FF3800D1FFDF012C01D030
:1096B000FFDF70BDFFF790FF040000D1FFDF2078CF
:1096C00020F00F00401D20F0F00050302070658029
:1096D0000020207201202073BDE870407FE72DE953
:1096E000F04116460D460746FFF776FF040000D10D
:1096F000FFDF207820F00F00401D20F0F00005E093
:109700001C000020F403002038140020503020708A
:1097100067800120207228682061A888A0822673B3
:10972000BDE8F0415BE77FB5FFF7DFFC040000D147
:10973000FFDF02A92046FFF7EBFA054603A9204602
:10974000FFF700FB8DF800508DF80100BDF8080010
:10975000001DADF80200BDF80C00001DADF80400BE
:10976000E088ADF80600684609F024F9002800D02A
:10977000FFDF7FBD2DE9F05FFC4E8146307810B1F0
:109780000820BDE8F09F4846F7F789FD08B1102092
:10979000F7E7F74C207808B9FFF757FCA17A607A11
:1097A0004D460844C4B200F097FAA04207D2201AEE
:1097B000C1B22A460020FFF776FC0028E1D171688B
:1097C000EB48C91C002721F003017160B3463E46F7
:1097D0003D46BA463C4690F801800AE0204600F03B
:1097E00070FA4178807B0E4410FB0155641CE4B292
:1097F0007F1C4445F2D10AEB870000EBC600DC4E2B
:1098000000EB85005C46F17A012200EB8100DBF879
:109810000410451829464846FFF7B0FA070012D051
:109820000020FFF762FC05000BD005F11300616812
:1098300020F00300884200D0FFDF7078401E707077
:10984000656038469DE7002229464846FFF796FAAC
:1098500000B1FFDFD9F8000060604FF6FF70608054
:109860000120207000208CE72DE9F0410446BF481C
:1098700017460D46007810B10820BDE8F081084673
:10988000F7F7E7FC08B11020F7E7B94E307808B9D0
:10989000FFF7DBFB601E1E2807D8012C23D1287898
:1098A000FE2820D8B0770020E7E7A4F120001F2889
:1098B00005D8E0B23A462946BDE8F04127E4A4F1D4
:1098C00040001F2805D829462046BDE8F04100F099
:1098D000CEBAA4F1A0001F2805D829462046BDE82D
:1098E000F04100F000BB0720C7E72DE9F05F81469B
:1098F0000F460846F7F7D3FC48B94846F7F7EDFCA2
:1099000028B909F1030020F00301494501D01020D6
:1099100037E797484FF0000B4430817869B14178C0
:10992000804600EB411408343E883A460021204628
:1099300000F083FA050004D027E0A7F800B0052066
:109940001FE7B9F1000F24D03888B04201D90C25A7
:109950001FE0607800F00700824600F05AFA08EB3A
:109960000A063A4696F8E8014946401C86F8E8019E
:10997000204600F062FA054696F8E801401E86F897
:10998000E801032000F045FA2DB10C2D01D0A7F815
:1099900000B02846F5E6754F5046BAF1010F25D0C4
:1099A00002280DD0BAF1030F35D0FFDF98F801106F
:1099B0004046491CC9B288F801100F2937D038E059
:1099C000606828B16078000702D46088FFF734FE31
:1099D00098F8EA014446012802D17878F9F794FA18
:1099E00094F9EA010428E1DBFFDFDFE7616821B1D8
:1099F0004FF49072B86809F05BFE98F8E9014446AC
:109A0000032802D17878F9F77FFA94F9E90104285C
:109A1000CCDBFFDFCAE76078C00602D56088FFF7BD
:109A20000BFE98F9EB010628C0DBFFDFBEE780F8EC
:109A300001B08178491E88F8021096F8E801401CB0
:109A400086F8E801A5E770B50C460546F7F701FC76
:109A500018B92046F7F723FC08B1102070BD28463E
:109A60000BF025FD207008B1002070BD042070BDF2
:109A700070B505460BF034FDC4B22846F7F72DFC4F
:109A800008B1102070BD35B128782C7018B1A042F3
:109A900001D0072070BD2046FDF77EFE052805D1C8
:109AA0000BF021FD012801D0002070BD0F2070BDFA
:109AB00070B5044615460E460846F7F7CAFB18B9B6
:109AC0002846F7F7ECFB08B1102070BD022C03D03C
:109AD000102C01D0092070BD2A46314620460BF0DB
:109AE0002CFD0028F7D0052070BD70B514460D463A
:109AF0000646F7F7AEFB38B92846F7F7D0FB18B99A
:109B00002046F7F7EAFB08B1102070BD224629462F
:109B100030460BF014FD0028F7D0072070BD3EB58D
:109B20000446F7F7BCFB08B110203EBD684607F0BD
:109B300086FFFFF76EFB0028F7D19DF80600207026
:109B4000BDF808006080BDF80A00A08000203EBD7E
:109B500070B505460C460846F7F7BFFB20B95CB167
:109B60002068F7F79CFB28B1102070BD1C00002076
:109B7000B0030020A08828B121462846BDE87040E7
:109B8000FDF762BE0920F0E770B504460D460846B1
:109B9000F7F75FFB90BB601E1E280ED8032C01D97F
:109BA0000720E2E704B9FFDFFE4800EB840050F82D
:109BB000041C2846BDE870400847A4F120001F2877
:109BC00005D829462046BDE87040FAF746BBA4F107
:109BD00060001F2805D829462046BDE87040F8F7E8
:109BE000E4BCF02C0BD0BF2CDAD1A878298800F087
:109BF000010001F089FB78B10020B6E703E0A86816
:109C0000F7F727FB08B11020AFE7284608F037FF29
:109C1000BDE87040FFF7FDBA0820A6E770B504461E
:109C20000D460846F7F73BFB30B9601E1E280FD8DB
:109C30002846F7F70EFB08B1102096E7012C03D059
:109C4000022C01D0032C01D106208EE707208CE7DF
:109C5000A4F120001F28F9D829462046BDE870400D
:109C6000FAF76CBB09F03EBA38B50446CE48007B23
:109C700000F00105F9B904F0ECFB0DB1226800E039
:109C80000022CA484178C06807F00EFCC74810306F
:109C9000C0788DF8000010B1012802D004E0012046
:109CA00000E000208DF80000684607F035FFBD4851
:109CB000243808F071FC002D02D020682830206084
:109CC00038BD30B5B84D04466878A04200D8FFDFF3
:109CD000686800EB041030BD70B5B34800252C4611
:109CE000467807E02046FFF7ECFF4078641C2844E4
:109CF000C5B2E4B2B442F5D1284636E72DE9F041C9
:109D00000C4607464FF0000800F01FF90646FF28F2
:109D100001D94FF013083868C01C20F003023A60E4
:109D200054EA080421D1A048F3B2072128300DF0ED
:109D30000FFB09E0072C10D2DFE804F00604080846
:109D40000A0406009A4804E09A4802E09A4800E0B3
:109D50009A480DF01DFB054600E0FFDFA54200D04C
:109D6000FFDF641CE4B2072CE4D3386800EB061074
:109D70003860404681E5021D5143452900D2452106
:109D80000844C01CB0FBF2F0C0B270472DE9FC5F84
:109D9000064685484FF000088B464746444690F8F3
:109DA000019022E02046FFF78CFF050000D1FFDF85
:109DB000687869463844C7B22846FEF7A9FF82464C
:109DC00001A92846FEF7BEFF0346BDF8040052462F
:109DD000001D81B2BDF80000001D80B209F080FEB8
:109DE0006A78641C00FB0288E4B24C45DAD1306822
:109DF000C01C20F003003060BBF1000F00D0002039
:109E00004246394609F07AFE316808443060BDE8C0
:109E1000FC9F6549443108710020C8707047624951
:109E20004431CA782AB10A7801EB421108318142E3
:109E300001D001207047002070472DE9F04106460F
:109E40000078154600F00F0400201080601E0F46B9
:109E5000052800D3FFDF53482A46183800EB84005A
:109E6000394650F8043C3046BDE8F04118472DE92A
:109E7000F0414D4E0C46402806D0412823D04228C0
:109E80002BD0432806D123E0A07861780D18E17823
:109E9000814201D90720F0E42078012801D913205C
:109EA000EBE4FF2D08D80BF0B5FC07460CF0F2FEF2
:109EB000381A801EA84201DA1220DEE42068B06061
:109EC000207930730DE0BDE8F041084600F078B825
:109ED00008780228DED8307703E008780228D9D83D
:109EE00070770020C9E4F8B500242F4DA02805D0D4
:109EF000A12815D0A22806D00720F8BD087800F0C8
:109F00000100E8771FE00E4669463046FDF743FD45
:109F10000028F2D130882884B07885F8220012E039
:109F200008680921F82801D3820701D00846F8BD46
:109F30006A7C02F00302012A04D16A8BD73293B201
:109F40008342F3D868622046F8BD2DE9F047DFF878
:109F500058900026344699F8090099F80A2099F893
:109F600001700244D5B299F80B20104400F0FF08AC
:109F700008E02046FFF7A5FE817B407811FB0066D4
:109F8000641CE4B2BC42F4D199F8091099F80A00B3
:109F900029442944414400B1012008443044BDE82B
:109FA000F08700003C540200B00300201C00002099
:109FB0005B41000025B30000DD2F0000335201009B
:109FC00038B50446407800F00300012803D0022889
:109FD0000BD0072038BD606858B1F7F787F9D0B9C2
:109FE0006068F7F77AF920B915E06068F7F731F99A
:109FF00088B969462046FCF72FF80028EAD1607836
:10A0000000F00300022808D19DF8000028B1606824
:10A01000F7F763F908B1102038BD6189F8290DD828
:10A02000208988420AD8607800F003020A48012A91
:10A0300006D1D731426A89B28A4201D2092038BD9D
:10A0400094E80E0000F1100585E80E000AB9002121
:10A050000183002038BD0000B00300202DE9F0414D
:10A06000074614468846084601F08AFD064608EB76
:10A0700088001C22796802EBC0000D18688C58B16A
:10A080004146384601F08BFD014678680078C200F1
:10A09000082305F120000CE0E88CA8B141463846C1
:10A0A00001F084FD0146786808234078C20005F17C
:10A0B000240009F054FB38B1062121726681D0E9F1
:10A0C0000010C4E9031009E0287809280BD0052006
:10A0D000207266816868E060002028702046BDE834
:10A0E000F04101F02EBD072020726681F4E72DE9D2
:10A0F000F04116460D460746406801EB85011C22DB
:10A1000002EBC1014418204601F072FD40B100216C
:10A11000708865F30F2160F31F4106200DF0F2F9FE
:10A1200009202070324629463846BDE8F04195E7BF
:10A130002DE9F0410E46074600241C21F07816E078
:10A1400004EB8403726801EBC303D25C6AB1FFF7CE
:10A1500043FA050000D1FFDF6F802A4621463046D2
:10A16000FFF7C5FF0120BDE8F081641CE4B2A04206
:10A17000E6D80020F7E770B5064600241C21C07819
:10A180000AE000BF04EB8403726801EBC303D51837
:10A190002A782AB1641CE4B2A042F3D8402070BDF2
:10A1A00028220021284604F032F97068808928812D
:10A1B000204670BD70B5034600201C25DC780CE0FD
:10A1C00000EB80065A6805EBC6063244167816B1D5
:10A1D000128A8A4204D0401CC0B28442F0D8402087
:10A1E00070BDF0B5044600201C26E5780EE000BFE7
:10A1F00000EB8007636806EBC7073B441F788F427C
:10A2000002D15B78934204D0401CC0B28542EFD8A3
:10A210004020F0BD0078032801D0002070470120C5
:10A2200070470078022801D0002070470120704755
:10A230000078072801D000207047012070472DE9E1
:10A24000F041064688461078F1781546884200D3DA
:10A25000FFDF2C781C27641CF078E4B2A04201D800
:10A26000201AC4B204EB8401706807EBC1010844F2
:10A27000017821B14146884708B12C7073E72878EE
:10A28000A042E8D1402028706DE770B514460B88D5
:10A290000122A240134207D113430B8001230A225B
:10A2A000011D09F026FA047070BD2DE9FF4F81B041
:10A2B0000878DDE90E7B9A4691460E4640072CD47D
:10A2C000019809F0D2FC040000D1FFDF07F1040877
:10A2D00020461FFA88F108F011FE050000D1FFDFCB
:10A2E000204629466A4609F05CF80098A0F80370F9
:10A2F000A0F805A0284609F002F9017869F30601E3
:10A300006BF3C711017020461FFA88F108F039FE7F
:10A3100000B9FFDF019807F036F806EB0900017F6E
:10A32000491C017705B0BDE8F08F2DE9F84F0E46C6
:10A330009A4691460746032109F054FB0446008DD6
:10A34000DFF8B885002518B198F80000B0421ED19A
:10A35000384609F08AFC070000D1FFDF09F104014B
:10A36000384689B208F0CAFD050010D038462946A3
:10A370006A4609F016F8009800210A4601808170AB
:10A3800007F0BDF80098C01DCAF8000021E098F859
:10A390000000B04216D104F1260734F8341F012022
:10A3A00000FA06F911EA090F00D0FFDF2088012327
:10A3B00040EA090020800A22391D384609F0B4F924
:10A3C000067006E0324604F1340104F12600FFF77E
:10A3D0005CFF0A2188F800102846BDE8F88FFEB51A
:10A3E00015460C46064602AB0C220621FFF79DFFE0
:10A3F000002827D00299607812220A70801C4870C9
:10A4000008224A80A07002982988052381806988E3
:10A41000C180A9880181E988418100250C20CDE90E
:10A420000005062221463046FFF73FFF294600225D
:10A4300066F31F41F02310460CF0BAFF6078801CD1
:10A4400060700120FEBDFEB514460D46062206468C
:10A4500002AB1146FFF769FF002812D0029B1320C0
:10A4600000211870A8785870022058809C8006201F
:10A47000CDE900010246052329463046FFF715FFC6
:10A480000120FEBD2DE9FE430C46804644E002ABB0
:10A490000E2207214046FFF748FF002841D06068A0
:10A4A0001C2267788678BF1C06EB860102EBC1018F
:10A4B000451802981421017047700A214180698A69
:10A4C0000181E98A4181A9888180A98981813046F9
:10A4D00001F056FB029905230722C8806F70042003
:10A4E000287000250E20CDE9000521464046FFF7E3
:10A4F000DCFE294666F30F2168F31F41F02300229A
:10A5000006200CF055FF6078FD49801C6070626881
:10A510002046921CFFF793FE606880784028B6D1F1
:10A520000120BDE8FE83FEB50D46064638E002ABCD
:10A530000E2207213046FFF7F8FE002835D0686864
:10A540001C23C17801EB810203EBC202841802983C
:10A5500015220270627842700A224280A2894281EA
:10A56000A2888281084601F00BFB01460298818097
:10A57000618AC180E18A0181A088B8B10020207081
:10A5800000210E20CDE9000105230722294630468F
:10A59000FFF78BFE6A68DB492846D21CFFF74FFEA7
:10A5A0006868C0784028C2D10120FEBD0620E6E7D9
:10A5B0002DE9FE430C46814644E0204601F002FBB3
:10A5C000D0B302AB082207214846FFF7AEFE0028B1
:10A5D000A7D060681C2265780679AD1C06EB860161
:10A5E00002EBC10147180298B7F8108006210170EC
:10A5F000457004214180304601F0C2FA01460298BC
:10A6000005230722C180A0F804807D7008203870DF
:10A610000025CDE9000521464846FFF746FE2946BC
:10A6200066F30F2169F31F41F023002206200CF08E
:10A63000BFFE6078801C60706268B3492046121DBE
:10A64000FFF7FDFD606801794029B6D1012068E778
:10A650002DE9F34F83B00D4691E0284601F0B2FAA0
:10A6600000287DD068681C2290F806A00AEB8A01B9
:10A6700002EBC10144185146284601F097FAA1782F
:10A68000CB0069684978CA00014604F1240009F04A
:10A6900082F807468188E08B4FF00009091A8EB2D4
:10A6A00008B1C84607E04FF00108504601F053FAE0
:10A6B00008B9B61CB6B2208BB04200D80646B346E5
:10A6C00002AB324607210398FFF72FFE060007D0A2
:10A6D000B8F1000F0BD0504601F03DFA10B106E082
:10A6E00000201FE60299B8884FF002090880019601
:10A6F000E28B3968ABEB09001FFA80F80A44039833
:10A700004E46009209F0B1FADDE90021F61D4346FC
:10A71000009608F0C0FEE08B404480B2E083B98828
:10A72000884201D1012600E00026CDE900B6238A47
:10A73000072229460398FFF7B8FD504601F00BFAAF
:10A7400010B9E089401EE08156B1A078401CA0708D
:10A750006868E978427811FB02F1CAB2012300E08F
:10A7600007E081690E3008F0C4FF80F800A00020E7
:10A77000E0836A6865492846921DFFF760FD6868B6
:10A78000817940297FF469AF0120CBE570B5064699
:10A7900048680D4614468179402910D104EB8401A4
:10A7A0001C2202EBC101084401F043FA002806D044
:10A7B0006868294684713046BDE8704048E770BD3E
:10A7C000FEB50C460746002645E0204601F0FAF9A2
:10A7D000D8B360681C22417901EB810102EBC10111
:10A7E0004518688900B9FFDF02AB08220721384607
:10A7F000FFF79BFD002833D00299607816220A707B
:10A80000801C4870042048806068407901F0B8F9E5
:10A81000014602980523072281806989C1800820AA
:10A82000CDE9000621463846FFF73FFD6078801CE1
:10A830006070A88969890844B0F5803F00D3FFDFC4
:10A84000A88969890844A8816E81626830492046D8
:10A85000521DFFF7F4FC606841794029B5D1012011
:10A86000FEBD30B5438C458BC3F3C704002345B10F
:10A87000838B641EED1AC38A6D1E1D4495FBF3F392
:10A88000E4B22CB1008918B1A04200D8204603449C
:10A890004FF6FF70834200D3034613800C7030BD27
:10A8A0002DE9FC41074616460D46486802EB860135
:10A8B0001C2202EBC10144186A4601A92046FFF799
:10A8C000D0FFA089618901448AB2BDF8001091428D
:10A8D00012D0081A00D500206081686840794028AD
:10A8E0000AD1204601F09BF9002805D06868294666
:10A8F00046713846FFF764FFBDE8FC813000002058
:10A9000015A2000023A2000031A2000033BC000009
:10A910001FBC00002DE9FE4F0F46814615465088AA
:10A92000032109F05FF80190B9F8020001F01BF96A
:10A9300082460146019801F045F9002824D001988B
:10A940001C2241680AEB8A0002EBC0000C1820466A
:10A9500001F04EF9002817D1B9F80000E18A8842C9
:10A960000ED8A18961B1B8420ED100265146019896
:10A9700001F015F9218C01EB0008608B30B114E077
:10A98000504601F0E8F8A0B3BDE8FE8F504601F054
:10A99000E2F808B1678308E0022FF5D3B9F80400A4
:10A9A0006083618A884224D80226B81B87B2B8F82F
:10A9B0000400A28B801A002814DD874200DA384692
:10A9C0001FFA80FB688869680291D8F800100A4471
:10A9D000009209F038F9F61D009A5B46029900963C
:10A9E00008F025FDA08B384480B2A083618B88429B
:10A9F00007D96888019903B05246BDE8F04F01F0CD
:10AA000035B91FD14FF009002872B9F802006881EA
:10AA1000D8E90010C5E90410608BA881284601F030
:10AA200090F85146019801F0BAF8014601980823C0
:10AA300040680078C20004F1200008F090FE002079
:10AA4000A0836083504601F086F810B9A089401EAB
:10AA5000A0816888019903B00AF0FF02BDE8F04FB9
:10AA60001EE72DE9F041064615460F461C461846DE
:10AA7000F6F7EFFB18B92068F6F711FC10B11020BB
:10AA8000BDE8F0817168688C0978B0EBC10F01D323
:10AA90001320F5E73946304601F081F80146706829
:10AAA00008230078C20005F1200008F022FED4E956
:10AAB0000012C0E900120020E2E710B504460321AD
:10AAC00008F090FF0146007800F00300022805D04E
:10AAD0002046BDE8104001F1140280E48A8A204635
:10AAE000BDE81040AFE470B50446032108F07AFFDA
:10AAF000054601462046FFF75BFD002816D0294693
:10AB00002046FFF75DFE002810D029462046FFF7BB
:10AB10000AFD00280AD029462046FFF7B3FC00288A
:10AB200004D029462046BDE8704091E570BD2DE96E
:10AB3000F0410C4680461EE0E178427811FB02F1BC
:10AB4000CAB2816901230E3008F009FE07786068F7
:10AB50001C22C179491EC17107EB8701606802EBB5
:10AB6000C10146183946204601F02CF818B130468C
:10AB700001F037F820B16068C1790029DCD17FE7A6
:10AB8000FEF72AFD050000D1FFDF0A2028723846B3
:10AB900000F0F6FF68813946204601F007F80146CB
:10ABA000606808234078C20006F1240008F0D7FD51
:10ABB000D0E90010C5E90310A5F80280284600F08E
:10ABC000C0FFB07800B9FFDFB078401EB07057E723
:10ABD00070B50C460546032108F004FF01464068A5
:10ABE000C2792244C2712846BDE870409FE72DE932
:10ABF000FE4F8246507814460F464FF0000800285A
:10AC00004FD0012807D0022822D0FFDF2068B8608B
:10AC10006068F860B8E602AB0E2208215046FFF7E4
:10AC200084FB0028F2D002981521052301702178B9
:10AC300041700A214180C0F80480C0F80880A0F863
:10AC40000C80628882810E20CDE90008082221E074
:10AC5000A678304600F094FF054606EB86012C22CC
:10AC6000786802EBC1010822465A02AB11465046F1
:10AC7000FFF75BFB0028C9D00298072101702178FB
:10AC800041700421418008218580C680CDE90018EB
:10AC900005230A4639465046FFF707FB87F8088028
:10ACA00072E6A678022516B1022E13D0FFDF2A1D08
:10ACB000914602AB08215046FFF737FB0028A5D08C
:10ACC00002980121022E0170217841704580868012
:10ACD00002D005E00625EAE7A188C180E18801816C
:10ACE000CDE900980523082239465046D4E710B52F
:10ACF0000446032108F076FE014600F108022046D2
:10AD0000BDE8104073E72DE9F04F0F4605468DB0C2
:10AD100014465088032108F065FE4FF000088DF8B6
:10AD200014800646ADF81680042F7BD36A78002A7B
:10AD300078D028784FF6FF794FF01C0A132834D0CA
:10AD400008DC012871D006284AD007286ED01228C6
:10AD50000ED106E014286AD0152869D0162807D12C
:10AD6000AAE10C2F04D1307800F00301022907D0AA
:10AD7000CDF80880CDF80C8068788DF808004CE09C
:10AD800040F0080030706878B07001208DF8140031
:10AD9000A888ADF81800E888ADF81A002889ADF841
:10ADA0001C006889ADF81E0011E1B078904239D1DD
:10ADB0003078010736D5062F34D120F008003070E6
:10ADC0006088414660F31F4100200CF09BFB02208D
:10ADD0008DF81400ADF81890A888ADF81A00F6E0C8
:10ADE000082F1FD1A888EF88814600F0BCFE80465E
:10ADF0000146304600F0E6FE18B1404600F0ABFEDA
:10AE0000B8B1FC48D0E90010CDE902106878ADF87F
:10AE10000C908DF80800ADF80E70608802AA3146DB
:10AE2000FFF7E5FE0DB0BDE8F08FB6E01EE041E0B3
:10AE3000ECE0716808EB88002C2202EBC000085A95
:10AE4000B842EFD1EB4802AAD0E90210CDE90210D6
:10AE500068788DF8080008F0FF058DF80A506088C2
:10AE60003146FFF7C4FE224629461FE0082FD9D1FC
:10AE7000B5F80480E88800F076FE074601463046C3
:10AE800000F0A0FE0028CDD007EB870271680AEB26
:10AE9000C2000844028A4245C4D101780829C1D1C0
:10AEA000407869788842BDD1F9B222463046FFF732
:10AEB0001EF9B7E70E2F7FF45BAFE9886F898B46E9
:10AEC000B5F808903046FFF775F9ABF1400140291D
:10AED00001D309204AE0B9F1170F01D3172F01D28E
:10AEE0000B2043E040280ED000EB800271680AEB93
:10AEF000C20008440178012903D14078697888426A
:10AF000090D00A2032E03046FFF735F9014640285C
:10AF10002BD001EB810372680AEBC30002EB00083F
:10AF2000012288F800206A7888F801207068AA88D1
:10AF30004089B84200D93846AD8903232372A282E2
:10AF4000E7812082A4F80C906582084600F018FE84
:10AF50006081A8F81490A8F81870A8F80E50A8F806
:10AF600010B0204600F0EDFD5CE7042005212172C1
:10AF7000A4F80A80E081012121739E49D1E90421CE
:10AF8000CDE9022169788DF80810ADF80A006088D3
:10AF900002AA3146FFF72BFEE3E7062F89D3B078EC
:10AFA00090421AD13078010717D520F00800307090
:10AFB0006088414660F31F4100200CF0A3FA022094
:10AFC0008DF81400A888ADF81800ADF81A906088C4
:10AFD000224605A9F9F7EDF824E704213046FFF7EA
:10AFE00000F905464028BFD0022083030090224686
:10AFF0002946304600F003FE4146608865F30F2184
:10B0000060F31F4106200CF07DFA0BE70E2FABD149
:10B0100004213046FFF7E5F881464028A4D0414698
:10B02000608869F30F2160F31F4106200CF06AFA73
:10B03000A8890B906889099070682F894089B84267
:10B0400000D938468346B5F80680A8880A90484655
:10B0500000F096FD60810B9818B1022000900B9BC8
:10B0600024E0B8F1170F1ED3172F1CD30420207231
:10B0700009986082E781A4F810B0A4F80C8009EB6D
:10B08000890271680AEBC2000D18DDE90913A5F801
:10B090001480A5F818B0E9812B82204600F051FDFC
:10B0A00006202870BEE601200B2300902246494668
:10B0B000304600F0A4FDB5E6082F8DD1A9883046B2
:10B0C000FFF778F80746402886D000F044FD0028B6
:10B0D0009BD107EB870271680AEBC20008448046E7
:10B0E00000F086FD002890D1ED88B8F80E002844C5
:10B0F000B0F5803F05D360883A46314600F0B6FD92
:10B1000090E6002DCED0A8F80E0060883A46314671
:10B11000FFF73CFB08202072384600F031FD6081CB
:10B12000A5811EE72DE9F05F0C4601281FD0957917
:10B1300092F8048092F8056005EB85011F2202EB6E
:10B14000C10121F0030B08EB060111FB05F14FF6DD
:10B15000FF7202EAC10909F1030115FB0611264F2E
:10B1600021F0031ABB6840B101283ED125E0616897
:10B17000E57891F800804E78DEE75946184608F0E9
:10B180006CFA606000B9FFDF5A460021606803F086
:10B190003EF9E5705146B86808F05FFA61684861A9
:10B1A00000B9FFDF6068426902EB090181616068F4
:10B1B00080F800806068467017E060685246416918
:10B1C000184608F075FA5A466168B86808F070FACF
:10B1D000032008F0AFFB0446032008F0B3FB201A5D
:10B1E000012802D1B86808F02DFA0BEB0A00BDE87F
:10B1F000F09F000048540200300000200246002169
:10B2000002208FE7F7B5FF4C0A2016462070009801
:10B2100060B100254FEA0D0008F001FA0021A1708D
:10B220006670002D01D10099A160FEBD01250020AE
:10B23000F2E770B50C46154638220021204603F08F
:10B24000E6F8012666700A22002104F11C0003F0D2
:10B25000DEF805B9FFDF297A207861F3010020705C
:10B26000A87900282DD02A4621460020FFF75AFF52
:10B2700061684020E34A88706168C870616808713D
:10B2800061684871616888716168288808816168AF
:10B2900068884881606886819078002811D061684C
:10B2A0000620087761682888C885616828884886EC
:10B2B000606806856068698892880186818646850F
:10B2C000828570BDC878002802D00022012029E7BD
:10B2D000704770B50546002165F31F4100200CF052
:10B2E00011F90321284608F07DFB040000D1FFDF9F
:10B2F00021462846FEF71CFF002804D0207840F0A5
:10B3000010002070012070BD70B505460C4603206A
:10B3100008F002FB08B1002070BDBA488570848037
:10B32000012070BD2DE9FF4180460E460F0CFEF74F
:10B3300053F9050007D06F800321384608F052FB0F
:10B34000040008D106E004B03846BDE8F0411321FE
:10B35000F9F75ABBFFDF5FEA080005D0B8F1060F26
:10B3600018D0FFDFBDE8FF8120782A4620F00800D2
:10B3700020700020ADF8020002208DF800004FF68A
:10B38000FF70ADF80400ADF8060069463846F8F7DE
:10B3900010FFE7E7C6F3072101EB81021C23606879
:10B3A00003EBC202805C042803D008280AD0FFDF28
:10B3B000D8E7012000904FF440432A46204600F091
:10B3C0001EFCCFE704B02A462046BDE8F041FEF758
:10B3D0008EBE2DE9F05F05464089002790460C4659
:10B3E0003E46824600F0BFFB8146287AC01E0828F0
:10B3F0006BD2DFE800F00D04192058363C47722765
:10B400001026002C6CD0D5E90301C4E902015CE0F0
:10B4100070271226002C63D00A2205F10C0104F1DA
:10B42000080002F0CAFF50E071270C26002C57D00C
:10B43000E868A06049E0742710269CB3D5E90301B1
:10B44000C4E902016888032108F0CCFA8346FEF7BC
:10B45000C3F802466888508049465846FEF7FEFD0C
:10B4600033E075270A26ECB1A88920812DE07627E4
:10B470001426BCB105F10C0004F1080307C883E8E9
:10B48000070022E07727102664B1D5E90301C4E95B
:10B4900002016888032108F0A5FA01466888FFF7D1
:10B4A00046FB12E01CE073270826CCB16888032114
:10B4B00008F098FA01460078C00606D56888FEF7BD
:10B4C00037FE10B96888F8F781FAA8F800602CB147
:10B4D0002780A4F806A066806888A080002086E601
:10B4E000A8F80060FAE72DE9FC410C461E46174615
:10B4F0008046032108F076FA05460A2C0AD2DFE8D6
:10B5000004F005050505050509090907042303E0FD
:10B51000062301E0FFDF0023CDE90076224629461D
:10B520004046FEF7C2FEBDE8FC81F8B50546A0F531
:10B530007F40FF382BD0284608F085FB040000D15F
:10B54000FFDF204607F00BFF002821D001466A46A6
:10B55000204607F026FF00980321B0F80560284632
:10B5600008F040FA0446052E13D0304600F0FBFAEE
:10B5700005460146204600F025FB40B1606805EB1A
:10B5800085013E2202EBC101405A002800D0012073
:10B59000F8BD007A0028FAD00020F8BDF8B50446BE
:10B5A000408808F050FB050000D1FFDF6A462846BE
:10B5B000616800F0C4FA01460098091F8BB230F8A8
:10B5C000032F0280428842800188994205D1042AD3
:10B5D00008D0052A20D0062A16D022461946FFF7A1
:10B5E00099F9F8BD001D0E46054601462246304633
:10B5F000F6F749FF0828F4D1224629463046FCF7E1
:10B600006AF9F8BD30000020636864880A46011DAD
:10B610002046FAF78FF9F4E72246001DFFF773FB87
:10B62000EFE770B50D460646032108F0DBF904008C
:10B6300004D02078000704D5112070BD43F2020029
:10B6400070BD2A4621463046FEF7C9FE18B9286863
:10B6500060616868A061207840F0080020700020D8
:10B6600070BD70B50D460646032108F0BBF9040015
:10B6700004D02078000704D4082070BD43F20200F3
:10B6800070BD2A4621463046FEF7DDFE00B9A58290
:10B69000207820F008002070002070BD2DE9F04FC8
:10B6A0000E4691B08046032108F09CF904464046BE
:10B6B00008F0DBFA07460020079008900990ADF8E3
:10B6C00030000A9002900390049004B9FFDF0DF15E
:10B6D0000809FFB9FFDF1DE038460BA9002207F07B
:10B6E00001FD9DF82C0000F07F050A2D00D3FFDF3F
:10B6F0006019017F491E01779DF82C00000609D5CD
:10B700002A460CA907A8FEF7C0FD19F80510491C28
:10B7100009F80510761EF6B2DED204F13400F84DB9
:10B7200004F1260BDFF8DCA304F12A07069010E0F1
:10B730005846069900F08CFA064628700A2800D36D
:10B74000FFDF5AF8261040468847E08CC05DB042C3
:10B7500002D0208D0028EBD10A202870E94D4E46FA
:10B7600028350EE00CA907A800F072FA0446375DF0
:10B7700055F8240000B9FFDF55F82420394640462B
:10B780009047BDF81E000028ECD111B0BDE8F08F45
:10B7900010B5032108F026F9040000D1FFDF0A22CA
:10B7A000002104F11C0002F032FE207840F0040079
:10B7B000207010BD10B50C46032108F013F9204489
:10B7C000007F002800D0012010BD2DE9F84F8946E8
:10B7D00015468246032108F005F9070004D02846E3
:10B7E000F5F737FD40B903E043F20200BDE8F88FFA
:10B7F0004846F5F754FD08B11020F7E7786828B1FE
:10B8000069880089814201D90920EFE7B9F8000071
:10B810001C2488B100F0A7F980460146384600F0A4
:10B82000D1F988B108EB8800796804EBC000085CA6
:10B8300001280BD00820D9E73846FEF79CFC80464B
:10B84000402807D11320D1E70520CFE7FDF7C4FE3C
:10B8500006000BD008EB8800796804EBC0000C18D8
:10B86000B9F8000020B1E88910B113E01120BDE75C
:10B870002888172802D36888172801D20720B5E73F
:10B88000686838B12B1D224641463846FFF7E9F873
:10B890000028ABD104F10C0269462046FEF7E1FF17
:10B8A000288860826888E082B9F8000030B1022000
:10B8B0002070E889A080E889A0B12BE003202070E7
:10B8C000A889A08078688178402905D180F8028015
:10B8D00039465046FEF7D6FD404600F051F9A9F82A
:10B8E000000021E07868218B4089884200D9084611
:10B8F0002083A6F802A004203072B9F800007081FD
:10B90000E0897082F181208B3082A08AB08130463C
:10B9100000F017F97868C178402905D180F80380D4
:10B9200039465046FEF7FFFD00205FE770B50D4633
:10B930000646032108F056F804000ED0284600F011
:10B9400012F905460146204600F03CF918B1284698
:10B9500000F001F920B1052070BD43F2020070BD76
:10B9600005EB85011C22606802EBC101084400F070
:10B970003FF908B1082070BD2A462146304600F044
:10B9800075F9002070BD2DE9F0410C461746804640
:10B99000032108F027F80546204600F0E4F80446A5
:10B9A00095B10146284600F00DF980B104EB840101
:10B9B0001C22686802EBC1014618304600F018F9F5
:10B9C00038B10820BDE8F08143F20200FAE7052013
:10B9D000F8E73B46324621462846FFF742F8002862
:10B9E000F0D1E2B229464046FEF75AFF708C083883
:10B9F000082803D242484078F7F786FA0020E1E7AA
:10BA00002DE9F0410D4617468046032107F0EAFF75
:10BA10000446284600F0A7F8064624B13846F5F754
:10BA200018FC38B902E043F20200CBE73868F5F7BA
:10BA300010FC08B11020C5E73146204600F0C2F8DE
:10BA400060B106EB86011C22606802EBC10145185B
:10BA5000284600F0CDF818B10820B3E70520B1E77B
:10BA6000B888A98A884201D90C20ABE76168E88CC4
:10BA70004978B0EBC10F01D31320A3E7314620462C
:10BA800000F094F80146606808234078C20005F190
:10BA9000240007F02EFED7E90012C0E90012F2B22E
:10BAA00021464046FEF772FE00208BE72DE9F04765
:10BAB0000D461F4690468146032107F093FF04463A
:10BAC000284600F050F806463CB14DB13846F5F72F
:10BAD00004FC50B11020BDE8F08743F20200FAE701
:10BAE000606858B1A0F80C8027E03146204600F08D
:10BAF00069F818B1304600F02EF828B10520EAE7C1
:10BB0000300000206054020006EB86011C226068B1
:10BB100002EBC1014518284600F06AF808B1082078
:10BB2000D9E7A5F80880F2B221464846FEF7B8FEEC
:10BB30001FB1A8896989084438800020CBE707F045
:10BB400030BC017821F00F01491C21F0F0011031C7
:10BB50000170FDF744BD20B94E48807808B101203E
:10BB60007047002070474B498988884201D10020E6
:10BB70007047402801D2402000E0403880B2704732
:10BB800010B50446402800D9FFDF2046FFF7E3FF49
:10BB900010B14048808810BD4034A0B210BD40684C
:10BBA00042690078484302EBC0007047C2784068A1
:10BBB000037812FB03F24378406901FB032100EB99
:10BBC000C1007047C2788A4209D9406801EB8101FF
:10BBD0001C2202EBC101405C08B10120704700202B
:10BBE00070470078062801D901207047002070476F
:10BBF0000078062801D00120704700207047F0B47B
:10BC000001EB81061C27446807EBC6063444049DFB
:10BC100005262670E3802571F0BCFEF71FBA10B52B
:10BC2000418911B1FFF7DDFF08B1002010BD0120EF
:10BC300010BD10B5C18C8278B1EBC20F04D9C18997
:10BC400011B1FFF7CEFF08B1002010BD012010BDDB
:10BC500010B50C4601230A22011D07F080FD007873
:10BC60002188012282409143218010BDF0B402EB73
:10BC700082051C264C6806EBC505072363554B68F7
:10BC80001C79402C03D11A71F0BCFEF791BCF0BCBA
:10BC9000704700003000002010B5EFF3108000F076
:10BCA000010472B6F8484178491C41704078012877
:10BCB00001D10BF05FF8002C00D162B610BD70B559
:10BCC000F14CA07848B90125A570FFF7E5FF0BF00E
:10BCD00062F820B100200BF02CF8002070BD4FF06E
:10BCE0008040E570C0F80453F7E770B5EFF31080BB
:10BCF00000F0010572B6E44C607800B9FFDF6078AF
:10BD0000401E6070607808B90BF038F8002D00D143
:10BD100062B670BDDC4810B5817821B10021C170D8
:10BD20008170FFF7E2FF002010BD10B504460BF054
:10BD300032F8D5498978084000D0012020600020E1
:10BD400010BD10B5FFF7A8FF0BF025F80222012364
:10BD5000CD49540728B1CD48026023610320087201
:10BD600002E00A72C4F804330020887110BD2DE986
:10BD7000F84FDFF814934278817889F80420002680
:10BD800089F80510074689F806600078DFF800B3E7
:10BD9000354620B1012811D0022811D0FFDF0BF069
:10BDA0000CF84FF0804498B10BF00EF8B0420FD170
:10BDB00030460BF00DF80028FAD042E00126EEE7FD
:10BDC000FFF76AFF58460168C907FCD00226E6E77C
:10BDD0000120E060C4F80451AE490E600107D1F8BB
:10BDE0004412AC4AC1F3423124321160A9493431C2
:10BDF00008604FF0020AC4F804A3A060A6480168D6
:10BE0000C94341F3001101F10108016841F010013B
:10BE1000016001E019F02CF9D4F804010028F9D0F0
:10BE200030460AF0D5FF0028FAD0B8F1000F04D14F
:10BE30009948016821F010010160C4F808A3C4F812
:10BE4000045199F805004E4680B1387870B90AF06F
:10BE5000A2FF80460BF03AF96FF00042B8F1000FF4
:10BE600002D0C6E9032001E0C6E90302DBF80000C6
:10BE7000C00701D00AF08BFF387810B13572BDE8E9
:10BE8000F88F4FF01808C4F808830127A7614FF412
:10BE90002070ADF8000000BFBDF80000411EADF8F5
:10BEA0000010F9D2C4F80C51C4F810517648C01DE6
:10BEB0000AF0A0FF3570FFF744FF676175493079DC
:10BEC00020310860C4F80483D9E770B5050000D1BB
:10BED000FFDF4FF080424FF0FF30C2F8080300212F
:10BEE000C2F80011C2F80411C2F80C11C2F8101106
:10BEF000654C61700AF05BFF10B10120A0706070AA
:10BF000063480068C00701D00AF041FF2846BDE839
:10BF100070402CE75C48007A002800D00120704770
:10BF20002DE9FC5F5D48D0F800905C4A5C4908321E
:10BF300011608406D4F8080100B10120D4F8001182
:10BF400011B14FF0010801E04FF00008D4F80411DE
:10BF500001B101210191D4F80C1101B1012100912D
:10BF6000D4F8101101B10121474D8A4695F800B06F
:10BF7000002620B1C4F8086101200AF0DAFE424828
:10BF8000C01D0AF03FFF00B1FFDF0127B8F1000F2D
:10BF900010D0C4F80873E87818B1EE7000200AF0E9
:10BFA000C8FE287A022805D10320287237480221CA
:10BFB00001602761019808B1C4F80461009850B18C
:10BFC000C4F80C61287A032800D0FFDF2F480660F0
:10BFD0002F72FFF78AFEBAF1000F07D0C4F8106184
:10BFE000287A012801D100F05DF86761BBF1000FEC
:10BFF00007D02E70287A012801D1FFF7A2FEFFF7A3
:10C0000074FE2148C01D0AF013FF2449091DC1F820
:10C010000090BDE8FC9F1C4810B5C01D0AF0F2FE60
:10C02000194940B1012008704FF0E021C1F8000229
:10C03000BDE8104030E6087A012801D1FFF781FE03
:10C040001148BDE81040C01D0AF0F2BE70B50E4C9C
:10C05000A07808B90AF092FE01208507A861207A2D
:10C06000002603280AD100BFD5F80C0120B9002012
:10C070000AF0AEFE0028F7D1C5F80C6126724FF029
:10C08000FF30C5F8080370BD44000020340C0040A8
:10C090000C0400401805004010ED00E010050240BF
:10C0A0000100000170B5134C6079F0B1012803D094
:10C0B000A179401E814218DA0AF06DFE05460BF0A8
:10C0C00005F86179012902D9A179491CA1710DB145
:10C0D000216900E0E168411A022902DA11F1020F38
:10C0E000D1DC0DB1206100E0E060BDE8704028E6E1
:10C0F000C9E70000440000200F4A12680D498A4237
:10C100000CD118470C4A12680A4B9A4206D101B565
:10C110000AF0AEFF0BF081FABDE80140074909685B
:10C120000958084706480749054A064B704700006A
:10C1300000000000BEBAFECA5C000020040000201F
:10C14000C0130020C0130020F8B51D46DDE90647E6
:10C150000E000AD007F089FD2346FF1DBCB2314610
:10C160002A46009407F097F9F8BDD01922461946DF
:10C1700002F023F92046F8BD70B50D4604461022A2
:10C18000002102F044F9258117206081A07B40F056
:10C190000A00A07370BD4FF6FF720A8001460220AC
:10C1A0000BF0B0B9704700897047827BD30701D18B
:10C1B000920703D4808908800020704705207047CB
:10C1C000827B920700D58181704701460020098853
:10C1D00041F6FE52114200D00120704700B50346DF
:10C1E000807BC00701D0052000BD59811846FFF7AC
:10C1F000ECFFC00703D0987B40F004009873987B55
:10C2000040F001009873002000BD827B520700D5EA
:10C2100009B14089704717207047827B61F3C302E0
:10C22000827370472DE9FC5F0E46044601789646FE
:10C23000012000FA01F14DF6FF5201EA020962689D
:10C240004FF6FF7B1188594502D10920BDE8FC9FBC
:10C25000B9F1000F05D041F6FE55294201D0012069
:10C26000F4E741EA090111801D0014D000232B706E
:10C2700094F800C0052103221F464FF0020ABCF1CA
:10C280000E0F76D2DFE80CF0F909252F47646B77A3
:10C29000479193B4D1D80420D8E7616820898B7B7B
:10C2A0009B0767D517284AD30B89834247D38989CF
:10C2B000172901D3814242D185F800A0A5F80100D9
:10C2C0003280616888816068817B21F0020181731E
:10C2D000C6E0042028702089A5F801006089A5F82F
:10C2E00003003180BCE0208A3188C01D1FFA80F82D
:10C2F000414524D3062028702089A5F801006089D3
:10C30000A5F80300A089A5F805000721208ACDE93A
:10C310000001636941E00CF0FF00082810D00820FC
:10C3200028702089A5F801006089A5F803003180F4
:10C330006A1D694604F10C0009F001F910B15EE0D4
:10C340001020EDE730889DF800100844308087E029
:10C350000A2028702089A5F80100328044E00C20D2
:10C3600028702089A5F801006089A5F803003180B4
:10C370003AE082E064E02189338800EB41021FFA51
:10C3800082F843453BD3B8F1050F38D30E222A700B
:10C390000BEA4101CDE90010E36860882A46714646
:10C3A000FFF7D2FEA6F800805AE04020287060898E
:10C3B0003188C01C1FFA80F8414520D32878714687
:10C3C00020F03F00123028702089A5F80100608914
:10C3D000CDE9000260882A46E368FFF7B5FEA6F8BB
:10C3E0000080287840063BD461682089888037E047
:10C3F000A0893288401D1FFA80F8424501D20427E7
:10C400003DE0162028702089A5F801006089A5F874
:10C410000300A089CDE9000160882A46714623699E
:10C42000FFF792FEA6F80080DEE718202870207A39
:10C430006870A6F800A013E061680A88920401D42D
:10C4400005271CE0C9882289914201D0062716E001
:10C450001E21297030806068018821F4005101801C
:10C46000B9F1000F0BD061887823002202200AF076
:10C470009FFF61682078887006E03380032760683A
:10C48000018821EA090101803846DFE62DE9FF4FE6
:10C4900085B01746129C0D001E461CD03078C1078F
:10C4A00003D000F03F00192801D9012100E000214C
:10C4B0002046FFF7AAFEA8420DD32088A0F57F41B1
:10C4C000FF3908D03078410601D4000605D5082090
:10C4D00009B0BDE8F08F0720FAE700208DF80000D2
:10C4E0008DF8010030786B1E00F03F0C0121A81E72
:10C4F0004FF0050A4FF002094FF0030B9AB2BCF15E
:10C50000200F75D2DFE80CF08B10745E7468748CA9
:10C51000749C74B574BA74C874D474E1747474F18E
:10C5200074EF74EE74ED748B052D78D18DF8009056
:10C53000A0788DF804007088ADF8060030798DF889
:10C540000100707800F03F000C2829D00ADCA0F12F
:10C550000200092863D2DFE800F0126215621A6255
:10C560001D622000122824D004DC0E281BD01028C5
:10C57000DBD11BE016281FD01828D6D11FE0207869
:10C58000800701E020784007002848DAEEE02078B4
:10C590000007F9E72078C006F6E720788006F3E781
:10C5A00020784006F0E720780006EDE72088C005F7
:10C5B000EAE720884005E7E720880005E4E72088CF
:10C5C000C004E1E72078800729D5032D27D18DF815
:10C5D00000B0B6F8010081E0217849071FD5062D8B
:10C5E0001DD381B27078012803D0022817D102E050
:10C5F000C9E0022000E0102004228DF800207278AB
:10C600008DF80420801CB1FBF0F2ADF8062092B248
:10C6100042438A4203D10397ADF80890A6E079E03F
:10C620002078000776D598B282088DF800A0ADF882
:10C630000420B0EB820F6DD10297ADF8061095E0A3
:10C640002178C90666D5022D64D381B206208DF803
:10C650000000707802285DD3B1FBF0F28DF8040081
:10C66000ADF8062092B242438A4253D1ADF8089009
:10C670007BE0207880064DD5072003E02078400637
:10C680007FD508208DF80000A088ADF80400ADF833
:10C690000620ADF8081068E02078000671D5092062
:10C6A000ADF804208DF80000ADF8061002975DE0AB
:10C6B0002188C90565D5022D63D381B20A208DF882
:10C6C0000000707804285CD3C6E72088400558D560
:10C6D000012D56D10B208DF80000A088ADF8040084
:10C6E00044E021E026E016E0FFE72088000548D579
:10C6F000052D46D30C208DF80000A088ADF804006D
:10C70000B6F803006D1FADF80850ADF80600ADF89F
:10C710000AA02AE035E02088C00432D5012D30D1AE
:10C720000D208DF8000021E02088800429D4B6F87F
:10C730000100E080A07B000723D5032D21D33078B2
:10C7400000F03F001B2818D00F208DF80000208833
:10C7500040F40050A4F80000B6F80100ADF8040061
:10C76000ED1EADF80650ADF808B003976946059880
:10C77000F5F7D2FB050008D016E00E208DF800007A
:10C78000EAE7072510E008250EE0307800F03F00CA
:10C790001B2809D01D2807D0022005990AF0B2FEF7
:10C7A000208800F400502080A07B400708D5204658
:10C7B000FFF70BFDC00703D1A07B20F00400A0739E
:10C7C000284685E61FB5022806D101208DF8000015
:10C7D00088B26946F5F7A0FB1FBD0000F8B51D46FD
:10C7E000DDE906470E000AD007F03FFA2346FF1D99
:10C7F000BCB231462A46009406F04DFEF8BDD01971
:10C800002246194601F0D9FD2046F8BD2DE9FF4F1B
:10C810008DB09B46DDE91B57DDF87CA00C46082B4C
:10C8200005D0E06901F0FEF850B11020D2E0288870
:10C83000092140F0100028808AF80010022617E035
:10C84000E16901208871E2694FF420519180E1692A
:10C850008872E06942F601010181E069002181737B
:10C860002888112140F0200028808AF80010042632
:10C8700038780A900A2038704FF0020904F1180045
:10C880004D460C9001F0C6FBB04681E0BBF1100FA5
:10C890000ED1022D0CD0A9EB0800801C80B2022121
:10C8A000CDE9001005AB52461E990D98FFF796FF93
:10C8B000BDF816101A98814203D9F74800790F90F5
:10C8C00004E003D10A9808B138702FE04FF002015C
:10C8D000CDE900190DF1160352461E990D98FFF788
:10C8E0007DFF1D980088401B801B83B2C6F1FF00AE
:10C8F000984200D203461E990BA8D9B15FF00002FE
:10C90000DDF878C0CDE9032009EB060189B2CDE955
:10C9100001C10F980090BDF8161000220D9801F08B
:10C920000EFC387070B1C0B2832807D0BDF8160075
:10C9300020833AE00AEB09018A19E1E7022011B0ED
:10C94000BDE8F08FBDF82C00811901F0FF08022D21
:10C950000DD09AF80120424506D1BDF82010814241
:10C9600007D0B8F1FF0F04D09AF801801FE08AF8D1
:10C970000180C94800680178052902D1BDF8161068
:10C98000818009EB08001FFA80F905EB080085B2E9
:10C99000DDE90C1005AB0F9A01F03FFB28B91D989B
:10C9A0000088411B4145BFF671AF022D13D0BBF18A
:10C9B000100F0CD1A9EB0800801C81B20220CDE938
:10C9C000000105AB52461E990D98FFF707FF1D9811
:10C9D0000580002038700020B1E72DE9F8439C461F
:10C9E000089E13460027B26B9AB3491F8CB2F18F91
:10C9F000A1F57F45FF3D05D05518AD882944891D17
:10CA00008DB200E000252919B6F83C800831414577
:10CA100020D82A44BCF8011022F8021BBCF80310ED
:10CA200022F8021B984622F8024B914607F00BF9B8
:10CA30004FF00C0C41464A462346CDF800C006F0A4
:10CA4000F6FCF587B16B00202944A41D2144088021
:10CA500003E001E0092700E083273846BDE8F883BA
:10CA600010B50B88848F9C420CD9846BE018048825
:10CA700044B1848824F40044A41D23440B80106036
:10CA8000002010BD0A2010BD2DE9F0478AB0002516
:10CA9000904689468246ADF8185007274BE0059826
:10CAA00006888088000446D4A8F8006007A801958D
:10CAB00000970295CDE903504FF4007300223146F0
:10CAC000504601F03CFB04003CD1BDF81800ADF825
:10CAD0002000059804888188B44216D10A0414D431
:10CAE00001950295039521F400410097049541F4C6
:10CAF000804342882146504601F0BFF804000BD124
:10CB00000598818841F40041818005AA08A948461A
:10CB1000FFF7A6FF0400DCD0009705980295019569
:10CB2000039504950188BDF81C300022504601F0A1
:10CB3000A4F80A2C06D105AA06A94846FFF790FFDB
:10CB40000400ACD0ADF8185004E00598818821F4B9
:10CB50000041818005AA06A94846FFF781FF002809
:10CB6000F3D00A2C03D020460AB0BDE8F08700209D
:10CB7000FAE710B50C46896B86B051B10C218DF8DF
:10CB80000010A18FADF80810A16B01916946FAF76A
:10CB900037FB00204FF6FF71A063E187A08706B046
:10CBA00010BD2DE9F0410D460746896B0020069E19
:10CBB0001446002911D0012B0FD1324629463846A0
:10CBC000FFF762FF002808D1002C06D03246294624
:10CBD0003846BDE8F04100F034BFBDE8F0812DE9F2
:10CBE000FC411446DDE9087C0E46DDE90A15521DBC
:10CBF000BCF800E092B2964502D20720BDE8FC8165
:10CC0000ACF8002017222A70A5F80160A5F80330BF
:10CC10000522CDE900423B462A46FFF7DFFD002012
:10CC2000ECE770B50C46154648220021204601F07D
:10CC3000EEFB04F1080044F81C0F00204FF6FF71D2
:10CC4000E06161842084A5841720E08494F82A00A0
:10CC500040F00A0084F82A0070BD4FF6FF720A8087
:10CC6000014603200AF04EBC30B585B00C4605469F
:10CC7000FFF77FFFA18E284629B101218DF8001012
:10CC80006946FAF7BDFA0020E0622063606305B0F0
:10CC900030BDB0F8400070476000002090F846209A
:10CCA000920703D4408808800020F4E70620F2E7CA
:10CCB00090F846209207EED5A0F84410EBE7014625
:10CCC000002009880A0700D5012011F0F00F01D0DB
:10CCD00040F00200CA0501D540F004008A0501D5E4
:10CCE00040F008004A0501D540F010000905D2D5F2
:10CCF00040F02000CFE700B5034690F84600C0079B
:10CD000001D0062000BDA3F842101846FFF7D7FF58
:10CD100010F03E0F05D093F8460040F0040083F871
:10CD2000460013F8460F40F001001870002000BDC7
:10CD300090F84620520700D511B1B0F84200AAE79A
:10CD40001720A8E710F8462F61F3C3020270A2E78C
:10CD50002DE9FF4F9BB00E00DDE92B34DDE929788A
:10CD6000289D24D02878C10703D000F03F0019285F
:10CD700001D9012100E000212046FFF7D9FFB04290
:10CD800015D32878410600F03F010CD41E290CD0A1
:10CD9000218811F47F6F0AD13A8842B1A1F57F4210
:10CDA000FF3A04D001E0122901D1000602D5042087
:10CDB0001FB0C5E5FA491D984FF0000A08718DF8BB
:10CDC00018A08DF83CA00FAA0A60ADF81CA0ADF821
:10CDD00050A02978994601F03F02701F5B1C04F1B6
:10CDE000180C4FF0060E4FF0040BCDF858C01F2A58
:10CDF0007ED2DFE802F07D7D107D267DAC7DF47D66
:10CE0000F37DF27DF17DF47DF07D7D7DEF7DEE7D26
:10CE10007D7D7D7DED0094F84610B5F80100890711
:10CE200001D5032E02D08DF818B01EE34FF4006137
:10CE3000ADF85010608003218DF83C10ADF8400033
:10CE4000D4E2052EEFD1B5F801002083ADF81C0027
:10CE5000B5F80310618308B1884201D9012079E156
:10CE60000020A07220814FF6FF702084169801F0F8
:10CE7000D1F8052089F800000220029083460AAB11
:10CE80001D9A16991B9801F0C8F890BB9DF82E00CA
:10CE9000012804D0022089F80100102003E00120BD
:10CEA00089F8010002200590002203A90BA808F0D0
:10CEB00046FBE8BB9DF80C00059981423DD13988BD
:10CEC000801CA1EB0B01814237DB02990220CDE9E6
:10CED00000010DF12A034A4641461B98FFF77EFCEC
:10CEE00002980BF1020B801C81B217AA029101E09B
:10CEF0009CE228E003A90BA808F021FB02999DF809
:10CF00000C00CDE9000117AB4A4641461B98FFF7DC
:10CF100065FC9DF80C000AAB0BEB00011FFA81FBCE
:10CF200002991D9A084480B2029016991B9800E05D
:10CF300003E001F072F80028B6D0BBF1020F02D076
:10CF4000A7F800B04FE20A208DF818004BE200214C
:10CF50000391072EFFF467AFB5F801002083ADF809
:10CF60001C00B5F80320628300283FF477AF90429D
:10CF70003FF674AF0120A072B5F8050020810020B3
:10CF8000A073E06900F04EFD78B9E1690120887175
:10CF9000E2694FF420519180E1698872E16942F6BB
:10CFA00001000881E06900218173F01F20841E9830
:10CFB000606207206084169801F02CF8072089F839
:10CFC00000000120049002900020ADF82A0028E023
:10CFD00019E29FE135E1E5E012E2A8E080E043E0FC
:10CFE0000298012814D0E0698079012803D1BDF8A6
:10CFF0002800ADF80E00049803ABCDE900B04A4616
:10D0000041461B98FFF7EAFB0498001D80B204908C
:10D01000BDF82A00ADF80C00ADF80E00059880B2FE
:10D0200002900AAB1D9A16991B9800F0F6FF28B9DA
:10D0300002983988001D05908142D1D202980128BA
:10D0400081D0E0698079012803D1BDF82800ADF8CE
:10D050000E00049803ABCDE900B04A4641461B9848
:10D06000FFF7BCFB0298BDE1072E02D0152E7FF41E
:10D07000DAAEB5F801102183ADF81C10B5F8032025
:10D08000628300293FF4EAAE91423FF6E7AE012108
:10D09000A1724FF0000BA4F808B084F80EB0052E72
:10D0A00007D0C0B2691DE26908F047FA00287FF492
:10D0B0004AAF4FF6FF70208401A906AA14A8CDF844
:10D0C00000B081E885032878214600F03F031D9ACF
:10D0D0001B98FFF79BFB8246208BADF81C0082E17A
:10D0E0000120032EC3D14021ADF85010B5F8011036
:10D0F0002183ADF81C100AAAB8F1000F00D000235C
:10D10000CDE9020304921D98CDF804800090388880
:10D110000022401E83B21B9801F011F88DF8180010
:10D1200090BB0B2089F80000BDF8280035E04FF0D7
:10D13000010C052E9BD18020ADF85000B5F80110F0
:10D140002183B5F803002084ADF81C10B0F5007FF2
:10D1500003D907208DF8180087E140F47C4222842F
:10D160000CA8B8F1000F00D00023CDE90330CDE9C1
:10D17000018C1D9800903888401E83B21B9800F0E7
:10D18000DEFF8DF8180018B18328A8D10220BFE077
:10D190000D2189F80010BDF83000401C22E100008C
:10D1A00060000020032E04D248067FF53CAE00202C
:10D1B00018E1B5F80110ADF81C102878400602D52A
:10D1C0008DF83CE002E007208DF83C004FF00008AD
:10D1D0000320CDE902081E9BCDF810801D98019315
:10D1E000A6F1030B00901FFA8BF342461B9800F048
:10D1F00044FD8DF818008DF83C80297849060DD53E
:10D200002088C00506D5208BBDF81C10884201D1AE
:10D21000C4F8248040468DF81880E3E0832801D1CB
:10D220004FF0020A4FF48070ADF85000BDF81C00BA
:10D230002083A4F820B01E9860620320608413212C
:10D24000CDE0052EFFF4EFADB5F80110ADF81C10E0
:10D25000A28F6AB3A2F57F43FE3B29D008228DF846
:10D260003C2000BF4FF0000B0523CDE9023BDDF869
:10D2700078C0CDF810B01D9A80B2CDF804C040F44B
:10D2800000430092B5F803201B9800F0F6FC8DF8DF
:10D290003CB04FF400718DF81800ADF850108328A1
:10D2A00010D0F8B1A18FA1F57F40FE3807D0DCE0A7
:10D2B0000B228DF83C204FF6FE72A287D2E7A4F82D
:10D2C0003CB0D2E000942B4631461E9A1B98FFF7E3
:10D2D00084FB8DF8180008B183284BD1BDF81C00E1
:10D2E000208353E700942B4631461E9A1B98FFF784
:10D2F00074FB8DF81800E8BBE18FA06B0844831D18
:10D300008DE888034388828801881B98FFF767FCB3
:10D31000824668E095F80180022E70D15FEA08002D
:10D3200002D0B8F1010F6AD109208DF83C0007A89E
:10D3300000908DF840804346002221461B98FFF75D
:10D3400030FC8DF842004FF0000B8DF843B050B91F
:10D35000B8F1010F12D0B8F1000F04D1A18FA1F5DF
:10D360007F40FF380AD0A08F40B18DF83CB04FF419
:10D37000806000E037E0ADF850000DE00FA91B9889
:10D38000F9F73EFF82468DF83CB04FF48060ADF86F
:10D390005000BAF1020F06D0FC480068C07928B1ED
:10D3A0008DF8180027E0A4F8188044E0BAF1000FC7
:10D3B00003D081208DF818003DE007A80090434677
:10D3C000012221461B98FFF7ECFB8DF8180021463F
:10D3D0001B98FFF7CEFB9DF8180020B9192189F89A
:10D3E0000010012038809DF83C0020B10FA91B9847
:10D3F000F9F706FF8246BAF1000F33D01BE018E0C0
:10D400008DF818E031E02078000712D5012E10D1F8
:10D410000A208DF83C00E088ADF8400003201B99FD
:10D420000AF070F80820ADF85000C0E648067FF515
:10D43000FAAC4FF0040A2088BDF850100843208051
:10D44000BDF8500080050BD5A18FA1F57F40FE38B7
:10D4500006D11E98E06228982063A6864FF0030A42
:10D460005046A5E49DF8180078B1012089F8000025
:10D47000297889F80110BDF81C10A9F802109DF850
:10D48000181089F80410052038802088BDF8501045
:10D4900088432080E4E72DE9FF4F8846087895B05F
:10D4A000012181404FF20900249C0140ADF8201079
:10D4B0002088DDF88890A0F57F424FF0000AFF3AFF
:10D4C00006D039B1000705D5012019B0BDE8F08FAD
:10D4D0000820FAE7239E4FF0000B0EA886F800B054
:10D4E00018995D460988ADF83410A8498DF81CB02C
:10D4F000179A0A718DF838B0086098F80000012872
:10D500003BD0022809D003286FD1307820F03F00AB
:10D510001D303070B8F80400E08098F80010032047
:10D52000022904D1317821F03F011B31317094F888
:10D530004610090759D505ABB9F1000F13D00021EA
:10D5400002AA82E80B000720CDE90009BDF83400EB
:10D55000B8F80410C01E83B20022159800F0EFFD49
:10D560000028D1D101E0F11CEAE7B8F80400A6F8E0
:10D570000100BDF81400C01C04E198F805108DF8F6
:10D580001C1098F80400012806D04FF4007A0228F5
:10D590002CD00328B8D16CE12188B8F8080011F428
:10D5A0000061ADF8201020D017281CD3B4F840102B
:10D5B000814218D3B4F84410172901D3814212D103
:10D5C000317821F03F01C91C3170A6F80100032118
:10D5D000ADF83410A4F8440094F8460020F002009E
:10D5E00084F8460065E105257EE177E1208808F1B1
:10D5F000080700F4FE60ADF8200010F0F00F1BD01B
:10D6000010F0C00F03D03888228B9042EBD199B92B
:10D61000B878C00710D0B9680720CDE902B1CDF8BD
:10D6200004B00090CDF810B0FB88BA8839881598FE
:10D6300000F023FB0028D6D12398BDF82010401C11
:10D6400080294ED006DC10290DD020290BD040298E
:10D6500087D124E0B1F5807F6ED051457ED0B1F501
:10D66000806F97D1DEE0C80601D5082000E01020C9
:10D6700082460DA907AA0520CDE902218DF83800C0
:10D68000ADF83CB0CDE9049608A93888CDE9000191
:10D690005346072221461598FFF7B8F8A8E09DF8F1
:10D6A0001C2001214FF00A0A002A9BD105ABB9F1D9
:10D6B000000F00D00020CDE902100720CDE90009BD
:10D6C000BDF834000493401E83B2218B00221598CC
:10D6D00000F035FD8DF81C000B203070BDF81400F3
:10D6E00020E09DF81C2001214FF00C0A002A22D1D5
:10D6F00013ABB9F1000F00D00020CDE902100720D4
:10D70000CDE900090493BDF83400228C401E83B299
:10D71000218B159800F013FD8DF81C000D20307042
:10D72000BDF84C00401CADF8340005208DF83800E1
:10D73000208BADF83C00BCE03888218B88427FF418
:10D7400052AF9DF81C004FF0120A00281CD1606AED
:10D75000A8B1B878C0073FF446AF00E018E0BA6857
:10D760000720CDE902B2CDF804B00090CDF810B09A
:10D77000FB88BA88159800F080FA8DF81C001320F9
:10D7800030700120ADF8340093E00000600000200C
:10D790003988208B8142D2D19DF81C004FF0160AA7
:10D7A0000028A06B08D0E0B34FF6FF7000215F4661
:10D7B000ADF808B0019027E068B1B978C907BED1CB
:10D7C000E18F0DAB0844821D03968DE80C0243885F
:10D7D0008288018809E0B878C007BCD0BA680DAB70
:10D7E00003968DE80C02BB88FA881598FFF7F7F9C5
:10D7F00005005ED0072D72D076E0019005AA02A93F
:10D800002046FFF72DF90146E28FBDF8080082425D
:10D8100001D00029F1D0E08FA16B08440780019866
:10D82000E08746E09DF81C004FF0180A40B1208BBD
:10D83000C8B13888208321461598FFF79AF938E057
:10D8400004F118000090237E012221461598FFF76D
:10D85000A8F98DF81C000028EDD1192030700120A6
:10D86000ADF83400E7E7052521461598FFF781F963
:10D870003AE0208800F40070ADF8200050452DD12A
:10D88000A08FA0F57F41FE3901D006252CE0D8F805
:10D8900008004FF0160A48B1A063B8F80C10A18731
:10D8A0004FF6FF71E187A0F800B002E04FF6FF707D
:10D8B000A087BDF8200030F47F611AD078230022C1
:10D8C0000320159909F074FD98F800002071208854
:10D8D000BDF82010084320800EE000E007252088D6
:10D8E000BDF8201088432080208810F47F6F1CD062
:10D8F0003AE02188814321809DF8380020B10EA9AB
:10D900001598F9F77DFC05469DF81C000028EBD022
:10D9100086F801A001203070208B70809DF81C00DB
:10D9200030710520ADF83400DEE7A18EE1B1189822
:10D930000DAB0088ADF834002398CDE90304CDE9A0
:10D940000139206B0090E36A179A1598FFF700FAE7
:10D95000054601208DF838000EA91598F9F750FCFE
:10D9600000B10546A4F834B094F8460040070AD543
:10D970002046FFF7A4F910F03E0F04D114F8460F2B
:10D9800020F0040020701898BDF83410018028465B
:10D990009BE500B585B0032806D102208DF8000074
:10D9A00088B26946F9F72CFC05B000BD10B5384CBB
:10D9B0000B782268012B02D0022B2AD111E01378B8
:10D9C0000BB1052B01D10423137023688A889A8038
:10D9D0002268CB88D38022680B89138149895181C1
:10D9E0000DE08B8893802268CB88D38022680B89D6
:10D9F00013814B8953818B89938109691161216856
:10DA0000F9F7FEFB226800210228117003D00028DC
:10DA100000D0812010BD832010BD806B002800D075
:10DA2000012070478178012909D10088B0F5205F75
:10DA300003D042F60101884201D10020704707203F
:10DA40007047F0B587B0002415460E460746ADF87E
:10DA5000184011E005980088288005980194811DE0
:10DA6000CDE902410721049400918388428801880E
:10DA7000384600F002F930B905AA06A93046FEF78B
:10DA8000EFFF0028E6D00A2800D1002007B0F0BD43
:10DA90006000002010B58B7883B102789A4205D1DE
:10DAA0000B885BB102E08B79091D4BB18B789A42F0
:10DAB000F9D1B0F801300C88A342F4D1002010BD98
:10DAC000812010BD072826D012B1012A27D103E0FA
:10DAD000497801F0070102E04978C1F3C201052944
:10DAE0001DD2DFE801F00318080C12000AB1032070
:10DAF00070470220704704280DD250B10DE0052870
:10DB000009D2801E022808D303E0062803D0032888
:10DB100003D005207047002070470F2070478120F8
:10DB20007047C0B282060BD4000607D5FA48807A47
:10DB30004143C01D01EBD00080B2704708467047DA
:10DB40000020704770B513880B800B781C0625D514
:10DB5000F14CA47A844204D843F0100008700020ED
:10DB600070BD956800F0070605EBD0052D78F540EF
:10DB700065F304130B701378D17803F0030341EAC3
:10DB8000032140F20123B1FBF3F503FB1511926869
:10DB9000E41D00FB012000EBD40070BD906870BD57
:10DBA00037B51446BDF804101180117841F0040116
:10DBB00011709DF804100A061ED5D74AA368C1F358
:10DBC0000011927A824208D8FE2811D1D21DD208C3
:10DBD0004942184600F01BFC0AE003EBD00200F0BB
:10DBE0000703012510789D40A84399400843107011
:10DBF000207820F0100020703EBD2DE9F04107464E
:10DC0000C81C0E4620F00300B04202D08620BDE8BA
:10DC1000F081C14D002034462E60AF802881AA7269
:10DC2000E8801AE0E988491CE980810614D4E1788B
:10DC300000F0030041EA002040F20121B0FBF1F2C4
:10DC400001FB12012068FFF76CFF2989084480B2AC
:10DC50002881381A3044A0600C3420784107E1D480
:10DC60000020D4E7AC4801220189C08800EB4000C5
:10DC700002EB8000084480B270472DE9FF4F89B065
:10DC80001646DDE9168A0F46994623F440450846B4
:10DC900000F054FB040002D02078400703D4012098
:10DCA0000DB0BDE8F08F099805F062FE0290207873
:10DCB000000606D59848817A0298814201D88720CB
:10DCC000EEE7224601A90298FFF73CFF83460020B9
:10DCD0008DF80C004046B8F1070F1AD001222146FA
:10DCE000FFF7F0FE0028DBD12078400611D5022096
:10DCF0008DF80C00ADF81070BDF80400ADF81200FE
:10DD0000ADF814601898ADF81650CDF81CA0ADF819
:10DD100018005FEA094004D500252E46A8460127D1
:10DD20000CE02178E07801F0030140EA012040F2A4
:10DD30000121B0FBF1F2804601FB12875FEA494006
:10DD400009D5B84507D1A178207901F0030140EA4F
:10DD50000120B04201D3BE4201D90720A0E7A81993
:10DD60001FFA80F9B94501D90D2099E79DF80C00FB
:10DD700028B103A90998F9F741FA002890D1B845CC
:10DD800007D1A0784FEA192161F30100A07084F84F
:10DD900004901A9800B10580199850EA0A0027D01B
:10DDA000199830B10BEB06002A46199900F005FBD3
:10DDB0000EE00BEB06085746189E099805F043FF46
:10DDC0002B46F61DB5B239464246009505F02FFBAD
:10DDD000224601A90298FFF7B5FE9DF804002246ED
:10DDE00020F010008DF80400DDE90110FFF7D8FEE7
:10DDF000002055E72DE9FF4FDFF81C91824685B0E2
:10DE0000B9F80610D9F8000001EB410100EB8104DC
:10DE100040F20120B2FBF0F1174600FB1175DDE97D
:10DE2000138B4E4629460698FFF77BFE0346FFF705
:10DE300019FF1844B1880C30884202D9842009B0F7
:10DE40002FE70698C6B2300603D5B00601D50620E6
:10DE5000F5E7B9F80620521C92B2A9F80620BBF1EA
:10DE6000000F01D0ABF80020B00602D5C4F808803E
:10DE70000AE0B9F808201A4492B2A9F80820D9F8A3
:10DE80000000891A0844A0602246FE200699FFF788
:10DE900087FEE77025712078390A61F301002A0AAC
:10DEA000A17840F0040062F30101A17020709AF89B
:10DEB00002006071BAF80000E0800025257330068A
:10DEC00002D599F80A7000E00127B00601D54FF09D
:10DED00000084E4600244FF007090FE0CDE9025834
:10DEE0000195CDF800900495F1882046129B089A80
:10DEF000FFF7C3FE0028A2D1641CE4B2BC42EDD3FC
:10DF000000209CE700B5FFF7ADFE03490C308A887E
:10DF1000904203D9842000BD00060020CA8808680A
:10DF200002EB420300EB8300521C037823F004034E
:10DF30000370CA80002101730846ECE72DE9F04721
:10DF4000804600F0FBF9070005D000264446F74D57
:10DF500040F2012916E00120BDE8F087204600F0DC
:10DF6000EDF90278C17802F0030241EA0222B2FB25
:10DF7000F9F309FB13210068FFF7D3FD3044641C5B
:10DF800086B2A4B2E988601E8142E7DCA8F10100F4
:10DF9000E8802889801B288100203870DCE710B5D4
:10DFA000144631B1491E218005F0E2FCA07000202A
:10DFB00010BD012010BD70B50446DC48C18803685F
:10DFC00001E0401C20802088884207D200EB4002FC
:10DFD00013EB820202D015786D07F2D580B2884229
:10DFE00016D2AAB15079A072D08820819178107988
:10DFF00001F0030140EA0120A081A078E11CFFF7B5
:10E00000A1FD20612088401C2080E080002070BDA0
:10E010000A2070BD0121018270472DE9FF4F85B0B4
:10E020004FF6FF798246A3F8009048681E460D46D9
:10E0300080788DF8060048680088ADF8040000205C
:10E040008DF80A00088A0C88A04200D304462C826E
:10E0500051E03878400708D4641C288AA4B2401CD8
:10E06000288208F10100C0B246E0288A401C2882BC
:10E07000781D6968FFF70EFDD8BB3188494501D18D
:10E08000601E30803188A1EB080030806888A04293
:10E0900038D3B878397900F0030041EA002801A9A3
:10E0A000781DFFF7F7FC20BB298949452ED00022B7
:10E0B00039460798FFF706FDD8B92989414518D197
:10E0C000E9680391B5F80AC0D7F808B05046CDF812
:10E0D00000C005F0B8FDDDF800C05A460CF1070C91
:10E0E0001FFA8CFC43460399CDF800C005F069F98E
:10E0F00060B1641CA4B200208046204600F01EF9E6
:10E100000700A6D1641E2C820A2098E674807879D4
:10E11000B071F888B0803978F87801F0030140EAEE
:10E1200001207081A6F80C80504605F021FC3A468B
:10E1300006F10801FFF706FD306100207FE62DE9BA
:10E14000FF4F87B081461C469246DDF860B0DDF88F
:10E150005480089800F0F2F8050002D028784007B3
:10E1600002D401200BB09CE5484605F001FC29785B
:10E17000090605D56D49897A814201D88720F1E7E2
:10E18000CAF309062A4601A9FFF7DCFC07461498E2
:10E1900007281CD000222946FFF794FC0028E1D173
:10E1A0002878400613D501208DF808000898ADF8AE
:10E1B0000C00BDF80400ADF80E00ADF81060ADF82D
:10E1C000124002A94846F9F719F80028CAD129785F
:10E1D000E87801F0030140EA0121AA78287902F0E9
:10E1E000030240EA0220564507D0B1F5007F04D96A
:10E1F000611E814201DD0B20B4E7864201D9072070
:10E20000B0E7801B85B2A54200D92546BBF1000FBF
:10E2100001D0ABF80050179818B1B9192A4600F090
:10E22000CCF8B8F1000F0DD03E4448464446169F46
:10E2300005F01BFD2146FF1DBCB232462B46009463
:10E2400005F029F900208DE72DE9F04107461D462C
:10E250001646084600F072F8040002D02078400705
:10E2600001D40120D3E4384605F082FB2178090669
:10E2700005D52E49897A814201D88720C7E42246F4
:10E280003146FFF75FFC65B12178E07801F00301CA
:10E2900040EA0120B0F5007F01D8012000E0002015
:10E2A00028700020B3E42DE9F04107461D461646CC
:10E2B000084600F043F8040002D02078400701D45B
:10E2C0000120A4E4384605F053FB2178090605D562
:10E2D0001649897A814201D8872098E4224631463E
:10E2E000FFF75EFCFF2D14D02178E07801F00302E7
:10E2F00040EA022040F20122B0FBF2F302FB1300DD
:10E3000015B900F2012080B2E070000A60F301014B
:10E31000217000207BE410B50C4600F00FF810B11E
:10E320000178490704D4012010BD00000006002038
:10E33000C18821804079A0700020F5E70749CA888C
:10E34000824209D340B1096800EB40006FF00B0234
:10E3500002EB800008447047002070470006002050
:10E3600070B504460D4621462B460AB9002070BD03
:10E3700001E0491C5B1C501E021E03D008781E7869
:10E38000B042F6D008781E78801BF0E730B50C4616
:10E3900001462346051B954206D202E0521E9D5CB3
:10E3A0008D54002AFAD107E004E01D780D70491C55
:10E3B0005B1C521E002AF8D130BDF0B50E46014656
:10E3C000334680EA030404F00304B4B906E002B95A
:10E3D000F0BD13F8017B01F8017B521E01F0030729
:10E3E000002FF4D10C461D4602E080CD80C4121FE0
:10E3F000042AFAD221462B4600BF04E013F8014B51
:10E4000001F8014B521E002AF8D100BFE0E7F0B539
:10E410000C460146E6B204E002B9F0BD01F8016B1A
:10E42000521E01F00307002FF6D10B46E5B245EA74
:10E43000052545EA054501E020C3121F042AFBD249
:10E44000194602E001F8016B521E002AFAD100BF02
:10E45000E3E710B509F0D5FAF4F73AFA09F04CF908
:10E46000BDE8104009F014BA202834BF0120002074
:10E470007047012303FA00F04FF0A042002914BFB7
:10E48000C2F80C05C2F8080570474FF0A041012200
:10E4900002FA00F0C1F81805704770B50346002075
:10E4A00002466FF02F050EE09C5CA4F130060A2EA8
:10E4B00002D34FF0FF3070BD00EB800005EB400051
:10E4C000521C2044D2B28A42EED370BD30B50A232A
:10E4D0000BE0B0FBF3F403FB1404B0FBF3F08D1876
:10E4E0003034521E05F8014CD2B2002AF1D130BDB1
:10E4F00030B500234FF6FF7510E0040A44EA00200F
:10E5000084B2C85C6040C0F30314604005EA003484
:10E510004440E0B25B1C84EA40109BB29342ECD3CF
:10E5200030BD00002DE9F041FE4B0026012793F895
:10E5300064501C7893F868C0B8B183F89140A3F890
:10E54000921083F8902083F88E70BCF1000F0CBFFE
:10E5500083F8946083F89450F3488068008805F04D
:10E5600072FBBDE8F04105F009B84FF6FF7083F883
:10E570009140A3F8920083F8902083F88E70BCF14C
:10E58000000F14BF83F8945083F89460BDE8F081C5
:10E590002DE9F041E44D296891F89C200024012ADE
:10E5A00023D091F89620012A30D091F86C301422B3
:10E5B000DC4E0127012B32D091F88E30012B4FD049
:10E5C00091F8A620012A1CBF0020BDE8F08144700C
:10E5D0001F2200F8042B2222A731FFF7EEFE286845
:10E5E00080F8A6400120BDE8F08144701B22027033
:10E5F000D1F89D204260D1F8A120826091F8A52039
:10E60000027381F89C400120BDE8F081447007222C
:10E610000270D1F89820426081F89640E2E7804687
:10E62000447000F8042B20226E31FFF7C6FE88F8F4
:10E630000870286880F86C4090F86E000028D1D1EE
:10E64000B6F87000A6F89800A868417B86F89A1082
:10E6500086F89670008805F0F6FA04F09EFFC1E790
:10E6600091F86C30012B0BD0447017220270D1F856
:10E6700090204260B1F89420028181F88E40B1E789
:10E680008046447000F8042B20226E31FFF795FE7F
:10E6900088F80870286880F86C4090F86E000028B0
:10E6A000A0D1CDE7A048006890F86C10002914BFF5
:10E6B000B0F870004FF6FF70704770B59A4C064680
:10E6C0002068002808BFFFDF0025206845706660CD
:10E6D000002808BFFFDF2068417800291CBFFFDF4A
:10E6E00070BDCC220021FFF792FE2068FF2101704F
:10E6F0007F2180F8371013214184282180F8691088
:10E70000012180F85C1080F8615009F0D7FEBDE867
:10E71000704009F01EB884490968097881420CBF2D
:10E720000120002070478048006890F82200C0F364
:10E73000400070477C48006890F8220000F001001B
:10E7400070477948006890F82200C0F300107047C5
:10E750002DE9F0437448D0F800C09CF82400BCF8C0
:10E760002240C0F38001C0F34002114400F00100D8
:10E770000144C4F30010B0B1102C02BF6B4830F854
:10E780001100BDE8F083122C14BF132C684806D08A
:10E79000152C1BBFFFDF00206648BDE8F08330F872
:10E7A0001100BDE8F0839CF85E209CF85F002E26E7
:10E7B00000234FF47A774FF014084FF04009022AF3
:10E7C00004BF4AF2D745B5FBF7F510D0012A04BFC4
:10E7D0004AF22F75B5FBF7F510D04AF62315B5FBB5
:10E7E000F7F5082A08BF4E4613D0042A18D01E4653
:10E7F000082A0ED0042A13D0022A49D003F1280691
:10E80000042A0FD0082A1CBF4FF01908082204D090
:10E810000AE04FF0140806F5A8764FF0400203E036
:10E8200006F5A8764FF0100218FB026212FB0152A7
:10E83000C1EB0111404D01EB810105EB8101114458
:10E8400014F0010F4FF4C8724FF4BF7504BFC4F346
:10E850004006002E72D0C4F3400601F5A571EEB15A
:10E86000082804BF174640260CD0042804BF2F46B2
:10E87000102607D0022807BF03F11807042603F16A
:10E880002807082606EB860808EB86163E441BE0A0
:10E8900003F118064FF019080422C5E7082804BF41
:10E8A000164640270CD0042804BF2E46102707D058
:10E8B000022807BF03F11806042703F128060827DA
:10E8C00007EB871706EB870631449C31082804BF05
:10E8D000164640270CD0042804BF2E46102707D028
:10E8E000022807BF03F11806042703F128060827AA
:10E8F000C7EBC70707EB470706EB470631449831DC
:10E9000014F0010F26D0082808BF40201BD004288F
:10E9100004BF2A46102016D0022804BF03F11802B3
:10E9200004200CE00C06002068000020C454020003
:10E93000BC540200CC540200D4FEFFFF4DE01CBFCB
:10E9400003F12802082000EB400303EB0010104401
:10E9500001443EE0082804BF144640260CD0042899
:10E9600004BF2C46102607D0022807BF03F1180465
:10E97000042603F12804082606EB8616BCF840C0DE
:10E9800004EB86042144BCF1EB0F22D944F2552458
:10E990000CF10B0C0CFB04FC4FEA9C5C082807D024
:10E9A000042802D0022805D008E02A46102008E0FA
:10E9B000402006E003F11802042002E003F12802DF
:10E9C000082000EB801002EB800000F5A5700CFB26
:10E9D000001101F5B470BDE8F08301F5A5740828B5
:10E9E00004BF164640210CD0042804BF2E46102137
:10E9F00007D0022807BF03F11806042103F12806F7
:10EA0000082101EB8111BCF848C006EB81012144CB
:10EA1000BCF1EB0FDDD944F255240CF10B0C0CFBCF
:10EA200004FC4FEA9C5C0828C2D00428BDD0022810
:10EA3000C4D1BFE7FE4840F271210068806A4843B4
:10EA40007047FB48006890F83600002818BF012086
:10EA5000704710B5F74C207B022818BF032808D157
:10EA6000207D04F115010EF046FA08281CBF012094
:10EA700010BD207B002816BF022800200120BDE821
:10EA800010400AF02FB9EB4908737047E84909684C
:10EA900081F8300070472DE9F047E54C2168087B8C
:10EAA000002816BF022800200120487301F10E0142
:10EAB0000AF002F92168087B022816BF0328012208
:10EAC000002281F82F204FF0080081F82D00487BAC
:10EAD00001F10E034FF001064FF00007012804BFBB
:10EAE0005B7913F0C00F0AD001F10E03012804D1A5
:10EAF000587900F0C000402801D0002000E001203B
:10EB000081F82E00002A04BF91F8220010F0040FB3
:10EB100007D0087D01F115010EF0EDF9216881F8AB
:10EB20002D002068476007F0BBF82168C14D4FF009
:10EB30000009886095F82D000EF0E9F9804695F8F7
:10EB40002F00002818BFB8F1000F04D095F82D0051
:10EB50000EF011F868B195F8300000281CBF95F848
:10EB60002E0000281DD0697B05F10E0001290ED072
:10EB700012E06E734A4605F10E0140460AF0F2F8C3
:10EB800095F82D1005F10E000EF0C3FA09E040795A
:10EB900000F0C000402831D0394605F10E000AF0DF
:10EBA00019F92068C77690F8220010F0040F08BF0A
:10EBB000BDE8F087002795F82D000EF077F80500E6
:10EBC00008BFBDE8F087102102F08DF8002818BFBB
:10EBD000BDE8F08720683A4600F11C01C676284659
:10EBE0000AF0C0F8206800F11C0160680EF0EEFB2E
:10EBF0006068BDE8F04701210EF003BC0EF0C6FAD4
:10EC00004A4605F10E010AF0ADF8CAE7884A1268D3
:10EC1000137B0370D2F80E000860508A888070471A
:10EC200078B584490446824D407B08732A68207871
:10EC300010706088ADF8000080B200F00101C0F3F0
:10EC4000400341EA4301C0F3800341EA8301C0F37A
:10EC5000C00341EAC301C0F3001341EA0311C0F34A
:10EC6000401341EA4311C0F3801041EA8010508400
:10EC7000E07D012808BF012603D0022814BFFFDF72
:10EC80000226286880F85E60607E012808BF0126A1
:10EC900003D0022814BFFFDF0226286880F85F60D7
:10ECA000217B80F82410418C1D290CBF0021616854
:10ECB0008162617D80F83610A17B002916BF022990
:10ECC000002101210175D4F80F10C0F81510B4F817
:10ECD0001310A0F81910A17E90F86B2061F30712B1
:10ECE00080F86B20E17E012918BF002180F83410E4
:10ECF000002078BD4E480068408CC0F3001131B14F
:10ED0000C0F38000002804BF1F20704702E0C0F35A
:10ED1000400109B10020704710F0010F14BFEE2030
:10ED2000FF20704742480068408CC0F3001119B1C1
:10ED3000C0F3800028B102E0C0F3400008B1002019
:10ED40007047012070473A49002209684A664B8C97
:10ED50001D2B0CBF81F8682081F8680070470023E4
:10ED6000334A126882F85D30D164A2F85000012065
:10ED700082F85D0070472E4A0023126882F85C30EA
:10ED8000A2F858000120516582F85C0070472849BC
:10ED9000096881F8350070472549096881F86100E4
:10EDA00070472348006890F9610070472048006868
:10EDB00090F82200C0F3401070471D48006890F89A
:10EDC0002200C0F3C0007047012070471848006857
:10EDD00090F85F00704770B509F051FB09F030FB07
:10EDE00009F0F1F909F09EFA114C2068416E491CB6
:10EDF000416690F83300002530B109F05FFB08F060
:10EE0000A8FC206880F833502068457090F83810CE
:10EE100021B1BDE8704004200AF0BDBB90F8681035
:10EE200001B3406E81421DD804200AF0B4FB03E018
:10EE3000680000200C060020206890F8220010F0E6
:10EE4000010F07D0A06843220188BDE8704001206F
:10EE5000FFF768BBBDE8704043224FF6FF7100200A
:10EE6000FFF760BBBDE8704000200AF094BB2DE9BD
:10EE7000F04782B00F468246FE4E4FF000093068E0
:10EE8000458C15F0030F10D015F0010F05F00200AE
:10EE900005D0002808BF4FF0010906D004E0002883
:10EEA00018BF4FF0020900D1FFDF4FF000084446C1
:10EEB00015F0010F05F002000DD080B915F0040F18
:10EEC0000DD048F00800002F1CBF40F0010040F0BA
:10EED000020438D06EE010B115F0040F0DD015F01B
:10EEE000070F10D015F0010F05F002002ED00028FA
:10EEF00008BF15F0040F1FD035E0002F18BF48F0F1
:10EF0000090457D12CE02FB148F0080415F0200F68
:10EF10004CD04FE0306805F02001B0F848000843BD
:10EF200008BF48F0010445D048F0180415F0200F40
:10EF300008BF44F001043DE048F00800002F18BF6E
:10EF400040F0010436D140F0100433E0002818BF2F
:10EF500015F0040F07D0002F18BF48F00B0429D17B
:10EF600048F0180426E015F0030F22D115F0040F25
:10EF70001FD03FB128F0020040F0080415F0200F28
:10EF800014D017E0306805F02001B0F848000843BD
:10EF900008BF48F003040DD048F0180015F0200F0A
:10EFA00008BF40F0010040F0020403E024F0010437
:10EFB00000E0FFDF15F0400F12D07FB93068B0F8E5
:10EFC0004810002904BF408C10F0010F06D110F04A
:10EFD000020F04BF10F0200F15F0010F44F04004A1
:10EFE0007068A0F80080017821F0200101704FF0D6
:10EFF00007010EF0B7F9494670680EF0AAFB2146EA
:10F0000070680EF0B2FB14F0010F0CD04FF0060345
:10F010004FF00002984970680EF081FB3068417B28
:10F0200070680EF0E1F914F0020F18D0D6E9001064
:10F03000BAF1000F4FF006034FF0010207D01C3168
:10F040000EF06DFB012170680EF0DBF907E0153161
:10F050000EF065FB3068017D70680EF0D2F914F097
:10F06000040F18BFFFDF14F0080F19D0CDF800808F
:10F070003068BDF800200223B0F86A1061F30B027B
:10F08000ADF8002090F86B00032201099DF8010003
:10F0900061F307108DF80100694670680EF03FFBC0
:10F0A000012F62D13068B0F84810E1B390F8220027
:10F0B000C0F34000B8BB70680EF047FB401CC7B2FD
:10F0C0003068C7F1FF05B0F84820B0F85A10511A5F
:10F0D000A942B8BF0D46AA423BD990F8220010F0D1
:10F0E000010F36D144F01004214670680EF03DFB4C
:10F0F000F81CC0B2ED1E284482B23068B0F86A1025
:10F10000436EC1F30B0151FA83F190F860305B4F0D
:10F110001944BC460023E1FB07C31B096FF0240C14
:10F1200003FB0C1100E020E080F8601090F85F0015
:10F13000012101F008F90090BDF800009DF80210CF
:10F14000032340EA01400190042201A970680EF0F7
:10F15000E6FA3068AAB2416C70680EF034FB306891
:10F16000B0F85A102944A0F85A1014F0400F06D0F5
:10F17000D6E900100123062261310EF0D0FA14F016
:10F18000200F18BFFFDF0020002818BFFFDF02B0EC
:10F19000BDE8F0872DE9F043364C89B0206800289F
:10F1A00008BFFFDF20684178002936D10178FF29A8
:10F1B00033D0002680F83160A0F85A60867080F85D
:10F1C0003860304609F0CEF82D4802AD00F1240138
:10F1D00091E80E1085E80E10D0E90D10CDE906106B
:10F1E00002A809F0ADF808F00AFD206890F9610066
:10F1F00008F0DAFD234808F0DDFD234809F08CF81B
:10F20000606809F0B2F8206890F8240010F0010F4F
:10F2100007D0252008F0D6FD0AE009B00C20BDE893
:10F22000F08310F0020F18BF262077D008F0CAFD37
:10F23000206890F85E10252008F0ADFC206880F86A
:10F240002C6009F089F8206890F85E10002008F022
:10F25000B5FE0F21052008F07BFD206890F82E10E8
:10F26000002901BF90F82F10002990F8220010F01B
:10F27000040F0BE0680000201A06002053E4B36E70
:10F28000B0540200B8540200B554020075D006F024
:10F2900007FD054620682946806807F0F9F9DFF880
:10F2A0002C84074690FBF8F008FB1070414228467A
:10F2B00006F0DDF92168886097FBF8F04A68104491
:10F2C00048600DF015FE01462068426891426FD8F3
:10F2D000C0E90165FE4D4FF0010895F82D000DF0D5
:10F2E00016FE814695F82F000127002818BFB9F1B6
:10F2F000000F04D095F82D000DF03DFCA8B195F855
:10F30000300000281CBF95F82E00002825D0687B0F
:10F3100005F10E01012816D01AE0FFE710F0040FE6
:10F3200014BF2720FFDF81D182E73A466F7305F1D2
:10F330000E01484609F016FD95F82D1005F10E0056
:10F340000DF0E7FE09E0487900F0C000402815D034
:10F35000414605F10E0009F03DFD206890F82200BD
:10F3600010F0040F24D095F82D000DF09FFC05003F
:10F370001ED0102101F0B7FC40B119E00DF006FFDE
:10F380003A4605F10E0109F0EDFCE6E720683A4641
:10F3900000F11C01C776284609F0E4FC206800F162
:10F3A0001C0160680EF012F8012160680EF029F867
:10F3B0002068417B0E3008F0ADFC206890F85C10AE
:10F3C00061B3B0F85810A0F84810416D416490F84E
:10F3D0002210C1F30011F1B9B0F86A000221C0F3A4
:10F3E0000B05ADF80050684607F086FD28B1BDF862
:10F3F0000000C0F30B00A84204D1BDF80000401C7F
:10F40000ADF800002168BDF80000B1F86A2060F393
:10F410000B02A1F86A20206880F85C60206890F8F0
:10F420005D1039B1B0F85010A0F84010C16CC16344
:10F4300080F85D60B0F86A10426EC1F30B0151FABA
:10F4400082F190F86020DFF88CC2114463460022FC
:10F45000E1FB0C3212096FF0240302FB031180F868
:10F4600060100DF0BEFD032160680DF042FE2168C2
:10F4700081F8330009B00020BDE8F0839649886028
:10F4800070472DE9F043944C83B0226892F83130F4
:10F490003BB1508C1D2808BFFFDF03B0BDE8F0432F
:10F4A00099E401260027F1B1054692F8600008F0C2
:10F4B00089FC206890F85F10FF2008F06CFB206842
:10F4C0004FF4A57190F85F20002008F03FFE2068FF
:10F4D00090F8221011F0030F00F02C81002D00F0A5
:10F4E000238100F027B992F822108046D07EC1F324
:10F4F0000011002956D0054660680780017821F088
:10F5000020010170518C132937D01FDC102908BF4E
:10F51000022144D0122908BF062140D0FFDF6C4DE4
:10F52000606805F10E010DF043FF697B60680DF026
:10F530005BFF2068418C1D2918BF152963D0B0F8E6
:10F540004820416C60680DF068FF5CE0152918BF29
:10F550001D29E3D14FF001010DF004FF606801782F
:10F5600041F020010170216885B11C310DF02EFFA2
:10F57000012160680DF045FFD1E700210DF0F2FE9A
:10F580006068017841F020010170C8E715310DF085
:10F590001DFF2068017D60680DF033FFBFE70DF0AF
:10F5A000E1FEBCE70021FFF762FC6068C17811F062
:10F5B0003F0F28D0017911F0100F24D00DF0D0FEAC
:10F5C0002368024693F82410C1F38000C1F3400C75
:10F5D000604401F00101084493F82C10C1F3800C41
:10F5E000C1F34005AC4401F001016144401AC1B2CD
:10F5F00093F85E0000F0A7FE009003230422694602
:10F6000060680EF08CF82068002590F8241090F8BF
:10F610002C0021EA000212F0010F18BF01250ED1C3
:10F6200011F0020F04D010F0020F08BF022506D01F
:10F6300011F0040F03D010F0040F08BF0425B8F137
:10F64000000F2BD0012D1BD0022D08BF26201BD070
:10F65000042D14BFFFDF272016D0206890F85E101D
:10F66000252008F098FA206890F82210C1F30011C4
:10F6700069B101224FF49671002008F067FD0DE09A
:10F68000252008F09FFBE8E708F09CFBE5E790F8F1
:10F690005E204FF49671002008F058FD206890F825
:10F6A0002C10294380F82C1090F8242032EA010114
:10F6B0001CD04670418C13292BD026DC102904BFA6
:10F6C00003B0BDE8F083122923D007E040420F00C9
:10F6D0000C06002053E4B36E68000020C1F3001054
:10F6E000002818BFFFDF03B0BDE8F083418C1D295F
:10F6F00008BF80F82C70DCD0C1F30011002914BFC2
:10F7000080F8316080F83170D3E7152918BF1D29C2
:10F71000DBD190F85E2003B04FF00101BDE8F0436B
:10F72000084608F008BF00BF90F85F200121084696
:10F7300008F001FF2168002DC87E7CD04A8C3D4630
:10F74000C2F34000002808BF47F0080512F0400F40
:10F7500018BF45F04005002819BFD1F83C90B1F81A
:10F760004080D1F84490B1F8488060680721078054
:10F770000DF0F8FD002160680DF0EBFF2946606890
:10F780000DF0F3FF15F0080F17D02068BDF800103A
:10F790000223B0F86A2062F30B01ADF8001090F874
:10F7A0006B00032201099DF8010061F307108DF839
:10F7B0000100694660680DF0B2FF60680DF08EFED2
:10F7C0002168C0F1FE00B1F85A20A8EB0201814285
:10F7D000A8BF0146CFB2D019404544D245F0100130
:10F7E00060680DF0C2FF60680DF078FE2168C0F11E
:10F7F000FE00B1F85A10A8EB01018142A8BF0146F2
:10F80000CFB260680DF0A1FF3844421C2068B0F808
:10F810006A10436EC1F30B0151FA83F190F8603026
:10F82000F74D1944AC460023E1FB05C34FEA131C16
:10F830006FF0240300E03CE00CFB031180F8601043
:10F8400090F85F00012100F07EFD0090BDF80000FF
:10F850009DF80210032340EA01400190042201A90F
:10F8600060680DF05CFF216891F8220010F0400FF5
:10F8700005D001230622613160680DF050FF206839
:10F880003A46B0F85A0000EB090160680DF09BFFA2
:10F890002068B0F85A103944A0F85A1009F03DF920
:10F8A000002818BFFFDF20684670867003B0BDE8EF
:10F8B000F0830121FFF7DBFAF0E7D24810B50068CA
:10F8C000417841B90078FF2805D000210846FFF7AC
:10F8D000D8FD002010BD08F0D2FD08F0B1FD08F001
:10F8E00072FC08F01FFD0C2010BD2DE9F041C54D44
:10F8F0000446174628680E4690F86C00002818BF8A
:10F90000FFDF2868002F80F86E7018BFBDE8F08117
:10F910002188A0F870106188A0F88610A188A0F84E
:10F920008810E188A0F88A1094F8891180F88C106A
:10F9300090F82F10002749B1427B00F10E01012AF7
:10F9400004D1497901F0C001402935D090F8301038
:10F9500041B1427B00F10E01012A04BF497911F047
:10F96000C00F29D000F17A00F3F746FB6868FF2E3C
:10F970000178C1F380116176D0F80310C4F81A1031
:10F98000B0F80700E08328681ED0C0F88010E18B33
:10F99000A0F8841000F17402511E30460DF0C6FA32
:10F9A000002808BFFFDF286890F8731041F00201BB
:10F9B00080F87310BDE8F081D0F80E10C0F87A100E
:10F9C000418AA0F87E10D1E7C0F88070A0F884705A
:10F9D000617E80F87310D4F81A104167E18BA0F8AB
:10F9E0007810BDE8F08170B5864C0125206890F84C
:10F9F0002200C0F3C00038B13C22FF21A068FFF70D
:10FA000074FF206880F86C50206890F8220010F095
:10FA1000010F1CBFA06801884FF03C0212BF0120FB
:10FA20004FF6FF710020FEF77DFD206880F838500A
:10FA300070BD7449096881F8320070472DE9F041C2
:10FA4000704C00272068417801253E46012906D0E8
:10FA5000022901D003297BD0FFDFBDE8F081817846
:10FA600002260029418C37D0C1F34002002A08BF8A
:10FA700011F0010F6DD090F85F204FF001014FF0B1
:10FA8000000008F058FD216891F82200C0F3400002
:10FA9000002814BF0C20222091F85F1008F07BF89A
:10FAA0002068467090F8330020B107F03EFE4020F9
:10FAB00008F0F1FC206890F83400002818BF08F026
:10FAC00017FD0021962008F07FFC09F01DF80028A2
:10FAD00018BFFFDFBDE8F081C1F3001282B1102929
:10FAE0003ED090F8330020B107F01FFE402008F010
:10FAF000D2FC206890F8221011F0040F35D042E0BB
:10FB000090F8242090F82C309A4229D1B0F848007F
:10FB1000002808BF11F0010F05D111F0020F08BF36
:10FB200011F0200F6BD04FF001014FF00000FFF7F4
:10FB3000A8FC2068418C11F0010F04BFC1F3400103
:10FB400000290AD1B0F85A10B0F84820914201E0DB
:10FB500032E026E018BFBDE8F08180F83150B9E707
:10FB6000BDE8F041002101208BE490F83610012916
:10FB700014BF0329102747F00E0190F85E204FF0C4
:10FB8000000008F0D8FC206890F83400002818BF66
:10FB900008F0AEFC0021962008F016FC20684670A4
:10FBA00098E7B0F85A10B0F84800814240D0BDE85C
:10FBB000F0410121084664E48178D9B1418C11F00B
:10FBC000010F21D080F86C5090F86E20B0F87010C2
:10FBD0000120FEF7A7FC2068467008F050FC08F0F2
:10FBE0002FFC08F0F0FA08F09DFBBDE8F04103207F
:10FBF00009F0D1BC8178BDE8F041012041E417E073
:10FC000053E4B36E6800002011F0020F08BFFFDF5D
:10FC10003FF460AFB0F85A10B0F84000814207D00E
:10FC200001210846FFF72DFC21680320487051E7A9
:10FC3000BDE8F041FFF7CFB8FFF7CDB810B5FE4CE7
:10FC4000206890F8341049B1373008F05CFC18B9DE
:10FC500021687F2081F8370008F040FC206890F888
:10FC6000330018B108F02AFC07F073FD0AF06EF8B3
:10FC7000A8B1206890F82210C1F3001179B1407842
:10FC8000022818BFFFDF00210120FFF7FAFB2068E0
:10FC9000417800291EBF40780128FFDF10BDBDE874
:10FCA0001040FFF798B82DE9F047E34C0F46804627
:10FCB0002168B8F1030F488C08BFC0F3400508D095
:10FCC00000F0010591F83200002818BF4FF001093B
:10FCD00001D14FF0000908F069F80646B8F1030FAA
:10FCE0000CBF4FF002084FF0010835EA090008BFC9
:10FCF000BDE8F087206890F8330068B10DF054F942
:10FD000038700146FF2807D06068C01C0DF025F947
:10FD100038780DF056F9064360680178C1F3801217
:10FD200021680B7D9A4208D10622C01C1531FEF7CE
:10FD300017FB002808BF012000D000203978FF29D8
:10FD400006D0C8B9206890F82D00884216D113E07B
:10FD5000A0B1616811F8030BC0F380100DF0CBF86F
:10FD600005460DF026FA38B128460CF09FFF18B171
:10FD7000102100F0B8FF08B1012000E00020216848
:10FD800091F8221011F0040F01D0F0B11AE0CEB9B1
:10FD9000AA4890F83600002818BF404515D1616880
:10FDA00011F8030BC0F380100DF0A5F804460DF018
:10FDB00000FA38B120460CF079FF18B1102100F09C
:10FDC00092FF10B10120BDE8F0870020BDE8F08768
:10FDD0002DE9F04F984D044683B0286800264078FE
:10FDE000022818BFFFDF28684FF07F0A90F8341010
:10FDF00049B1373008F087FB002804BF286880F835
:10FE000037A008F06BFB68680DF0CEFA8046002C36
:10FE100000F0418207F098FF002800F03C820124A6
:10FE200000274FF0FF09B8F1050F1ED1686890F860
:10FE3000240000F01F00102817D9286890F835001A
:10FE400098B18DF8009069460520FFF72CFF002837
:10FE500000F02182286880F8A64069682222A73035
:10FE6000C91CFEF7AAFA00F016BA68680DF027FC64
:10FE7000002800F010824046DFF8C0814FF0030BED
:10FE8000062880F01D82DFE800F0FCFCFC03FCFB90
:10FE90008DF8009069460320FFF705FF002800F069
:10FEA000F180296891F8340010B191F89C00D8B124
:10FEB0002868817801294DD06868042107800DF0F9
:10FEC00051FA08F10E0168680DF072FA98F80D10F9
:10FED00068680DF089FA2868B0F84020C16B68683E
:10FEE0000DF0BFFA00F05FB99DF8000081F89C406A
:10FEF0000A7881F89D20FF280FD001F19F029E31E2
:10FF00000DF014F8002808BFFFDF286890F89E1055
:10FF100041F0020180F89E100DE068680278C2F39B
:10FF2000801281F89E20D0F80320C1F89F20B0F8FD
:10FF30000700A1F8A300286800F1A50490F8370095
:10FF40007F2808BFFFDF286890F83710217080F8FD
:10FF500037A0ADE790F822000721C0F38019384898
:10FF60000479686869F3861407800DF0FBF90021B5
:10FF700068680DF0EEFB214668680DF0F6FB06237D
:10FF8000002208F10E0168680DF0C9FB2868417B6A
:10FF900068680DF029FA68680DF0A0FA2968B1F8D0
:10FFA0004020C0F1FE018A42B8BF1146CFB2BA422A
:10FFB0003CD9F81EC7B244F0100A514668680DF0EB
:10FFC000D4FB68680DF0C1FB384400F101082868D3
:10FFD000B0F86A10426EC1F30B0151FA82F190F849
:10FFE0006020184C0A44A4460023E2FB04C319090C
:10FFF0006FF0240301FB032180F8601090F85F008C
:020000040001F9
:100000004246012100F09FF90190BDF804009DF8DF
:100010000610032340EA01400290042202A9686806
:100020000DF07DFB514668680DF09FFBB9F1000FA4
:100030000FD0D5E9001007E0680000200C06002072
:10004000B054020053E4B36E0123062261310DF077
:1000500066FB28683A46C16B68680DF0B4FB2868F7
:10006000A0F85A70B0F840108F420CBF0121002157
:1000700080F8311008F051FD002818BFFFDF92E032
:1000800007E01DE128688078002840F0068100F034
:1000900002B98DF8009068680178C1F38019D0F832
:1000A00003100191B0F80700ADF80800694605207B
:1000B000FFF7F9FD0028286879D08178002978D0E9
:1000C00090F85FA0D5E90104D0F80F10C4F80E1025
:1000D000B0F813106182417D2175817D6175B0F8A2
:1000E0001710E182B0F819106180B0F81B10A180E0
:1000F000B0F81D10E18000F11F0104F1080015F0B7
:10010000BEF8686890F8241001F01F01217690F87D
:1001100024000021400984F8890184F864A084F84F
:1001200065A004F130000DF04FFD2868002290F822
:10013000691084F8661090F8610084F867009DF8F3
:100140000010A868FFF7D1FB022009F024FAAD489F
:100150000DF1040A08210468686807800DF002F9AF
:10016000002168680DF0F5FA214668680DF0FDFA87
:100170000623002208F10E0168680DF0D0FA286805
:10018000417B68680DF030F9494668680DF039F92F
:1001900006230122514668680DF0C1FA08F0BDFC43
:1001A000002818BFFFDF286880F801B077E06DE015
:1001B000FFE76868D5F808804FF00109027898F8E1
:1001C0000D10C2F34012114088F80D10D0F80F1036
:1001D000C8F80E10B0F81310A8F81210417D88F876
:1001E0001410817D88F81510B0F81710A8F81610B3
:1001F000B0F81910A8F80210B0F81B10A8F80410F5
:10020000B0F81D10A8F8061000F11F0108F1080051
:1002100015F035F8686890F8241001F01F0188F88F
:10022000181090F824000021400988F8890188F806
:10023000649088F8659008F130000DF0C5FC2868DE
:10024000002290F8691088F8661090F8610088F82C
:1002500067009DF80010A868FFF747FB286880F842
:100260006C4090F86E20B0F870100120FEF75AF93B
:100270002868477008F003F908F0E2F807F0A3FFD8
:1002800008F050F8012009F086F908E090F8220003
:10029000C0F3001008B1012601E0FEF79CFD2868BC
:1002A00090F8330018B108F009F907F052FA96B146
:1002B00009F04CFD60B100210120FFF7E2F813E0E6
:1002C000286890F82200C0F300100028E5D0E2E78B
:1002D000FEF781FD08E028688178012904D190F8B3
:1002E0005F10FF2007F057FC28684178002919BFEC
:1002F0004178012903B0BDE8F08F4078032818BF8A
:10030000FFDF03B0BDE8F08F70B53F4C06460D46E9
:100310002068807858B107F0A5FB21680346304675
:1003200091F85F202946BDE8704009F0BEBE07F095
:1003300099FB21680346304691F85E202946BDE8C6
:10034000704009F0B2BE78B50C4600210091082833
:1003500004BF4FF4C87040210DD0042804BF4FF4EF
:10036000BF70102107D0022807BF01F11800042137
:1003700001F128000821521D02FB010622489DF8C8
:100380000010006890F8602062F3050141F040051C
:100390008DF8005090F85F00012804BF9DF802001E
:1003A00020F0E0002BD0022818BFFFDF22D000BFD2
:1003B00025F080008DF80000C4EB041000EB8000F5
:1003C0001E2101EB800006FB04041048844228BF74
:1003D000FFDF0F48A0FB0410BDF80110000960F317
:1003E0000C01ADF80110BDF800009DF8021040EAC4
:1003F000014078BD9DF8020020F0E00020308DF82B
:100400000200D5E7B054020068000020C4BF03001A
:10041000898888880023C383428401EBC202521E6C
:10042000B2FBF1F10184704770B46FF01F02010C50
:1004300002EA90251F23A1F5AA4054381CBFA1F55C
:10044000AA40B0F1550009D0A1F52850AA381EBF26
:10045000A1F52A40B0F1AA00012000D100204FF000
:10046000000C62465FF001048CEA0106F643164375
:10047000B6F1FF3F11D005F001064FEA5C0C4CEAE3
:10048000C63C03F0010652086D085B08641C42EA92
:10049000C632162CE8DD70BC704770BC0020704777
:1004A0002DE9F04701270025044600293BD05522BD
:1004B00033234FF4FA4C01297DD0022900F05481F6
:1004C000032918BFBDE8F08704F17000217B01F01B
:1004D0001F01217384F889505FF0000104EB010CC7
:1004E0009CF8085002EA550CA5EB0C0C0CF0FF0C24
:1004F0000CF0330503EA9C0CAC4445180CEB1C1CB7
:100500000CF00F0C85F814C0457E491CAC44C9B2F0
:1005100080F819C00529E1D30CF0FF00252888BF19
:10052000FFDFBDE8F08704F170068022002130462D
:10053000FDF76DFFB571F57135737573F57335742E
:100540007571B576F576212086F84000412086F851
:100550004100FE2086F87400268870220021204683
:10056000FDF755FF268084F8647084F865702820B4
:1005700084F86600002104F130000DF025FB1B22F9
:10058000A4F84E20A4F85020A4F85220A4F8542037
:100590004FF4A470A4F85600A4F8580067734FF401
:1005A00048606080A4F8F050A4F8F250A4F8F45029
:1005B000A4F8F65000E021E0A4F8F85084F8FA50CE
:1005C00084F8FD50A4F8065184F80451A4F8185199
:1005D000A4F81A5184F8B65184F8B75184F8C05180
:1005E00084F8C15184F88C5184F88F5184F8A85153
:1005F000C4F8A051C4F8A451BDE8F087A4F806518E
:1006000084F8FB506088FE490144B1FBF0F1A4F886
:1006100090104BF68031A4F89210E688A4F8985018
:10062000B4F89C80F60008FB00F8B6FBF0F698FBE7
:10063000F0F8761CA4F89C80B6B206FB00F804F132
:100640007001A4F89A60B8F5C84FC4BF761E4E85F5
:10065000BCFBF0FC0CF1010CA1F830C000F5802CC3
:100660000CF5EE3CACF10106B6FBF0FCA1F820C0A5
:10067000CE8B06FB00FCBCFBF0F0C8830846217B58
:1006800001F01F01217345765FF0000104EB010CBE
:100690009CF808C002EA5C06ACEB060C0CF0FF0C00
:1006A0000CF0330603EA9C0CB44446180CEB1C1CFB
:1006B0000CF00F0C86F814C0467E491CB444C9B235
:1006C00080F819C00529E1D30CF0FF00252888BF68
:1006D000FFDF13F05BFAE8B3D4F80E106FF01F02DF
:1006E000080C02EA9126A0F5AA414FF01F0C5439DC
:1006F0001CBFA0F5AA41B1F155010AD0A0F52851BF
:10070000AA391EBFA0F52A41B1F1AA014FF0010993
:1007100001D14FF0000900221146012382EA0008AE
:100720006FEA080848EA0108B8F1FF3F18D006F060
:100730000108520842EAC83249080CF0010876085C
:100740005B1C41EAC8314FEA5C0C162BE6DDB9F1BF
:10075000000F00E000E003D084F88851BDE8F08786
:1007600084F88871BDE8F087B4F8B011B4F8B4210A
:10077000638804F17000A4F89850B4F89C40D2004B
:100780005C43B2FBF1F294FBF1F4521C848592B20B
:1007900002FB01F44285B4F5C84FC4BF521E428526
:1007A000BCFBF1F2521C0286428C01EBC202521ECB
:1007B000B2FBF1F20284C28B5A43B2FBF1F1C18366
:1007C000BDE8F0872DE9F04104460025A1B355238B
:1007D0004FF4FA464FF0330C01297DD0022900F086
:1007E000E180032918BFBDE8F08104F17000217B8E
:1007F00001F01F01217384F8895000216218127AD8
:1008000003EA5205521BD2B202F033050CEA9202FF
:100810002A44451802EB121202F00F022A75457E97
:10082000491C2A44C9B242760529E7D3D0B225280B
:1008300098BFBDE8F081B1E0FFE704F170068022C7
:1008400000213046FDF7E3FDB571F5713573757321
:10085000F57335747571B576F576212086F840000C
:10086000412086F84100FE2086F874002688702218
:1008700000212046FDF7CBFD2680012684F8646028
:1008800084F86560282084F86600002104F13000B7
:100890000DF09AF91B22A4F84E20A4F85020A4F8D9
:1008A0005220A4F854204FF4A470A4F85600A4F8E1
:1008B00058006673A4F8F850202084F8FA0084F8F1
:1008C000F050C4F8F45084F8245184F8255184F889
:1008D0002E5184F82F5100E005E084F8145184F87B
:1008E0002051BDE8F081618845480844B0FBF1F033
:1008F000A4F890004BF68030A4F89200E288A4F8A7
:100900009850B4F89C70D2004F43B2FBF1F297FBC1
:10091000F1F7521CA4F89C7092B202FB01F704F1AB
:100920007000A4F89A20B7F5C84FC4BF521E428584
:10093000B6FBF1F2521C028601F5802202F5EE327E
:10094000561EB6FBF1F20284C68B06FB01F2B2FB27
:10095000F1F1C1830146207B00F01F0020734D762A
:1009600000202218127A03EA5205521BD2B202F07A
:1009700033050CEA92022A440D1802EB121202F01F
:100980000F022A754D7E401C2A44C0B24A760528C3
:10099000E7D3D0B2252898BFBDE8F081FFDFBDE8DE
:1009A000F08100BFD0F81811628804F17003488903
:1009B000C989A4F89850B4F89CC0C9000CFB02FC8B
:1009C000B1FBF0F19CFBF0FC491CA4F89CC089B27F
:1009D00001FB00FCA4F89A10BCF5C84FC4BF491E27
:1009E0005985B6FBF0F1491C1986598C00EBC10101
:1009F000491EB1FBF0F11984D98B514302E000008C
:100A0000FFDB0500B1FBF0F0D883BDE8F0812DE9F4
:100A1000F003447E0CB1252C03D9BDE8F00312206D
:100A20007047002A02BF0020BDE8F003704791F82C
:100A30000DC01F260123F94D4FF00008BCF1000F37
:100A400074D0BCF1010F1EBF1F20BDE8F00370473A
:100A5000B0F800C00A7C8F7B91F80F907A404F7CF1
:100A600087EA090742EA072282EA0C0C5FF00007D6
:100A70000CF0FF094FEA1C2C99FAA9F99CFAACFC7E
:100A80004FEA19694FEA1C6C49EA0C2C0CEB0C1C60
:100A90007F1C9444FFB21FFA8CFC032FE8D38CEA2E
:100AA000020CDE4F0022ECFB057212096FF02405E8
:100AB00002FB05C2D2B201EBD207827602F0070533
:100AC0003F7A03FA05F52F4218BFC2767ED104FBA8
:100AD0000CF2120C521CD2B25FF0000400EB040CBA
:100AE0009CF814C094453CBFA2EB0C02D2B212D3C6
:100AF0000D194FF0000C2D7A03FA0CF73D421CBF84
:100B0000521ED2B2002A69D00CF1010C0CF0FF0C7D
:100B1000BCF1080FF0D304F1010C0CF0FF04052C1C
:100B2000DCD33046BDE8F0037047FFE790F81AC009
:100B30000C7E474604FB02C2B84C4FF0000CE2FBAF
:100B4000054C4FEA1C1C6FF024040CFB0422D2B2AB
:100B500001EBD204827602F0070C247A03FA0CFC33
:100B600014EA0C0F1FBFC2764046BDE8F003704781
:100B700090F819C0B2FBFCF40CFB1422521CD2B248
:100B80005FF0000400EB040C9CF814C094453CBFDB
:100B9000A2EB0C02D2B212D30D194FF0000C2D7A39
:100BA00003FA0CF815EA080F1CBF521ED2B272B13C
:100BB0000CF1010C0CF0FF0CBCF1080FF0D304F1A8
:100BC000010C0CF0FF04052CDCD3AAE709E00CEBC8
:100BD000C401C1763846BDE8F00370470CEBC40190
:100BE000C1764046BDE8F00370478D4A016812683F
:100BF00011408C4A126811430160704730B48A4931
:100C0000874B00244FF0010C0A78521CD2B20A70B4
:100C1000202A08BF0C700D781A680CFA05F52A42D4
:100C2000F2D0097802680CFA01F15140016030BC41
:100C3000704790F804C03CF01F011CBF00207047B3
:100C400030B40178552202EA5103C91AC9B201F041
:100C50003304332303EA91012144447801EB111159
:100C600002EA5405641BE4B204F0330503EA940479
:100C70002C4404EB141401F00F0104F00F040C4495
:100C80008178C07802EA5105491BC9B201F03305E9
:100C900003EA9101294401EB111101F00F012144F4
:100CA00002EA5004001BC0B200F0330403EA9000D3
:100CB000204400EB101000F00F00014402EA5C0039
:100CC000ACEB0000C0B200F0330203EA9000104425
:100CD00000EB101000F00F00084401288CBF012029
:100CE000002030BC70470A000ED00123012A0BDB24
:100CF000491EC9B210F801C0BCF1000F01D000209C
:100D000070475B1C9342F3DD01207047002A08BF47
:100D100070471144401E12F0010F03D011F8013D3D
:100D200000F8013F520808BF704700BF11F8013CAE
:100D3000437011F8023D00F8023F521EF6D1704791
:100D400070B58CB000F110041D4616460DF1FF3C45
:100D50005FF0080014F8012C8CF8012014F8022D23
:100D60000CF8022F401EF5D101F1100C6C460DF16C
:100D70000F0108201CF8012C4A701CF8022D01F804
:100D8000022F401EF6D1204612F00EFD7EB16A1EE3
:100D900004F130005FF0080110F8013C537010F8C6
:100DA000023D02F8023F491EF6D10CB070BD089812
:100DB0002860099868600A98A8600B98E8600CB0F1
:100DC00070BD38B505460C46684607F09CFB002808
:100DD00008BF38BD9DF900202272E07E607294F950
:100DE0000A100020511A48BF494295F82D308B4215
:100DF000C8BF38BDFF2B08BF38BDE17A491CC9B256
:100E0000E17295F82E30994203D8A17A7F2918BF54
:100E100038BDA2720020E072012038BD53E4B36EE9
:100E2000EC540200F0540200740000200C2818BF9B
:100E30000B2810D00D2818BF1F280CD0202818BF51
:100E4000212808D0222818BF232804D024281EBF18
:100E50002628002070474FF0010070470C2963D20C
:100E6000DFE801F006090E13161B323C415C484EC8
:100E7000002A5BD058E0072A18BF082A56D053E052
:100E80000C2A18BF0B2A51D04EE00D2A4ED04BE051
:100E9000A2F10F000C2849D946E023B1A2F11000BD
:100EA0000B2843D940E0122A18BF112A3ED090F8EF
:100EB000380020B1122A37D31A2A37D934E0162A3B
:100EC00032D31A2A32D92FE0A2F10F0103292DD9EA
:100ED00090F8380008B31B2A28D925E0002B08BF5A
:100EE000042A21D122E013B1062A1FD01CE0012AD6
:100EF0001AD11BE01C2A1CBF1D2A1E2A16D013E083
:100F00001F2A18BF202A11D0212A18BF222A0DD04B
:100F1000232A1CBF242A262A08D005E013B10E2A52
:100F200004D001E0052A01D000207047012070475D
:100F30002DE9F0410D460446866805F05FF858B982
:100F400004F0AEFE40F2367104F091FBA060204642
:100F500005F054F80028F3D095B13046A16805F0AB
:100F600097FB00280CDD2844401EB0FBF5F707FB7B
:100F700005F1304604F07BFBA0603846BDE8F08107
:100F80000020BDE8F08170B50446904228BF70BDD6
:100F9000101B64280BD325188D4206D8042105F0B8
:100FA000AAFB00281CBF284670BD204670BD6420E7
:100FB000F1E711F00C0F13D001F0040100290DBF6F
:100FC0004022102296214FF4167101F5BC71A0EB5E
:100FD000010388428CBF93FBF2F0002080B270477F
:100FE000022919BF6FF00D0101EBD0006FF00E0167
:100FF00001EB9000F2E7084418449830002A14BF2F
:1010000004210021084470470120704710680866D9
:10101000704710F0010F1CBF0120704710F0020F45
:101020001CBF0220704710F0040018BF0820704752
:101030002DE9F041054617468846012608460CF082
:101040001CFD044640460CF01CFD034610F0010F49
:1010500018BF012008D113F0020F18BF022003D1DE
:1010600013F0040018BF082014F0010F18BF4FF050
:10107000010C20D050EA0C0108BF002613F0030F2A
:1010800008BF002014F0030F08BF4FF0000C95F8C4
:101090006410814208BF0020387095F865106145E2
:1010A00008BF4FF0000C87F801C0002808BFBCF152
:1010B000000F1CD10DE014F0020F18BF4FF0020C0E
:1010C000D8D114F0040F14BF4FF0080C4FF0000CEF
:1010D000D0E740460CF0DBFCB5F87010401A00B2C7
:1010E00047F6FE71884201DC002800DC002630460D
:1010F000BDE8F08101281CBF02280020704718B409
:10110000CBB2C1F3072CC1B2C0F30720012B05D02D
:10111000022B08BFBCF1020F1BD002E0BCF1010F93
:1011200017D0012904D0022908BF022811D001E0FC
:1011300001280ED001EA0C0161F3070210EA030056
:1011400060F30F22D0B210F0020F18BF02200BD1B3
:1011500006E0084003EA0C01084060F30702EFE7ED
:1011600010F0010018BF01208DF80000C2F3072025
:1011700010F0020F18BF022003D110F0010018BFB9
:1011800001208DF80100BDF8000018BC7047162A38
:1011900010D12A220C2818BF0D280FD04FF0230C95
:1011A0001F280DD031B10878012818BF002805D0BC
:1011B000162805D000207047012070471A70FBE701
:1011C00083F800C0F8E7012902D0022905D007E022
:1011D000002804BF40F2E240704740F6C410704758
:1011E00000B5FFDF40F2E24000BD002A14BF4FF41B
:1011F00029614FF4A471002B14BF4FF429624FF4FE
:10120000A47200280CBF012000201144983100284E
:1012100018BF0420084470470178406829B190F84D
:101220002C1190F88C0038B901E001F0CFBC19B155
:10123000042901D0012070470020704770B50C468A
:101240000546062102F0CEFB606008B1002006E0F2
:101250000721284602F0C6FB606018B1012020700B
:10126000002070BD022070BD2DE9FC470C460646EB
:101270006946FFF7E3FF00287DD19DF8000050B1DB
:10128000FDF710FAB0427CD0214630460AF0B2F8A1
:10129000002873D12DE00CF0BFFDB04271D0214683
:1012A000304611F099FD002868D1019D95F8F000B5
:1012B00022E0012000E00020804695F839004FF040
:1012C000010A4FF00009F0B195F83A0080071AD5ED
:1012D00084F8019084F800A084F80490E68095F8E2
:1012E0003B102172A98F6181E98FA18185F8399026
:1012F00044E0019D95F82C0170350028DBD1287F52
:101300000028D8D0D5E7304602F0AFFC070000D166
:10131000FFDF384601F0BFFE40B184F801900F2195
:101320002170E680208184F804A027E0304602F096
:101330008AFC070000D1FFDFB8F1000F21D038464A
:1013400001F001FFB8B19DF8000038B90198D0F85C
:1013500018014188B14201D180F80090304607F071
:1013600029FC84F801900C21217084F80490E68017
:10137000697F217200E004E085F81C900120BDE83F
:10138000FC870020FBE71CB56946FFF757FF00B15B
:10139000FFDF684601F026FCFE4900208968A1F8BD
:1013A000F2001CBD2DE9FC4104460E46062002F069
:1013B000C1FA0546072002F0BDFA2844C7B200254D
:1013C000A8463E4417E02088401C80B22080B042EE
:1013D00002D34046A4F8008080B2B84204D3B042A1
:1013E00002D20020BDE8FC816946FFF727FF0028F4
:1013F000F8D06D1CEDB2AE42E5D84FF6FF702080FC
:101400001220EFE738B54FF6FF70ADF800000DE0A1
:101410000621BDF8000002F0F7FA04460721BDF8E6
:10142000000002F0F1FA0CB100B1FFDF00216846C4
:10143000FFF7B8FF0028EBD038BD70B507F028FCE7
:101440000BF0A2FBD44C4FF6FF7600252683668373
:10145000D2A0257001680079A4F14002657042F8BD
:10146000421FA11C1071601C11F0D3FD1B202081B4
:101470004FF4A4716181A081E1810321217761771B
:101480002174042262746082A082A4F13E00E18291
:1014900005704680BF480C300570A4F1100005703F
:1014A000468084F8205070BD70B5BA4C16460D4683
:1014B0006060217007F064FBFFF7A4FFFFF7BDFF3A
:1014C00020780FF008FBB7480CF0ECFD217860683D
:1014D00011F044FD20780AF08FFD284608F099FBB2
:1014E000B048FDF7EAF8217860680AF05DF8314607
:1014F000207811F0F1FFBDE870400BF045BB10B54E
:1015000001240AB1002010BD21B1012903D000241B
:10151000204610BD02210CF093F9F9E710B50378CD
:101520000446002B406813460A46014608D00120B5
:10153000FFF75BFE6168496A884203D9012010BD4C
:101540000020F5E7002010BD887800B90320C97895
:1015500001B90321107019700020704730B587B0B1
:10156000044600886946FFF769FE002806D1A08876
:1015700030B1012804D0022802D0122007B030BDBB
:1015800004AB03AA21466846FFF7DEFF0400F5D14D
:101590009DF80010012000250029019906D081F84E
:1015A000C101019991F80C1291BB29E081F82F013A
:1015B000019991F8561139B9019991F82E1119B97B
:1015C000019991F8971009B13A2415E0069501990F
:1015D00081F82E01019A9DF80C0082F83001019BE0
:1015E0009DF8102083F831218DF818008DF819200E
:1015F00006AA0020FFF70AFD019880F82F5122E08B
:10160000019991F8C01119B9019991F8971009B190
:101610003A2415E00695019981F8C001019A9DF8D8
:101620000C0082F8C201019B9DF8102083F8C321B1
:101630008DF818008DF8192006AA0120FFF7E6FCA6
:10164000019880F8C151204698E710B50446002063
:10165000A17801B90120E2780AB940F0020001F056
:10166000D0FA002803D12046BDE8104076E710BD2F
:1016700070B50D460446018900238088FFF7BBFC46
:10168000696A81421DD2401A401CA1884008091A8B
:101690008AB2A2802189081A2081668895F8641090
:1016A0001046FFF786FC864200D230466080E6880E
:1016B00095F865102089FFF77CFC864200D2304601
:1016C000E08070BDF0B585B00D46064603A9FFF772
:1016D000B5FD00282DD19DF80C0060B300220499BF
:1016E000FB20B1F84E30FB2B00D30346B1F850403D
:1016F000FB20FB2C00D30446DFF8ACC09CE8811033
:1017000000900197CDF808C0ADF80230ADF8064062
:101710006846FFF7ADFF6E80BDF80400E880BDF8B5
:1017200008006881BDF80200A880BDF80600288185
:10173000002005B0F0BD0122D1E72DE9F04186B0CF
:10174000044600886946FFF779FD00287ED121898B
:10175000E08801F070FA00287FD1A188608801F04C
:101760006AFA002879D12189E08801F05AFA002824
:1017700073D1A188608801F054FA07006DD12088E8
:1017800002A9FFF79FFF00B1FFDFBDF810106288CC
:1017900009200BE07800002018080020FFFFFFFF61
:1017A0001F000000D8060020F4540200914254D3D8
:1017B000BDF80C10E28891424FD3BDF81210BDF86D
:1017C0000E2023891144A2881A44914245D39DF8E2
:1017D0000010019D4FF00008012640F6480041B17D
:1017E00085F8B761019991F8F81105F5DB7541B9F4
:1017F0001AE085F82561019991F84A1105F592756D
:1018000009B13A2726E0E18869806188E980218969
:10181000814200D30146A980A188814200D20846B6
:101820002881012201990FE0E18869806188E980BF
:101830002189814200D30146A980A188814200D23A
:101840000846288101990022284600E005E0FFF7BC
:101850000FFF2E7085F80180384606B0BDE8F08194
:101860006BE770B504460CF08DFAB0B120781828FB
:1018700011D1207901280ED1E088062102F0B2F8BA
:10188000040008D0208807F095F92088062102F08E
:10189000BBF800B1FFDF012070BDF94D28780028AA
:1018A000FAD0002666701420207020223146201DB8
:1018B000FCF7ADFD022020712E70ECE710B5044658
:1018C000FCF766FE002813D0207817280FD1207966
:1018D00068B1E088072102F085F840B1008807F080
:1018E00069F9E088072102F08FF800B1FFDF0120DD
:1018F00010BD2DE9F0475FEA000800D1FFDFE048A6
:1019000002211A308146FFF74DFD00B1FFDFDC4CAC
:101910000620678B02F00EF80546072002F00AF851
:101920002844C5B2681CC6B2608BB04203D14046A1
:10193000FFF7C4FF58B9608BA84203D14046FFF7B8
:1019400090FF20B9608B4146FFF78EFC38B14046CE
:1019500001F07FF90028E7D10120BDE8F0870221DE
:101960004846FFF71FFD10B9608BB842DCD14046F6
:10197000BDE8F04711F0F6BD10B501F0CFF808B1A1
:101980000C2010BD0BF054F9002010BD10B504461A
:10199000007818B1012801D0122010BD01F0CFF855
:1019A00020B10BF097FA08B10C2010BD207801F09F
:1019B0008FF8E21D04F11703611CBDE810400BF025
:1019C000B1B910B5044601F0A9F808B10C2010BD5A
:1019D000207828B1012803D0FF280BD0122010BD99
:1019E00001F076F8611C0BF0E3F808B1002010BD9F
:1019F000072010BD01200BF015F9F7E710B50BF02B
:101A00006CFA08B1002010BD302010BD10B504469E
:101A100001F095F808B10C2010BD20460BF057FAE4
:101A2000002010BD10B501F08AF820B10BF052FA79
:101A300008B10C2010BD0BF0CDF9002010BDFF2126
:101A400081704FF6FF7181808E4949680A788271F2
:101A50008A880281498841810121417000207047B4
:101A60001CB5002412F1080F15D00CDC12F1280F60
:101A700011D012F1140F0ED012F1100F0BD012F181
:101A80000C0F0ED107E012F1040F04D01AB1032A93
:101A900001D0042A05D1012806D0022808D0032845
:101AA0000AD0122420461CBD1046FDF775F9F9E74F
:101AB00010460CF0F2FAF5E7084614466946FFF7BF
:101AC000BDFB08B10224EDE79DF80000019880F805
:101AD00067400024E6E710B513460122FFF730F90E
:101AE000002010BD10B504460FF0BAFD052804D043
:101AF00020460EF0DFFF002010BD0C2010BD10B5F9
:101B0000044601F01CF808B10C2010BD214600204D
:101B100007F0BFF8002010BD10B504460FF059F8CB
:101B200050B108F0F0FA38B1207808F07EF820784B
:101B30000CF074FD002010BD0C2010BD10B5044643
:101B400000F0FDFF08B10C2010BD2146012007F078
:101B5000A0F8002010BD38B504464FF6FF70ADF870
:101B60000000A079E179884216D02079FCF77CFC4E
:101B700090B16079FCF778FC70B10022A079114631
:101B800012F0ECF840B90022E079114612F0E6F8C4
:101B900010B9207A072801D9122038BD08F0C0FA00
:101BA00060B90FF05DFD48B900216846FFF7FAFB08
:101BB00020B1204605F0C8FF002038BD0C2038BDFC
:101BC0002DE9FC41817805461A2925D00EDC16291D
:101BD0002ED2DFE801F02D2D2D2D2D212D2D2D2D97
:101BE0002D2D2D2D2D2D2D2D2D2121212A291FD0BB
:101BF0000BDCA1F11E010C291AD2DFE801F0191942
:101C00001919191919191919190D3A3904290FD265
:101C1000DFE801F00E020E022888B0F5706F07D2DF
:101C200001276946FFF70AFB20B10220BDE8FC81CD
:101C30001220FBE79DF8000000F051FF019C10B15D
:101C400004F58A7401E004F5C6749DF8000000F004
:101C500046FF019E10B106F2151601E006F28D1640
:101C60006846FFF7D9FA08B1207808B10C20DDE703
:101C70002770A8783070684600F0B4FF0020D5E7E0
:101C800018080020780000207CB50D466946FFF753
:101C9000D5FA002618B12E602E7102207CBD9DF869
:101CA000000000F01CFF019C9DF80000703400F063
:101CB00016FF019884F8426081682960017B2971D0
:101CC00094F842100029F5D100207CBD10B50446DF
:101CD00000F035FF20B10BF0FDF808B10C2010BD6D
:101CE000207800F0F5FEE279611C0BF06FFA08B184
:101CF000002010BD022010BD10B5886E60B100221A
:101D000041F8682F0120CA718979884012F01AF8C9
:101D1000002800D01F2010BD0C2010BD1CB50C46A3
:101D20006946FFF78BFA002809D19DF800000028CA
:101D30000198B0F8700000D0401C208000201CBD2D
:101D40001CB5044600886946FFF778FA08B10220FE
:101D50001CBD606828B1DDE90001224600F0CDFF1E
:101D60001CBDDDE90001FFF7C7FF1CBD2DE9F041F7
:101D700004460078012804D018B1022801D00328B5
:101D80001ED1607828B1012803D0022801D0032891
:101D900016D1E07B10B9A078012811D1A07830F0DD
:101DA00005020DD110F0050F0AD0400801D0112016
:101DB00054E5E078E68862890F4618B1012801D021
:101DC00012204BE5104600F0D6FF302558B13946B9
:101DD000304600F0DAFF30B1A07B0028F0D00728B1
:101DE000EED800203AE5284638E51FB5044600F055
:101DF0008AFE10B10C2004B010BD022104F10A00CB
:101E000000F0CDFFA0788DF80800A0788DF80000D4
:101E100060788DF8040020788DF80300A07B8DF8A1
:101E20000500E07B00B101208DF80600A078C00716
:101E30000CD0E078012812D098B100208DF8010074
:101E4000E088ADF80A006089ADF80C0002A80EF039
:101E5000CCFE0028CFD168460CF0E5FBCBE7022092
:101E6000ECE70120EAE710B504460121FFF77EFF09
:101E7000002803D12046BDE81040B6E710BD027827
:101E8000012A01D0BAB118E042783AB1012A05D04E
:101E9000022A12D189B1818879B100E059B1418813
:101EA00049B1808838B101EB8101490000EB800025
:101EB000B1EB002F01D2002070471220704770B59F
:101EC000044600780D46012809D00FF0C9FB05280B
:101ED00003D00EF09AFD002800D00C2070BD0CF04D
:101EE00096FA88B10CF0A8FA0CF07DFB0028F5D129
:101EF00025B160780CF02EFB0028EFD1A188608816
:101F0000BDE870400EF08CBE122070BD10B50446C6
:101F10000121FFF7B4FF002804D12046BDE810409E
:101F20000121CCE710BDF0B5871FDDE9056540F65E
:101F30007B44A74213D28F1FA74210D288420ED8EB
:101F4000B2F5FA7F0BD2A3F10A00241FA04206D2F9
:101F5000521C4A43B2EB830F01DAAE4201D9002092
:101F6000F0BD0120F0BD2DE9FC41477A88460446CA
:101F700017F0050F73D0F80871D1780701D511203B
:101F800054E694F83A0008B9012F68D100252E468E
:101F9000F8071BD088F00105208A294600F0EBFEE7
:101FA00048B36089294600F0F0FE20B3208A618999
:101FB000884254D8A18EE08DCDE90001238D628C3A
:101FC000A18BE08AFFF7AFFFA8B10125B8070ED5B6
:101FD00004EB4500828EC18DCDE90012038D428C49
:101FE000818BC08AFFF79FFF28B12E466D1CB8F188
:101FF000000F02D023E0302018E6228A012119E0E8
:10200000B14203D004EB4100008A024404EB4100DA
:10201000C38A878ABB4222D1838B478BBB421ED1A6
:10202000438C078CBB421AD1038DC08C834216D1DE
:10203000491CC9B2A942E3D3608990420FD32078EA
:1020400010B101280BD102E0A0780028F9D1607806
:1020500038B1012805D0022803D0032801D012206E
:10206000E4E50020E2E500217DE70178C90702D020
:10207000406811F04ABA11F017BA10B5007801287B
:1020800000D00020FCF783FE002010BD2DE9F047B2
:1020900088B00D46AFF6FC02D2E9009201469046A8
:1020A0002846FFF760FF06000CD100F02CFD40B978
:1020B000FE4F387828B90BF0AFFEA0F57F41FF390D
:1020C00002D00C2008B048E4032105F1100000F014
:1020D00066FEF64801AA3E380190F5480290F348A2
:1020E00006211038039006A801F04AFC040037D0FE
:1020F0000021FEF767FB04F130017B8ABA8ACB83AB
